:020000040800F2
:10000000B0AE0020A1020008E5C70008DDAA000884
:10001000F1C2000815350008C1FB0008000000000F
:1000200000000000000000000000000011D30008E4
:10003000C55000080000000051CD0008E9E30008A9
:10004000BB020008BB020008BB020008BB0200089C
:10005000BB020008BB020008C9500008BB02000830
:10006000BB020008D5500008E1500008BB020008A0
:10007000014B0008114B0008BB020008BB0200083E
:10008000BB020008BB020008BB02000839350008AB
:100090001935000829350008BB020008ED5000089A
:1000A000BB020008BB020008BB020008BB0200083C
:1000B000BB020008BB020008BB020008BB0200082C
:1000C000BB020008BB020008BB020008BB0200081C
:1000D000BB020008BB020008BB020008BB0200080C
:1000E000BB020008BB020008BB020008BB020008FC
:1000F000BB020008BB020008BB020008BB020008EC
:10010000BB020008BB020008BB020008BB020008DB
:10011000BB020008BB020008BB020008BB020008CB
:10012000BB020008214B0008314B0008414B00087E
:10013000BB020008BB020008BB02000869350008CA
:100140004935000859350008BB020008BB02000809
:10015000BB020008514B0008BB020008A5FB0008C9
:10016000BB020008BB020008BB020008BB0200087B
:10017000BB020008BB020008BB0200080000000030
:10018000BB020008BB02000800F002F800F05EF8B5
:100190000AA090E8000C82448344AAF10107DA45E2
:1001A00001D100F053F8AFF2090EBAE80F0013F0D6
:1001B000010F18BFFB1A43F0010318474460010008
:1001C000646001000A444FF0000C10F8013B13F08A
:1001D000070408BF10F8014B1D1108BF10F8015BA0
:1001E000641E05D010F8016B641E01F8016BF9D193
:1001F00013F0080F1EBF10F8014BAD1C0C1B09D1EA
:100200006D1E58BF01F801CBFAD505E014F8016B5B
:1002100001F8016B6D1EF9D59142D6D370470000ED
:100220000023002400250026103A28BF78C1FBD8FF
:10023000520728BF30C148BF0B6070471FB515F08B
:1002400040FE00F0DAF81FBD10B510BD00F09AF9BD
:100250001146FFF7F3FF0FF095FE00F0B8F903B475
:10026000FFF7F2FF03BC00F0BBF900000B49D1F827
:1002700000C04A685CF8043B1068184442F8040B5C
:100280008C4528BFA1F1DC0C8A4228BFA1F1DC0219
:10029000C1F800C04A6020F0004070474C040020C4
:1002A0000948804709480047FEE7FEE7FEE7FEE70A
:1002B000FEE7FEE7FEE7FEE7FEE7FEE70448054946
:1002C000054A064B70470000BDE40008890100089C
:1002D000B08E0020B0AE0020B09E0020B09E002066
:1002E00053EA020C00F069802DE9F04B4FF0000654
:1002F000002B1FBFB3FA83F503FA05F424FA05F6C1
:100300005E4012BF1643B2FA82F502FA05F4C5F157
:1003100020051EBF22FA05FC44EA0C04203556EAEB
:10032000044C4FEA144418BF641C4FF000084FF00F
:100330000009904271EB030C39D3002919BFB1FABF
:1003400081F701FA07F6B0FA80F700FA07F6C7F16D
:1003500020071EBF20FA07FC46EA0C062037B6FB32
:10036000F4FCA7EB0507103F07F01F0BCBF12006AD
:100370002CFA06F60CFA0BFB44BFB3460026202FDE
:10038000A4BF5E464FF0000B5BEA060C08BF4FF0BF
:10039000010B19EB0B0948EB0608ABFB027C06FBD3
:1003A00002CC0BFB03CCC01B71EB0C01C1E70B466D
:1003B000024641464846BDE8F08B13B5084318BFD6
:1003C0004FF0FF300146AFF30080BDE81C4070479E
:1003D0000B4910B5A1F17C020A4CC2E93712372152
:1003E00006E000EB104342F82130074B00FB0340CE
:1003F0000B1EA1F10101F4DC10BD0120E8E70000B3
:10040000EC030020E119D666CD0D0100032A40F26D
:10041000308010F0030C00F0158011F8013BBCF1A6
:10042000020F624498BF11F801CB00F8013B38BFBE
:1004300011F8013BA2F1040298BF00F801CB38BFCC
:1004400000F8013B11F0030300F02580083AC0F0EA
:10045000088051F8043B083A51F804CBA0E8081092
:10046000F5E7121D5CBF51F8043B40F8043BAFF3C5
:100470000080D20724BF11F8013B11F801CB48BF1F
:1004800011F8012B24BF00F8013B00F801CB48BF55
:1004900000F8012B704710B5203AC0F00B80B1E88E
:1004A0001850A0E81850B1E81850A0E81850203AA9
:1004B000BFF4F5AF5FEA027C24BFB1E81850A0E8B2
:1004C000185044BF18C918C0BDE810405FEA827CCC
:1004D00024BF51F8043B40F8043B08BF7047D207E3
:1004E00028BF31F8023B48BF11F8012B28BF20F884
:1004F000023B48BF00F8012B704702F0FF0343EABC
:10050000032242EA024200F002B84FF0000200B5B6
:10051000134694469646203922BFA0E80C50A0E826
:100520000C50B1F12001BFF4F7AF090728BFA0E8D4
:100530000C5048BF0CC05DF804EB890028BF40F8A0
:10054000042B08BF704748BF20F8022B11F0804FE2
:1005500018BF00F8012B704770477047704710B5FF
:1005600000F008F8006810BD10B5044600F002F86D
:10057000046010BD004870475404002000487047D4
:10058000540400207546FFF7F9FFAE4605006946A2
:10059000534620F00700854618B020B5FFF78EFEC1
:1005A000BDE820404FF000064FF000074FF0000874
:1005B0004FF0000BAC46ACE8C009ACE8C009ACE8B1
:1005C000C009ACE8C00921F007018D46704710B59D
:1005D0000446AFF300802046BDE81040FFF73FBE61
:1005E00001491820ABBEFEE726000200704700005C
:1005F00080B58AB008900791089820B9FFE7FF20DE
:100600008DF827009BE0079820B9FFE7FF208DF8C1
:10061000270094E0079890ED000A90ED013A90EDE4
:10062000021A90ED032A20EE030A21EE021A30EEA0
:10063000010A30EE000A8DED060A079890ED010AD6
:1006400090ED021A20EE000A21EE011A30EE010AA6
:1006500030EE001AB7EE000A8DED010A30EE410AC5
:100660008DED050A9DED060ADDED050A14F0B0F9E1
:100670009DED011A089880ED010A079890ED000A97
:1006800090ED013A90ED024A90ED032A20EE040A23
:1006900022EE032A30EE420A30EE000A8DED040A03
:1006A0009DED040AB0EEC00AB4EE410AF1EE10FA74
:1006B0000ADBFFE7DDED040A9FED230A0FF0AAFB3A
:1006C000089880ED020A07E09DED040A13F07EFE13
:1006D000089880ED020AFFE7079890ED000A90ED78
:1006E000011A90ED022A90ED033A20EE030A21EE62
:1006F000021A30EE010A30EE000A8DED030A079867
:1007000090ED020A90ED031A20EE000A21EE011A84
:1007100030EE010A30EE001AB7EE000A30EE410A60
:100720008DED020A9DED030ADDED020A14F050F989
:10073000089880ED000A00208DF82700FFE79DF95A
:1007400027000AB080BD00BFDB0FC93F80B58CB069
:100750000A9009918DED080A0A9820B9FFE7FF2059
:100760008DF82F0029E19DED081AB7EE000A80EE02
:10077000010A0A9880ED040A0A994FF07E50086039
:100780000A99002048600A9988600A99C860099807
:10079000002800F00E81FFE7099801680091406889
:1007A00015F0EEFA0246009801920A46019942ECD1
:1007B000101B8DED020B15F0E3FA9DED020B41ECE1
:1007C000110B14F005F88DED040B9DF8170080F067
:1007D00080008DF817000498059914F01DFE07900D
:1007E000099890ED000AB5EE400AF1EE10FA2BD10F
:1007F000FFE7099890ED010AB5EE400AF1EE10FA14
:1008000022D1FFE7099890ED020AB5EE400AF1EE19
:1008100010FA19D1FFE70A9940F2C560C3F64D708E
:1008200008600A9944F62D20C3F60D4048600A99E5
:100830004AF25640CBF6393088600A9944F2AD70DE
:10084000C3F61970C860B3E09DED070A9FED5D1A0D
:10085000B4EE410AF1EE10FA08DBFFE79DED070A5E
:10086000B5EE400AF1EE10FA19DDFFE70A9945F6F8
:100870006E10C3F67F7008600A9945F20C30C3F61B
:10088000B01048600A9948F6AB00CBF6BB308860E0
:100890000A9949F28550C3F69750C86087E09DEDEC
:1008A000070A9FED491AB4EE410AF1EE10FA0ADB8D
:1008B000FFE79DED070A9FED431AB4EE410AF1EE02
:1008C00010FA19DDFFE70A9940F2C560C3F64D70D2
:1008D00008600A9944F62D20C3F60D4048600A9935
:1008E0004AF25640CBF6393088600A9944F2AD702E
:1008F000C3F61970C86059E09DED070A9FED331AE1
:10090000B4EE410AF1EE10FA0ADBFFE79DED070AAB
:100910009FED2D1AB4EE410AF1EE10FA19DDFFE752
:100920000A9940F2C560C3F64D7008600A9944F612
:100930002D20C3F60D4048600A994AF25640CBF686
:10094000393088600A9944F2AD70C3F61970C860F6
:100950002BE09DED070A9FED1D1AB4EE410AF1EE62
:1009600010FA08DBFFE79DED070AB5EE400AF1EE4D
:1009700010FA19DDFFE70A9940F2C560C3F64D7021
:1009800008600A9944F62D20C3F60D4048600A9984
:100990004AF25640CBF6393088600A9944F2AD707D
:1009A000C3F61970C860FFE7FFE7FFE7FFE7FFE75F
:1009B000FFE700208DF82F00FFE79DF92F000CB016
:1009C00080BD00BFDB0FC93FDB0F49400000B442D0
:1009D00081B000900099002088604860086001B0F4
:1009E0007047000080B52DED048BB2B030902F9190
:1009F0002E922D93309828B9FFE7FF208DF8C7007D
:100A000000F0F7BD2F9828B9FFE7FF208DF8C70049
:100A100000F0EFBD2E9828B9FFE7FF208DF8C70042
:100A200000F0E7BD40F27401C2F200014EF69E7084
:100A3000C3F6275008602D9848B9FFE730982F99E2
:100A40002E9A00F0DDFD8DF8C70000F0D2BD2D9884
:100A5000006809902D98406808902D98806807904C
:100A60009DED090AB5EE400AF1EE10FA19D1FFE743
:100A70009DED080AB5EE400AF1EE10FA11D1FFE73C
:100A80009DED070AB5EE400AF1EE10FA09D1FFE735
:100A900030982F992E9A00F0B3FD8DF8C70000F022
:100AA000A8BD2F98006806902F98406805902F9851
:100AB000806804902E98006803902E9840680290F9
:100AC0002E988068019030989DED033A90ED010AD0
:100AD00090ED022A90ED031A20EE430A9DED023AB2
:100AE00022EE032A30EE420A9DED012A21EE021A7F
:100AF00030EE410AB6EE001A20EE010A8DED270A0B
:100B000030989DED034A90ED000A90ED023A90ED89
:100B1000032A20EE040A9DED014A23EE043A30EE4A
:100B2000030A9DED023A22EE032A30EE420A20EE3D
:100B3000010A8DED260A30989DED024A90ED000ADB
:100B400090ED013A90ED032A20EE040A9DED014A52
:100B500023EE043A30EE430A9DED033A22EE032AD7
:100B600030EE020A20EE010A8DED250A30989DED47
:100B7000014A90ED000A90ED013A90ED022A20EE34
:100B8000040A9DED024A23EE043A30EE030A9DED7D
:100B9000033A22EE032A30EE420A20EE010A8DEDDE
:100BA000240A9DED060AB5EE400AF1EE10FA11D1C5
:100BB000FFE79DED050AB5EE400AF1EE10FA09D106
:100BC000FFE79DED040AB5EE400AF1EE10FA00F0E1
:100BD0009984FFE79DED060A20EE000A9DED051AB7
:100BE00021EE011A30EE010A9DED041A21EE011AE0
:100BF00030EE010A09F074FF8DED2C0A9DED2C1AE0
:100C00009DED060A20EE010A8DED060A9DED2C1AD7
:100C10009DED050A20EE010A8DED050A9DED2C1AC9
:100C20009DED040A20EE010A8DED040A9DED090AEE
:100C300020EE000A9DED081A21EE011A30EE010A9D
:100C40009DED071A21EE011A30EE010A09F048FF66
:100C50008DED2C0A9DED2C1A9DED090A20EE010A5E
:100C60008DED090A9DED2C1A9DED080A20EE010A72
:100C70008DED080A9DED2C1A9DED070A20EE010A64
:100C80008DED070A309890ED000A30EE000A9DEDD8
:100C9000091A20EE010A8DED210A309890ED000A24
:100CA00030EE000A9DED081A20EE010A8DED200AB3
:100CB000309890ED000A30EE000A9DED071A20EE04
:100CC000010A8DED1F0A309890ED010A30EE000AFE
:100CD0009DED091A20EE010A8DED1E0A309890ED67
:100CE000000A30EE000A8DED190A309890ED010AE5
:100CF00030EE000A8DED180A309890ED020A30EEC1
:100D0000000A8DED170A309890ED030A30EE000AC4
:100D10008DED160A309890ED000A90ED021A30EE33
:100D2000000A20EE010A8DED150A309890ED020AB6
:100D300090ED031A30EE000A20EE010A8DED140A40
:100D4000309890ED000A20EE000A8DED130A3098DD
:100D500090ED000A90ED011A20EE010A8DED120AC5
:100D6000309890ED000A90ED021A20EE010A8DED08
:100D7000110A309890ED000A90ED031A20EE010A56
:100D80008DED100A309890ED010A20EE000A8DEDED
:100D90000F0A309890ED010A90ED021A20EE010A38
:100DA0008DED0E0A309890ED010A90ED031A20EEB9
:100DB000010A8DED0D0A309890ED020A20EE000A2E
:100DC0008DED0C0A309890ED020A90ED031A20EE9A
:100DD000010A8DED0B0A309890ED030A20EE000A0F
:100DE0008DED0A0A9DED091A9DED130A21EE000A08
:100DF0009DED202A309890ED025A90ED033A22EEB4
:100E0000032A30EE420A9DED1F2A22EE052A30EE1B
:100E1000020A9DED0F2A21EE022A30EE020A9DED14
:100E2000182A9DED084A22EE044A24EE054A30EEC7
:100E3000040A9DED074A22EE042A22EE032A30EE30
:100E4000020A9DED0C2A21EE022A30EE420A9DEDA7
:100E50000A2A21EE021A30EE410A8DED230A9DED99
:100E6000210A309890ED015A90ED024A90ED033A34
:100E700020EE030A9DED081A9DED132A21EE022AA9
:100E800030EE020A9DED1F2A22EE052A30EE420ABC
:100E90009DED1E2A22EE042A30EE020A9DED0F2A55
:100EA00021EE022A30EE420A9DED0C2A21EE022AA2
:100EB00030EE020A9DED172A9DED074A22EE042A24
:100EC00022EE032A30EE020A9DED0A2A21EE021AD2
:100ED00030EE410A8DED220A9DED230A20EE000A34
:100EE0009DED221A21EE011A30EE010A09F0F8FDFB
:100EF000B7EE006A86EE000A8DED1D0A9DED210A0F
:100F0000309890ED012A90ED021A90ED033A20EE10
:100F1000011A9DED200A20EE020A30EE412A9DEDD5
:100F2000071A9DED130A21EE000A30EE022A9DED0C
:100F30001E0A20EE030A30EE020A9DED0F2A21EE72
:100F4000022A30EE420A9DED172A9DED084A22EE54
:100F5000042A22EE032A30EE020A9DED0C2A21EE2D
:100F6000022A30EE420A9DED0A2A21EE021A30EEE4
:100F7000010A8DED1C0A9DED1D0A30EE000A8DED73
:100F80001B0A9DED1C0A30EE000A8DED1A0A9DED3C
:100F9000170ADDED0D0A30EEA02A9DED151A31EE8F
:100FA000422A9DED061A31EE021A20EE010A9DED4D
:100FB000181ADDED123A33EEA32A9DED143A32EE03
:100FC000032A9DED053A32EE432A21EE021A70EE15
:100FD000014A9DED1C3A309890ED011A90ED020AFD
:100FE000D0ED032A63EE001A9DED1D2A9DED0C7ACB
:100FF000B6EE004A8DED004A77EE445A9DED0A5A4E
:1010000035EE255A62EE055A9DED115A75EE606A6D
:1010100063EE266A75EEA66ADDED095A75EEA65AEC
:1010200061EEA51A71EEA41A62EE222A23EE011ACD
:1010300031EE621ADDED0E2ADDED104A72EEE42A81
:1010400062EE222ADDED0B4A73EEA43A63EE233AF8
:1010500072EEA32ADDED083A72EEE32A21EE221A9F
:1010600031EE211A22EE000A35EE205A22EE052A30
:101070009DED0F5A34EE455A35EE475A23EE053AA8
:1010800032EE032A9DED073A32EE432A20EE020AA1
:1010900030EE010A8DED2B0A9DED160ADDED0D2ACD
:1010A00032EEA21A9DED152A31EE421A9DED062A66
:1010B00031EE421A20EE010A9DED191ADDED126A99
:1010C00036EEA62A9DED143A32EE032A9DED053A3E
:1010D00032EE432A21EE021A30EE011A3098D0ED9A
:1010E000005AD0ED014AD0ED023A90ED032AB1EE5C
:1010F000000A24EE803A9DED0F7A37EE075A75EE1E
:10110000461ADDED0C0A30EEA05A75EE211A9DED5F
:10111000045A35EE215A23EE053A31EE031A9DEDBD
:101120001C5A65EE027A9DED1D3A74EE601A9DED33
:101130000A8A71EEC81A23EE218ADDED111A32EE09
:10114000E19A25EE099A38EE098A9DED099A38EE62
:10115000498A67EE887A31EE271A63EE233A65EE04
:10116000255A73EEA53ADDED0E5ADDED107A75EED7
:10117000E75A63EE255ADDED0B7A76EEA76A65EE47
:10118000266A75EEA65ADDED086A75EEE65A63EE3C
:10119000A53A31EE231A23EE022ADDED1A3A63EE68
:1011A000A43A32EE632A71EEA21A23EE213A34EE0B
:1011B000477A37EE607A25EE075A33EE053A9DED11
:1011C000075A33EE453A22EE032A31EE021A8DED2C
:1011D0002A1A9DED191ADDED0D0A30EEA03A9DEDAB
:1011E000152A32EE433A9DED062A32EE032A21EE0D
:1011F000021A9DED162ADDED124A34EEA43A9DED59
:10120000145A33EE053A9DED055A33EE453A22EE77
:10121000032A31EE022A309890ED001AD0ED011A1F
:10122000D0ED022AD0ED033A22EE800A9DED0F5A4E
:1012300035EE053A33EE467A9DED0C6A36EE063A07
:1012400033EE077A9DED043A33EE073A20EE030AB7
:1012500070EE025A9DED1B0A20EE620A9DED1C3ACB
:1012600023EE012A30EE420A9DED1D2A34EE467A25
:10127000DDED0A6A37EE667A62EE076A9DED117A55
:1012800070EEC77A63EE277A76EEA76ADDED097A0B
:1012900076EEE76A20EE260A30EE250A62EE211A83
:1012A00063EE233A71EEA31ADDED0E3ADDED105A2E
:1012B00073EEE53A62EE233ADDED0B5A74EEA54A81
:1012C00063EE244A73EEA43ADDED084A73EEE43A85
:1012D00061EEA31A30EE210A22EE011ADDED1A1A90
:1012E00061EEA21A31EE611A37EE207A22EE072A59
:1012F00034EE455A35EE465A23EE053A32EE032ACD
:101300009DED073A32EE432A21EE021A30EE010A31
:101310008DED290A9DED180A9DED0D7A37EE071A1D
:101320009DED152A31EE421A9DED062A31EE421A44
:1013300020EE010A9DED171ADDED122A32EEA22AE7
:101340009DED143A32EE032A9DED053A32EE432A22
:1013500021EE021A70EE013A9DED1B1A3098D0ED85
:10136000001A90ED010AD0ED020A90ED032A21EE59
:10137000022A9DED1C3A23EE001A31EE421A9DED31
:101380001D2A9DED0C5A34EE456ADDED0A4A36EE13
:10139000646A62EE064A9DED116A77EE465A63EE84
:1013A000255A74EEA54ADDED095A74EEE54A21EEA0
:1013B000241A31EE231A62EE211A63EE200A70EE2F
:1013C000E10ADDED0E1ADDED103A71EEE31A62EE80
:1013D000211ADDED0B3A72EEA32A63EE222A71EE9A
:1013E000A21ADDED082A71EEE21A60EEA10A31EED2
:1013F000201A22EE000A36EE076A22EE062A9DED3A
:101400000F6A34EE464A34EE454A23EE043A32EE91
:10141000032A9DED073A32EE432A20EE020A30EE0F
:10142000010A8DED280A9DED2B0A20EE000A9DEDA4
:101430002A1A21EE011A30EE010A9DED291A21EE39
:10144000011A30EE010A9DED281A21EE011A30EE44
:10145000010A09F045FB8DED2C0A9DED2C1A9DED3E
:101460002B0A20EE010A8DED2B0A9DED2C1A9DED25
:101470002A0A20EE010A8DED2A0A9DED2C1A9DED17
:10148000290A20EE010A8DED290A9DED2C1A9DED09
:10149000280A20EE010A8DED280A40F27400C2F2FB
:1014A000000090ED000A9DED2B1A20EE011A9DED33
:1014B000270A30EE410A8DED270A90ED000A9DEDD6
:1014C0002A1A20EE011A9DED260A30EE410A8DED12
:1014D000260A90ED000A9DED291A20EE011A9DEDD5
:1014E000250A30EE410A8DED250A90ED000A9DEDAA
:1014F000281A20EE011A9DED240A30EE410A8DEDE6
:10150000240AFFE79DED271A309890ED000A90ED30
:10151000042A21EE021A30EE010A80ED000A9DED48
:10152000261A309890ED010A90ED042A21EE021A55
:1015300030EE010A80ED010A9DED251A309890EDFC
:10154000020A90ED042A21EE021A30EE010A80ED23
:10155000020A9DED241A309890ED030A90ED042ABA
:1015600021EE021A30EE010A80ED030A309890ED68
:10157000000A90ED013A90ED022A90ED031A20EE58
:10158000000A23EE033A30EE030A22EE022A30EE7E
:10159000020A21EE011A30EE010A09F0A1FA8DEDDE
:1015A0002C0A9DED2C1A309890ED000A20EE010ACD
:1015B00080ED000A9DED2C1A309890ED010A20EE86
:1015C000010A80ED010A9DED2C1A309890ED020A77
:1015D00020EE010A80ED020A9DED2C1A309890ED64
:1015E000030A20EE010A80ED030A00208DF8C700EF
:1015F000FFE79DF9C70032B0BDEC048B80BD000051
:1016000080B5A0B01E901D911C921E9820B9FFE7D6
:10161000FF208DF87F00D3E21D9820B9FFE7FF205F
:101620008DF87F00CCE21C9820B9FFE7FF208DF8F1
:101630007F00C5E240F27401C2F2000142F60230BE
:10164000C3F6075008601D9800681B901D984068FD
:101650001A901D98806819901C98006818901C9822
:10166000406817901C98806816901E989DED183A57
:1016700090ED010A90ED022A90ED031A20EE430A44
:101680009DED173A22EE032A30EE420A9DED162A0E
:1016900021EE021A30EE410AB6EE001A20EE010ADF
:1016A0008DED100A1E989DED184A90ED000A90ED00
:1016B000023A90ED032A20EE040A9DED164A23EE2D
:1016C000043A30EE030A9DED173A22EE032A30EE7B
:1016D000420A20EE010A8DED0F0A1E989DED174A71
:1016E00090ED000A90ED013A90ED032A20EE040AF5
:1016F0009DED164A23EE043A30EE430A9DED183A6A
:1017000022EE032A30EE020A20EE010A8DED0E0AC7
:101710001E989DED164A90ED000A90ED013A90ED6D
:10172000022A20EE040A9DED174A23EE043A30EE19
:10173000030A9DED183A22EE032A30EE420A20EE0B
:10174000010A8DED0D0A9DED1B0AB5EE400AF1EE82
:1017500010FA11D1FFE79DED1A0AB5EE400AF1EE3D
:1017600010FA09D1FFE79DED190AB5EE400AF1EE36
:1017700010FA00F0AE81FFE79DED1B0A20EE000A93
:101780009DED1A1A21EE011A30EE010A9DED191A8B
:1017900021EE011A30EE010A09F0A2F98DED150AC9
:1017A0009DED151A9DED1B0A20EE010A8DED1B0A19
:1017B0009DED151A9DED1A0A20EE010A8DED1A0A0B
:1017C0009DED151A9DED190A20EE010A8DED190AFD
:1017D0001E9890ED000A30EE000A8DED0C0A1E985E
:1017E00090ED010A30EE000A8DED0B0A1E9890ED87
:1017F000020A30EE000A8DED0A0A1E9890ED030AE7
:1018000030EE000A8DED090A1E9890ED000AB1EE47
:10181000003A20EE030A8DED080A1E9890ED010AA9
:1018200020EE030A8DED070A1E9890ED020A20EEC5
:10183000030A8DED060A1E9890ED010AB2EE001A19
:1018400020EE010A8DED050A1E9890ED020A20EEA9
:10185000010A8DED040A1E9890ED000A20EE000AA0
:101860008DED030A1E9890ED010A20EE000A8DED21
:10187000020A1E9890ED020A20EE000A8DED010A80
:101880001E9890ED030A20EE000A8DED000A9DEDF2
:10189000081A9DED010A21EE000A9DED0A2A9DED30
:1018A0001B4A22EE042A30EE020A9DED022A21EEA6
:1018B000021A30EE010A9DED0B1A9DED1A2A21EE57
:1018C000021A30EE410A8DED140A9DED071A9DEDC6
:1018D000000A21EE000A9DED092A9DED1B4A22EE29
:1018E000042A30EE420A9DED032A22EE032A1E98B6
:1018F00090ED014A22EE042A30EE020A9DED0C2AF8
:101900009DED1A4A22EE042A30EE420A30EE410AD8
:101910009DED052A9DED024A22EE044A30EE040AAE
:101920009DED014A22EE042A30EE020A9DED192AAD
:1019300021EE021A30EE010A8DED130A9DED030A25
:1019400020EE030A1E9890ED021A20EE010A9DED8A
:101950000C1A9DED1B2A21EE021A30EE010A9DEDB4
:10196000061A9DED002A21EE022A30EE020A9DEDB4
:10197000092A9DED1A4A22EE042A30EE420A30EE80
:10198000410A9DED042A9DED024A22EE044A30EE02
:10199000040A9DED014A22EE042A30EE020A9DED72
:1019A000192A21EE021A30EE010A8DED120A9DED80
:1019B000020A20EE030A1E9890ED032A20EE020A86
:1019C0009DED0B1A9DED1B4A21EE041A30EE410AE3
:1019D0009DED011A21EE031A21EE021A30EE010AE2
:1019E0009DED0A1A9DED1A2A21EE021A30EE410AE7
:1019F0008DED110A9DED140A20EE000A9DED131ADB
:101A000021EE011A30EE010A9DED121A21EE011AA3
:101A100030EE010A9DED111A21EE011A30EE010A95
:101A200009F05EF88DED150A9DED151A9DED140A6D
:101A300020EE010A8DED140A9DED151A9DED130A95
:101A400020EE010A8DED130A9DED151A9DED120A87
:101A500020EE010A8DED120A9DED151A9DED110A79
:101A600020EE010A8DED110A40F27400C2F200006E
:101A700090ED000A9DED141A20EE011A9DED100A5A
:101A800030EE410A8DED100A90ED000A9DED131A1B
:101A900020EE011A9DED0F0A30EE410A8DED0F0A7E
:101AA00090ED000A9DED121A20EE011A9DED0E0A2E
:101AB00030EE410A8DED0E0A90ED000A9DED111AEF
:101AC00020EE011A9DED0D0A30EE410A8DED0D0A52
:101AD000FFE79DED101A1E9890ED000A90ED042A84
:101AE00021EE021A30EE010A80ED000A9DED0F1A78
:101AF0001E9890ED010A90ED042A21EE021A30EEB4
:101B0000010A80ED010A9DED0E1A1E9890ED020A61
:101B100090ED042A21EE021A30EE010A80ED020A4D
:101B20009DED0D1A1E9890ED030A90ED042A21EE0A
:101B3000021A30EE010A80ED030A1E9890ED000AA9
:101B400090ED013A90ED022A90ED031A20EE000A82
:101B500023EE033A30EE030A22EE022A30EE020AA6
:101B600021EE011A30EE010A08F0BAFF8DED150AD8
:101B70009DED151A1E9890ED000A20EE010A80EDE9
:101B8000000A9DED151A1E9890ED010A20EE010A3B
:101B900080ED010A9DED151A1E9890ED020A20EEC7
:101BA000010A80ED020A9DED151A1E9890ED030AB8
:101BB00020EE010A80ED030A00208DF87F00FFE788
:101BC0009DF97F0020B080BD84B08DED030ACDED7E
:101BD000020A9DED030A9DED021AB1EE411AB4EE20
:101BE000410AF1EE10FA07DAFFE79DED020AB1EEC5
:101BF000400A8DED010A18E09DED030A9DED021AE1
:101C0000B4EE410AF1EE10FA05DDFFE79DED020AA0
:101C10008DED000A04E09DED030A8DED000AFFE75B
:101C20009DED000A8DED010AFFE79DED010A04B06C
:101C30007047000080B541F6B460C2F20000006851
:101C400008210EF085FD80BD80B582B040F20862AB
:101C5000C2F20002002001901221132300F02CFA9E
:101C6000019802B080BD000080B5022001214FF034
:101C7000FF320EF0BFFD80BD81B000909FED010AE4
:101C800001B070470000C84380B541F6B460C2F2AD
:101C90000000006810210EF05BFD80BD80B540F2B1
:101CA0000860C2F20000C21D01200221062300F0DC
:101CB00003FA002080BD000080B5042001214FF010
:101CC000FF320EF097FD80BD80B58AB00890079175
:101CD000089820B9FFE7FE208DF82700B4E00798A8
:101CE00020B9FFE7FE208DF82700ADE041F2491052
:101CF000C2F200000078C00720B1FFE7FD208DF898
:101D00002700A1E00EF004FE41F6B461C2F200012A
:101D1000086020B9FFE7FE208DF8270094E00798BF
:101D20000899C862002006907E21B622049200F035
:101D300059FA049A0120142100F054FA1E2005904B
:101D400001F0C2FA0599069800F0F2F906990846E2
:101D500000F0EEF91E2804D0FFE7FC208DF82700E4
:101D600072E00120002100F0E3F90F2804D0FFE722
:101D7000FC208DF8270067E00320019001F014F8A3
:101D80000420029001F010F842F25D02C0F6000259
:101D9000002003900121009101F034FA019841F6EE
:101DA0003541C0F6000101F07DF8029841F6894105
:101DB000C0F6000101F076F803984021AA2200F055
:101DC00011FA009A0398412100F00CFA039853216C
:101DD000082200F007FA029A0398582100F002FA4C
:101DE000029A03987D2100F0FDF9322001F06CFA8F
:101DF000009A0F21104600F0F5F90098019A102181
:101E000000F0F0F90098039A162100F0EBF9009A1F
:101E10001821104600F0E6F900981521802200F004
:101E2000E1F90A2001F050FA0099019841F24912B3
:101E3000C2F20002117000F0E3FF029800F0E0FF30
:101E400003988DF82700FFE79DF927000AB080BDB1
:101E500084B00290029820B9FFE7FE208DF80F00B1
:101E60006AE040F20861C2F20001B1F80100ADF889
:101E70000600B1F80300ADF80400B1F80500ADF8B4
:101E80000200BDF9060000EE100AB8EEC00A029882
:101E900080ED040ABDF9040000EE100AB8EEC00A95
:101EA000029880ED050ABDF9020000EE100AB8EEB6
:101EB000C00A029880ED060A029890ED040A9FED90
:101EC000201A80EE010A80ED040A029890ED050ABE
:101ED00080EE010A80ED050A029890ED060A80EE78
:101EE000010A80ED060A487C897CC00040EA511056
:101EF000ADF80000BDF90000B0F5806F07DBFFE72B
:101F0000BDF80000A0F50060ADF80000FFE7BDF9E6
:101F1000000000EE100AB8EEC00AB4EE001A20EE7F
:101F2000010AB3EE071A30EE010A029880ED0A0AA0
:101F300000208DF80F00FFE79DF90F0004B07047F7
:101F400000A0AA4584B00290029820B9FFE7FE20C5
:101F50008DF80F007AE040F20860C2F20000B0F89D
:101F60000710ADF80610B0F80910ADF80410B0F87D
:101F70000B00ADF80200BDF9060000EE100AB8EE45
:101F8000C00A029880ED070ABDF9040000EE100AAD
:101F9000B8EEC00A029880ED080ABDF9020000EE12
:101FA000100AB8EEC00A029880ED090A029890ED76
:101FB000070A9FED281A80EE010A80ED070A0298B1
:101FC00090ED080A80EE010A80ED080A029890ED73
:101FD000090A80EE010A80ED090A029890ED070ACD
:101FE0009FED1D1A20EE010A80ED070A029890ED80
:101FF000080A20EE010A80ED080A029890ED090A0D
:1020000020EE010A80ED090A0298C16A91ED001ADA
:1020100090ED070A30EE410A80ED070A0298C16A86
:1020200091ED011A90ED080A30EE410A80ED080AA0
:102030000298C16A91ED021A90ED090A30EE410A48
:1020400080ED090AFE208DF80F00FFE79DF90F00D3
:1020500004B070476F12034235FA8E3C80B5012000
:1020600000F0FAFE68B9FFE70121084600F062FFC0
:1020700041F6B460C2F20000006802210EF068FB75
:10208000FFE7022000F0E8FE68B9FFE70220012127
:1020900000F050FF41F6B460C2F200000068042175
:1020A0000EF056FBFFE780BD80B5182001214FF0F0
:1020B000FF320EF09FFB80BD80B586B08DF8170013
:1020C0008DF8161004928DF80F30049808B9FFE7C8
:1020D0002BE09DF817000146029120B1FFE702981E
:1020E000012805D009E00120002100F023FF04E0D1
:1020F0000220002100F01EFFFFE79DF8160040F0CF
:10210000800040F21B61C2F20001087001220092BF
:1021100000230193184601F097F8009B0198049959
:102120009DF80F2001F02EF8FFE706B080BD0000FB
:1021300080B586B08DF816008DF81510012001F0DD
:10214000C3F89DF816000146049120B1FFE70498FA
:10215000012805D009E00120002100F0EBFE04E099
:102160000220002100F0E6FEFFE79DF8150040F098
:10217000800040F21B61C2F200010191087001224F
:1021800000230293184601F05FF80199029B022296
:10219000184600F0F7FF9DF816000146039120B1A4
:1021A000FFE7039801280CD017E00121084600F052
:1021B000C1FE40F21B60C2F2000040788DF81700AB
:1021C0000BE00220012100F0B5FE40F21B60C2F2DC
:1021D000000000788DF81700FFE79DF8170006B0A3
:1021E00080BD000080B584B08DF80F008DF80E1012
:1021F0008DF80D209DF80E0000F07F0040F21B616D
:10220000C2F2000108709DF80D004870012001F035
:102210005BF89DF80F000146029120B1FFE702989C
:10222000012805D009E00120002100F083FE04E030
:102230000220002100F07EFEFFE740F21B61C2F2A7
:10224000000102220023184600F0FEFF9DF80F0057
:102250000146019120B1FFE70198012805D009E06E
:102260000121084600F066FE04E00220012100F092
:1022700061FEFFE704B080BD80B586B08DF8160022
:1022800004918DF80F209DF80F0020B9FFE70A2078
:102290008DF80F00FFE741F2FC60C2F20000006819
:1022A00064210EF031F920B1FFE7FB208DF8170013
:1022B00070E041F2F860C2F2000000680290FFE7AF
:1022C0000298E0B1FFE7029800789DF81610884266
:1022D00011D1FFE702984068049988420BD1FFE7CB
:1022E00041F2FC60C2F2000000680EF0F1F9FF203C
:1022F0008DF817004EE0029800690290E0E7142084
:1023000000F040FE0190019858B9FFE741F2FC60EF
:10231000C2F2000000680EF0DBF9FE208DF8170015
:1023200038E09DF80F001C2100220DF0EBFF019911
:1023300088600198806870B9FFE7019800F02CFD73
:1023400041F2FC60C2F2000000680EF0C1F9FF200B
:102350008DF817001EE09DF816000199087004988A
:10236000019948609DF80F000199087341F2F861E6
:10237000C2F200010868019A10610198086041F2F8
:10238000FC60C2F2000000680EF0A2F900208DF897
:102390001700FFE79DF9170006B080BD82B00190DD
:1023A0008DF80310019802B07047000084B08DF8DA
:1023B0000B00019141F2F860C2F200000068009049
:1023C000FFE70098A8B1FFE7009800789DF80B1090
:1023D00088420AD1FFE7009840680199884204D1F9
:1023E000FFE700988068039006E00098006900907D
:1023F000E7E700200390FFE7039804B07047000070
:1024000082B000900098C068022809D1FFE70098C8
:1024100081680220042908BF03208DF8070008E026
:10242000009880680438B0FA80F040098DF8070001
:10243000FFE79DF8070002B07047000083B08DF8F9
:1024400007009DF80700022803DBFFE70020029049
:1024500018E09DF807000146009120B1FFE70098C1
:10246000012806D00BE040F66440C2F20000029062
:1024700008E040F68C40C2F20000029002E000202A
:102480000290FFE7029803B07047000080B586B065
:102490008DF8160004910392029341F24810C2F2A3
:1024A00000000078C00720B9FFE7FD208DF8170075
:1024B00037E0039820B9FFE7FE208DF8170030E0E1
:1024C00041F2FC60C2F20000006864210EF01CF8CA
:1024D00020B1FFE7FB208DF8170022E09DF81600E1
:1024E0000499FFF763FF019041F2FC60C2F2000023
:1024F00000680EF0EDF8019820B9FFE7FC208DF898
:1025000017000EE001980399029B00220DF09AFE3D
:1025100000900098002818BF4FF0FF308DF817008A
:10252000FFE79DF9170006B080BD000080B596B0AA
:1025300041F24810C2F200000078C00720B1FFE766
:10254000FD208DF85700A7E040F2B440C2F2000031
:102550006821FDF7DAFF00201490FFE714980128A6
:1025600009DCFFE79DF8500000F01CFBFFE7149822
:1025700001301490F2E741F20811C2F2000142F278
:102580009D30C0F60000086000200EF00DF80146F6
:1025900041F2FC60C2F200000160006820B9FFE770
:1025A000FF208DF8570077E041F24811C2F2000198
:1025B00007910120089008700AA803902821FDF7D0
:1025C000A4FF0399089A002009900F900A900B909D
:1025D000109011920C900D9012920E220292139272
:1025E0000E9040F66440C2F20000019003F0DEF964
:1025F000019804F0D9F8099842F2AD72C0F60002D1
:10260000062100F06FF8099942F62D32C0F600025B
:102610000592084600F066F8059A0899099800F0B6
:1026200061F8059A09980221049100F05BF801987D
:10263000032103F0E5F8029A039908980F920E908F
:1026400040F68C40C2F20000069003F0AFF9069805
:1026500004F0AAF8089842F69102C0F60002082198
:1026600000F040F8059A0999089800F03BF8059A9F
:102670000899084600F036F80499059A089800F081
:1026800031F80698112103F0BBF8079A08990998C8
:1026900011708DF85700FFE79DF9570016B080BD07
:1026A00080B584B002908DF8071041F20810C2F294
:1026B0000000006858B1FFE741F20810C2F20000C4
:1026C000026802989DF807109047039006E0029870
:1026D0009DF80710FFF762FE0390FFE7039804B030
:1026E00080BD000082B08DF806008DF805100092C4
:1026F00041F24810C2F200000078C00720B9FFE79D
:10270000FD208DF807002AE0009820B9FFE7FE20A1
:102710008DF8070023E09DF80600022804DBFFE7A0
:10272000FF208DF807001AE09DF805000D2804DB56
:10273000FFE7FF208DF8070011E000989DF80610D4
:1027400040F2B443C2F20003342211FB02319DF87F
:10275000052041F8220000208DF80700FFE79DF9D1
:10276000070002B07047000080B584B08DF80E00FD
:1027700002918DF8072041F24810C2F20000007863
:10278000C00720B9FFE7FD208DF80F0009E09DF894
:102790000E0002999DF80720FFF76EFD8DF80F00DF
:1027A000FFE79DF90F0004B080BD000080B598B030
:1027B00000200E90FFE70E98012867DCFFE79DF8E8
:1027C0003800FFF73BFE0D900D9808B9FFE759E080
:1027D000FFE70D98002103F0E1F9002851D0FFE751
:1027E0000D98002111AA0FAB03F002FA002847D17F
:1027F000FFE7139818B9FFE71198019002E01298CB
:102800000190FFE701980C9011A8FFF7F9FD8DF8F2
:102810002F000C989DF82F10FFF742FF0A909DF8AB
:1028200038000A99FFF7C2FD0990099838B3FFE70D
:102830000020089007900690059004900390029065
:102840009DF82F008DF808000C9803900A980490CA
:1028500015988DF81400149838B9FFE702A80D30C8
:10286000159A0FA9FDF7D2FDFFE704F0B9FE089015
:10287000099802A900231A460DF0C4FDFFE7FFE7FF
:10288000A7E7FFE70E9801300E9094E718B080BDDF
:1028900080B598B000200E90FFE70E98012867DC05
:1028A000FFE79DF83800FFF7C9FD0D900D9808B9B6
:1028B000FFE759E0FFE70D98012103F06FF90028C9
:1028C00051D0FFE70D98012111AA0FAB03F090F949
:1028D000002847D1FFE7139818B9FFE71198019036
:1028E00002E012980190FFE701980C9011A8FFF701
:1028F00087FD8DF82F000C989DF82F10FFF7D0FE64
:102900000A909DF838000A99FFF750FD0990099840
:1029100038B3FFE7002008900790069005900490D8
:10292000039002909DF82F008DF808000C980390FA
:102930000A98049015988DF81400149838B9FFE798
:1029400002A80D30159A0FA9FDF760FDFFE704F00E
:1029500047FE0890099802A900231A460DF052FD7F
:10296000FFE7FFE7A7E7FFE70E9801300E9094E737
:1029700018B080BD80B592B0844614988DF846C0DA
:102980008DF8451010920F938DF83B0041F24810DE
:10299000C2F200000078C00720B9FFE7FD208DF8E3
:1029A00047009EE09DF84600022804DBFFE7FF2079
:1029B0008DF8470095E00F9870B9FFE79DF8450046
:1029C000022809D0FFE79DF84500032804D0FFE75F
:1029D000FE208DF8470084E09DF83B00092804DBC9
:1029E000FFE7FF208DF847007BE09DF84600FFF7EA
:1029F00025FD0D900D9820B9FFE7FE208DF84700CA
:102A00006FE0002001900C900B900A9009900890C4
:102A10000790069005909DF8450001460291032815
:102A20001FD80299DFE801F002080F1610980590F0
:102A300000200790089018E0109806900420079056
:102A40000020089011E010980590002007900220C7
:102A500008900AE010980690042007900220089041
:102A600003E0FF208DF847003BE09DF83B00099014
:102A700000208DF828000F9868B1FFE79DF83B0013
:102A8000012808DBFFE705A818300F999DF83B20C7
:102A9000FDF7BCFCFFE70D9803F0B4F990B1FFE738
:102AA0000D9805A901F1180204AB02F0D3FE8DF8D0
:102AB0000F009DF80F0020B9FFE700208DF84700B8
:102AC0000FE0FFE79DF8460005A900F00FF920B1DF
:102AD000FFE700208DF8470003E0FF208DF8470056
:102AE000FFE79DF9470012B080BD000080B584B0BB
:102AF0008DF80E000291029820B9FFE7FE208DF8B4
:102B00000F000EE09DF80E0002990A684B1D09792E
:102B1000EC46CCF800100021FFF72CFF8DF80F00D9
:102B2000FFE79DF90F0004B080BD000080B58CB0B8
:102B300000200B90FFE70B98012831DCFFE70B9892
:102B40008DF82B009DF82B00FFF778FC0990099871
:102B500008B9FFE720E0FFE79DF82B0000F044F8FC
:102B6000C8B9FFE7099803F04DF908B9FFE712E08B
:102B70009DF82B0001A900F063F808B9FFE70AE00F
:102B8000099801A901F118026B4602F063FE08B131
:102B9000FFE700E0E0E7FFE70B9801300B90CAE7A2
:102BA0000CB080BD81B08DF803009DF803000228B1
:102BB00001DBFFE715E09DF8030000EBC01041F6D4
:102BC000BC61C2F2000101EBC0020020C2F80004A7
:102BD0009DF8032002EBC21201EBC201C1F804040C
:102BE000FFE701B07047000081B08DF802009DF84A
:102BF0000200022804DBFFE701208DF803001AE041
:102C00009DF8020000EBC01041F6BC61C2F2000169
:102C100001EBC000D0F800049DF8022002EBC212C4
:102C200001EBC201D1F80414401AB0FA80F0400957
:102C30008DF80300FFE79DF8030001B07047000026
:102C4000B0B584B08DF80E0002919DF80E000128F9
:102C500003DCFFE7029820B9FFE700208DF80F00A2
:102C600040E09DF80E0000EBC01141F6BC60C2F2DE
:102C7000000000EBC10001900198D0F80004019918
:102C8000D1F80414884204D1FFE700208DF80F002A
:102C900028E0029900910198D0F8043400EB431227
:102CA0005B01C0585368D2F808C0D2F80CE0146930
:102CB00055694D610C61C1F80CE0C1F808C04B606A
:102CC00008609069D269CA6188610198D0F80404EB
:102CD000013000F01F000199C1F8040401208DF8B3
:102CE0000F00FFE79DF80F0004B0B0BDF0B585B050
:102CF0008DF8120003919DF81200012803DCFFE714
:102D0000039820B9FFE700208DF8130040E09DF8FC
:102D1000120000EBC01141F6BC60C2F2000000EBF3
:102D2000C10002900298D0F80004013000F01F00AA
:102D3000019001980299D1F80414884204D1FFE768
:102D400000208DF8130023E0029ED6F8000406EB65
:102D500040114701039A0092D2F810E054691568B7
:102D600050689368D2F80CC0F5514C61C1F810E07E
:102D7000C1F80CC08B6048609069D269CA618861F3
:102D800001980299C1F8000401208DF81300FFE7B3
:102D90009DF8130005B0F0BD80B582B00190019898
:102DA0000FF0BAF802B080BD80B582B08DF8060091
:102DB0009DF8060001460091052815D80099DFE826
:102DC00001F0031313070B0F062004F08DFE0FE034
:102DD0000A2004F089FE0BE0172004F085FE07E0CE
:102DE000092004F081FE03E0FF208DF8070003E0D6
:102DF00000208DF80700FFE79DF9070002B080BDB5
:102E000080B582B08DF806009DF80600014600915D
:102E1000052815D80099DFE801F0031313070B0FFD
:102E2000062004F06BFE0FE00A2004F067FE0BE0C2
:102E3000172004F063FE07E0092004F05FFE03E0C2
:102E4000FF208DF8070003E000208DF80700FFE762
:102E50009DF9070002B080BD80B582B08DF80600F4
:102E60009DF80600072804DBFFE700208DF8070027
:102E700013E09DF8062045F6C871C0F6010101EB8C
:102E8000C200406831F8321004F07AFB0138B0FA21
:102E900080F040098DF80700FFE79DF8070002B0B9
:102EA00080BD000083B08DF80A000191019820B91F
:102EB000FFE7FE208DF80B0038E09DF80A00072898
:102EC00004DBFFE7FF208DF80B002FE09DF80A10D0
:102ED00045F6C870C0F6010030F83100ADF80200C8
:102EE00000208DF80100FFE79DF801000F2819DC94
:102EF000FFE7BDF802009DF80110C840C00750B1BF
:102F0000FFE701989DF8012040F21C51C2F2000138
:102F100041F8220006E0FFE79DF8010001308DF83E
:102F20000100E1E700208DF80B00FFE79DF90B00A1
:102F300003B0704780B582B08DF806008DF805109B
:102F40009DF80600072804DBFFE7FF208DF8070047
:102F500014E09DF8062045F6C871C0F6010101EBAA
:102F6000C200406831F832109DF8052002F00102DD
:102F700004F01EFB00208DF80700FFE79DF9070015
:102F800002B080BD80B582B0019001980EF022FDA4
:102F900002B080BD86B08DF816008DED040A9DF854
:102FA0001600052804DBFFE7FF208DF817008CE0F2
:102FB0009DED040AB7EE001AB4EE410AF1EE10FAE4
:102FC00004DDFFE74FF07E500490FFE79DED040A1B
:102FD000B5EE400AF1EE10FA03DAFFE700200490A4
:102FE000FFE79DF8161046F20000C0F6010050F809
:102FF00031100968C96A03919DED040A03990131F2
:1030000001EE101AB8EE411A20EE010ABCEEC00A19
:103010008DED020A9DF8161000EBC100808860B9A2
:10302000FFE702989DF8162046F20001C0F6010164
:1030300051F832100968486343E09DF8161046F2D3
:103040000000C0F6010000EBC100808804280DD10B
:10305000FFE702989DF8162046F20001C0F6010134
:1030600051F8321009688863019028E09DF8161025
:1030700046F20000C0F6010000EBC100808808287D
:103080000DD1FFE702989DF8162046F20001C0F628
:10309000010151F832100968C86300900CE00298F1
:1030A0009DF8162046F20001C0F6010151F83210D9
:1030B000096808640090FFE700980190FFE7019815
:1030C000FFE700208DF81700FFE79DF9170006B015
:1030D0007047000080B582B08DF806009DF80600AC
:1030E000052804DBFFE7FF208DF8070010E09DF8BE
:1030F000062046F20000C0F6010000EBC20150F8C5
:103100003200898806F018FF00208DF80700FFE7DD
:103110009DF9070002B080BD80B582B08DF8060031
:103120009DF80600052804DBFFE7FF208DF8070067
:1031300010E09DF8062046F20000C0F6010000EB0A
:10314000C20150F83200898806F0DCFF00208DF8BB
:103150000700FFE79DF9070002B080BD82B08DF83F
:1031600003009DF8030030B9FFE740F64870C2F253
:103170000000019002E000200190FFE7019802B0FA
:103180007047000080B584B08DF80E000291ADF854
:1031900006208DF805309DF80E00012804DBFFE7BE
:1031A000FF208DF80F0029E09DF80E00FFF7D6FFF5
:1031B0000090009820B9FFE7FF208DF80F001DE078
:1031C0009DF80500C00760B1FFE700980299BDF8BF
:1031D000062005F087FC002818BF01208DF80F009D
:1031E0000CE000980299BDF80620142305F052FB6C
:1031F000002818BF01208DF80F00FFE79DF90F0090
:1032000004B080BD82B08DF806008DF805100092E4
:10321000009820B9FFE7FE208DF8070010E0009825
:103220009DF8062040F26451C2F2000101EB421108
:103230009DF8052041F8220000208DF80700FFE7E7
:103240009DF9070002B0704780B584B08DF80E007C
:103250000291ADF806208DF805309DF80E0001288A
:1032600004DBFFE7FF208DF80F0029E09DF80E003A
:10327000FFF774FF0090009820B9FFE7FF208DF85A
:103280000F001DE09DF80500C00760B1FFE7009842
:103290000299BDF8062006F073F9002818BF012036
:1032A0008DF80F000CE000980299BDF80620142359
:1032B00005F038FD002818BF01208DF80F00FFE74A
:1032C0009DF90F0004B080BD80B586B004900CF06D
:1032D00003FF01464FF47A70B0FBF1F003900498BD
:1032E0000399B0FBF1F002900CF0B8FE0146481CC7
:1032F000019198B1FFE70198022820D3FFE70198D8
:1033000002280FD0FFE701980338022806D3FFE711
:1033100001986FF00041884215D1FFE7FF208DF83A
:10332000170014E0029818B1FFE70298009002E03D
:1033300001200090FFE700980CF04AFE03E004989B
:1033400003F0D0FEFFE700208DF81700FFE79DF99E
:10335000170006B080BD000080B58AB00CF0BCFE3E
:10336000079010F0D3FB079A4FF47A710191B1FBEB
:10337000F2F1484306904EF21800CEF2000002909F
:103380000068059010F0C2FB019A01460298079B65
:10339000B2FBF3F25143049100680390069804993C
:1033A000884215D1FFE704984FF47A72504305998B
:1033B00051434EF21402CEF2000212680132B1FB08
:1033C000F2F1401A00F57A7000210991089014E09A
:1033D00004984FF47A725043039951434EF2140209
:1033E000CEF2000212680132B1FBF2F1401A00F590
:1033F0007A70002109910890FFE7089809990AB0AE
:1034000080BD000083B08DF807009DF807000146DD
:10341000009120B1FFE70098012806D00BE041F2AF
:103420007800C2F20000029008E041F2C000C2F24F
:103430000000029002E000200290FFE7029803B033
:103440007047000080B582B0019001980068006864
:10345000C00600282AD5FFE7FFE70020009001986A
:10346000006800680090019800684068009000982B
:10347000FFE701980CF03EF900EBC00140F28850E4
:10348000C2F2000000EB8100006A70B1FFE7019812
:103490000CF030F900EBC00140F28850C2F200009D
:1034A00000EB8100006A8047FFE7FFE702B080BDC4
:1034B00082B08DF806008DF805100092009820B9B2
:1034C000FFE7FE208DF8070020E09DF806000128A8
:1034D00005DCFFE79DF80500092804DBFFE7FF2076
:1034E0008DF8070012E000989DF8061001EBC1026C
:1034F00040F28851C2F2000101EB82019DF80520E3
:1035000041F8220000208DF80700FFE79DF9070031
:1035100002B07047FFE7FEE780B540F66440C2F2B4
:10352000000002F0A7FC80BD80B540F66440C2F206
:10353000000002F09FFC80BD80B540F66440C2F2FE
:10354000000002F097FC80BD80B540F68C40C2F2CE
:10355000000002F08FFC80BD80B540F68C40C2F2C6
:10356000000002F087FC80BD80B540F68C40C2F2BE
:10357000000002F07FFC80BD82B00090009820B96E
:10358000FFE703208DF807001DE00098006846F271
:103590000041C4F20001884204D1FFE700208DF809
:1035A000070010E00098006846F60001C4F2000130
:1035B000884204D1FFE701208DF8070003E00320D3
:1035C0008DF80700FFE79DF8070002B07047000084
:1035D00082B001908DF80310019800699DF80310E6
:1035E00000EB4100407A02B07047000082B00190C9
:1035F0008DF80310019800699DF8031000EB41005D
:10360000007A02B07047000080B588B006908DF84F
:10361000171006989DF81710FFF7E8FF8DF81600B1
:1036200006989DF81710FFF7D3FF8DF815009DF849
:10363000160010280FD1FFE70698006A807900F085
:1036400001008DF814000698406A807900F00100AE
:103650008DF8130029E09DF8160011280FD1FFE71F
:103660000698006AC07900F001008DF814000698F1
:10367000406AC07900F001008DF8130014E006984C
:10368000006A9DF816100844007A00F001008DF8D9
:1036900014000698406A9DF816100844007A00F05D
:1036A00001008DF81300FFE7FFE79DF815000146C4
:1036B000039140B1FFE70398012815D0FFE7039875
:1036C000022824D02AE09DF814100020C907029097
:1036D00021B9FFE79DF813000290FFE7029800F080
:1036E00001008DF81F001DE09DF814100020C9078F
:1036F000019031B1FFE79DF8130080F001000190C7
:10370000FFE7019800F001008DF81F000AE09DF826
:10371000140000F001008DF81F0003E000208DF878
:103720001F00FFE79DF81F0008B080BD82B0019028
:103730008DF8031000208DF80200019890F82C00FD
:10374000012807D1FFE79DF8020040F001008DF845
:103750000200FFE7019890F84000012807D1FFE739
:103760009DF8020040F002008DF80200FFE701988A
:1037700090F85000012807D1FFE79DF8020040F0C3
:1037800004008DF80200FFE79DF803109DF8020089
:103790000840401AB0FA80F0400902B070470000BB
:1037A00080B586B08DED050ACDED040A03909DED40
:1037B000030AB8EE400A9FED151A20EE010A11F037
:1037C00005FB9FED131A20EE010AB0EEC00A9DED35
:1037D000051A30EE010A8DED020A9DED020A9DEDFB
:1037E000041AB4EE410AF1EE10FA05DDFFE79DED93
:1037F000040A8DED010A04E09DED020A8DED010A37
:10380000FFE79DED010A06B080BD00BF6F12833A4D
:10381000CDCC4C3E80B592B010900F910E92109886
:1038200018B1FFE70F9820B9FFE7FE208DF8470099
:103830009FE10E98109A059211685268401A4FF055
:1038400000010691914112F0C6FA059902460698C8
:1038500000EE102A9FEDC91A80EE010A81ED020ADE
:103860000E99109A5060116030B9FFE71098806887
:103870000CF0F0F960B914E01098806812F080FA4A
:1038800041EC100B51EC100B0CF0BCF948B1FFE708
:10389000109890ED020AB5EE400AF1EE10FA07DC3E
:1038A000FFE7109941F26F20C3F683208860FFE79D
:1038B000109890ED020A9FEDB21AB4EE410AF1EEB3
:1038C00010FA07DAFFE7109941F26F20C3F60320E0
:1038D0008860FFE7109890ED020A9FEDAA1AB4EEF7
:1038E000410AF1EE10FA07DDFFE710994CF6CD40E2
:1038F000C3F64C508860FFE710980F9909780E9A2C
:1039000000F0A2FA1098007C01460491012804D02E
:10391000FFE70498052806D00EE010990020886182
:103920001099486142E00F984068109948610F98DB
:1039300080681099886139E0109890ED0C1A90ED2C
:10394000B70A30EE410A8DED0D0A9DED0D0A11F01A
:1039500095F98DED0C0A9DED0D0A11F037FA8DEDFC
:103960000B0A9DED0C0A0F9890ED011A90ED022ABA
:1039700020EE010A9DED0B1A21EE021A30EE410AEB
:10398000109880ED050A9DED0B0A0F9890ED011A35
:1039900090ED022A20EE010A9DED0C1A21EE021A8A
:1039A00030EE010A109880ED060AFFE71098007CBF
:1039B0000146039106284BD80399DFE801F004047F
:1039C0000D1E3304080010990020C86140E00F98D4
:1039D000C0681099C8613BE0109901F59C70D1ED69
:1039E000021A91ED0C0AD1EDB70A9FED6A1A08F0A0
:1039F00031FF109880ED070A2AE0109901F59C70BC
:103A0000D1ED021A91ED0C0AD1EDB70A9FED601AC3
:103A100030EE010A9FED5F1A08F01CFF109880ED50
:103A2000070A15E0109890ED0D0A8DED020A0E9828
:103A30009FED550ADFED550AFFF7B2FEB0EE401AD2
:103A40009DED020A20EE010A109880ED070AFFE7BB
:103A5000109B03F1120003F1140103F1380293F9F2
:103A600011309FED4D0A08F045FC00208DF82B0029
:103A7000FFE79DF82B00109991F91110884274DA34
:103A8000FFE710989DF82B1000EB8100806B0990E8
:103A900010999DF82B2001EB421000F5C67001EB48
:103AA000021191EDA80A07F057F88DED080A109859
:103AB000007C0146019170B3FFE7019801380528A9
:103AC00004D3FFE70198062817D027E010999DF846
:103AD0002B20C2EB021001EB8000483001EB820288
:103AE00092ED0E0ADDED080AD1ED021A9FED291ABA
:103AF00008F0B0FE8DED070A10E010989DF82B102D
:103B000000EB810090ED0E0A9FED241A80EE010A71
:103B10008DED070A02E000200790FFE710989DF85E
:103B20002B1000EB411000F503709DED070A07F024
:103B300013F810989DF82B1000EB810080EDA30A7C
:103B400010999DF82B0001EB800000F52370C968E7
:103B5000D1ED1F0AB1EE600A00F0DEFAFFE79DF832
:103B60002B0001308DF82B0083E700208DF84700F3
:103B7000FFE79DF9470012B080BD00BF00007A4406
:103B80006F12033ACDCC4C3D9A99193FCDCC4C3FA6
:103B9000AB611C3F000000000000FA4300C0DA45A2
:103BA00080B58AB0089007918DED060A089820B973
:103BB000FFE7FE208DF82700F0E0FEF7B7FC07983E
:103BC0000899C860089900200874079890F8600068
:103BD0000146039106282ED80399DFE801F0040B73
:103BE00012181F2C250008990420487400208DF815
:103BF000170024E008990420487401208DF817006C
:103C00001DE00899022048748DF8170017E0089904
:103C10000420487403208DF8170010E00899042050
:103C200048748DF817000AE00899012048740520AF
:103C30008DF8170003E0FC208DF82700AEE008990E
:103C4000002048600860089988608DF81600FFE73A
:103C50009DF81600089991F91110884251DAFFE792
:103C600008989DF81610C1EB011100EB8100483057
:103C70009DED060A079901F120020021029108F04A
:103C800061FF08989DF8161000EB411000F5C67012
:103C90009DED060A0799D1ED190A06F0B9FF0898BB
:103CA0009DF8161000EB411000F503709DED060A1B
:103CB0000799D1ED1A0A06F0ABFF029808999DF812
:103CC000162001EB0211C1F8A00208999DF81620F8
:103CD00001EB0211C1F8A40208999DF8162001EB2E
:103CE0000211C1F89C0208999DF8162001EB0211FF
:103CF000C1F8A802FFE79DF8160001308DF8160004
:103D0000A6E7089800F59C709DED060A079901F159
:103D100040020021019108F015FF089812309DF82B
:103D2000171008F039FC01980899C8610899886152
:103D3000089948618DF81500FFE79DF8150008996E
:103D400091F9111088420FDAFFE708989DF81510D5
:103D500000EB81010020C1F88C02FFE79DF81500FF
:103D600001308DF81500E8E700200490FFE7049883
:103D7000089991F9111088420CDAFFE70898C06899
:103D8000049900EBC10007F089FDFFE704980130BA
:103D90000490ECE700208DF82700FFE79DF927004D
:103DA0000AB080BD80B586B00590059808B9FFE7D8
:103DB00048E000208DF81300FFE79DF813000599F7
:103DC00091F9111088421CDAFFE705989DF813104D
:103DD00000EB8100006A0390039808B9FFE70AE04E
:103DE000039805999DF8132001EB820191EDA30A38
:103DF00007F0F0FDFFE79DF8130001308DF8130088
:103E0000DBE700208DF80B00FFE79DF80B0005991C
:103E100091F91110884215DAFFE705989DF80B100B
:103E200000EB8100006A0190019820B1FFE7019842
:103E300007F096FBFFE7FFE79DF80B0001308DF8D8
:103E40000B00E2E706B080BD80B586B004908DF827
:103E50000F100292049820B9FFE7FE208DF817009A
:103E600068E09DF80F000499097C884204D1FFE7BF
:103E700000208DF817005DE09DF80F0004281CD18C
:103E8000FFE70498007C042817D0FFE70298FCF7AE
:103E90009FFAFCF7EBF900EBD07121F00101411A18
:103EA0000120002918BF4FF0FF3000EE100AB8EED5
:103EB000C00A049880ED0D0AFFE700208DF8070086
:103EC000FFE79DF80700049991F91110884229DA5B
:103ED000FFE704989DF80710C1EB011100EB81008A
:103EE000483008F0FBFE04989DF8071000EB4110E5
:103EF00000F5C6709FED110A8DED000A06F026FF51
:103F00009DED000A04989DF8071000EB411000F5A4
:103F1000037006F01BFFFFE79DF8070001308DF8E6
:103F20000700CEE79DF80F000499087400208DF873
:103F30001700FFE79DF9170006B080BD00000000E4
:103F400080B586B0049000208DF80F00FFE79DF843
:103F50000F00049991F91110884245DAFFE704989F
:103F6000C0689DF80F1000EBC10007F0C1FD049878
:103F7000C0689DF80F1000EBC10007F02BFC029009
:103F8000029804999DF80F2001EB820108620498C1
:103F90009DF80F1000EB8100006A01900298C0B1FB
:103FA000FFE704989DF80F1000EB0111DDF808C041
:103FB000DCF80800DCF80C20DCF81030DCF814C069
:103FC000C1F8A8C2C1F8A432C1F8A022C1F89C026D
:103FD00003E0FE208DF817000AE0FFE79DF80F00D0
:103FE00001308DF80F00B2E700208DF81700FFE7D1
:103FF0009DF9170006B080BD84B003908DED020AD4
:10400000CDED010A039890ED000A9DED021A30EE05
:10401000010A8DED000A9DED010AB5EE400AF1EEB0
:1040200010FA26DDFFE79DED000A9DED011AB4EEC2
:10403000410AF1EE10FA09DBFFE79DED011A9DED53
:10404000000A30EE410A8DED000A11E09DED000AF4
:10405000B5EE400AF1EE10FA09DAFFE79DED011A1C
:104060009DED000A30EE010A8DED000AFFE7FFE743
:10407000FFE700980399086004B0704785B08DEDA4
:10408000040ACDED030A8DED021A9DED040A9DEDA3
:10409000031A30EE410A8DED010A9DED020AB5EEDC
:1040A000400AF1EE10FA32DDFFE79DED020AB0EEB4
:1040B000001A80EE010A8DED000A9DED010A9DEDCA
:1040C000001AB4EE410AF1EE10FA09DDFFE79DEDAA
:1040D000021A9DED010A30EE410A8DED010A15E04C
:1040E0009DED010A9DED001AB1EE411AB4EE410AB0
:1040F000F1EE10FA09DAFFE79DED021A9DED010AD3
:1041000030EE010A8DED010AFFE7FFE7FFE79DEDC5
:10411000010A05B07047000083B002908DED010ADE
:10412000CDED000A029890ED000A9DED001AB4EE64
:10413000410AF1EE10FA04DDFFE7009802990860E9
:10414000FFE7029890ED000A9DED011AB4EE410AD6
:10415000F1EE10FA04DAFFE7019802990860FFE730
:1041600003B0704780B584B00290029820B9FFE791
:10417000FF208DF80F0017E0029800F09FF88DF8EF
:1041800007009DF80700029981F82C009DF80700B0
:10419000029981F840009DF80700029981F85000CB
:1041A00000208DF80F00FFE79DF90F0004B080BDDF
:1041B00080B586B00490049820B9FFE7FF208DF801
:1041C000170074E00498FFF7CDFF0498143000F056
:1041D0000DFC04981C3000F039FA0498283000F0E7
:1041E0000DF90498293000F059FCFFF7B5F811F0EB
:1041F000F2FD00EE100A9FED301A8DED021A80EEEE
:10420000010A049880ED000AFFF7A6F8049A0392C9
:104210009368D268C01A914111F0DDFD9DED021A3C
:104220000146039800EE101A80EE010A80ED010AA3
:10423000FFF792F80A460499CA608860049890F8DB
:104240002C0003280CDCFFE7049890F840000328BA
:1042500006DCFFE7049890F85000042807DBFFE72E
:10426000049800F0D3F8FD208DF817001FE00498A3
:1042700090F82C2040F22431C2F20001019101EBB0
:104280000211496888470199049890F8402001EB91
:104290000211896888470199049890F8502001EB31
:1042A0000211C968884700208DF81700FFE79DF9C3
:1042B000170006B080BD00BF0024744980B586B0E9
:1042C000049000200390FFE7039803283FDCFFE7FA
:1042D00004980069039910F811008DF80B009DF8FF
:1042E0000B000146019103282CD80199DFE801F069
:1042F00016200C02049800F0F3FB20B1FFE7032026
:104300008DF8170027E01DE0049800F0CFFB20B1E6
:10431000FFE702208DF817001DE013E0049800F07D
:10432000D7FB20B1FFE700208DF8170013E009E06C
:10433000049800F0C5FB20B1FFE701208DF81700BD
:1043400009E0FFE7FFE7039801300390BCE7052091
:104350008DF81700FFE79DF8170006B080BD00003C
:1043600083B001900091019818B1FFE7009820B93F
:10437000FFE7FF208DF80B0006E000980199086127
:1043800000208DF80B00FFE79DF90B0003B070478C
:1043900082B00090009820B9FFE7FF208DF8070059
:1043A00003E000208DF80700FFE79DF9070002B049
:1043B0007047000082B00090009820B9FFE7FF200E
:1043C0008DF8070003E000208DF80700FFE79DF956
:1043D000070002B07047000082B00090009820B93A
:1043E000FFE7FF208DF8070003E000208DF80700AD
:1043F000FFE79DF9070002B07047000081B0009010
:1044000000990020087001B07047000082B0009051
:10441000009820B9FFE7FF208DF807000AE0009917
:10442000002081F83000009981F84400009981F85B
:104430005200FFE79DF9070002B0704780B584B0D5
:104440000290029820B9FFE7FF208DF80F0035E0B9
:10445000029900208863029948630190FFE7019860
:104460000D2827D8FFE7019946F24810C0F6010051
:10447000405C8DF8030002989DF80310FFF756F991
:1044800098B1FFE702989DF80410FFF7BDF858B106
:10449000FFE7019940F20400C2F2000000EBC10006
:1044A000416802988847FFE7FFE7FFE7019801307E
:1044B0000190D4E700208DF80F00FFE79DF90F0071
:1044C00004B080BD80B584B00290029820B9FFE7A7
:1044D000FF208DF80F005BE00299012081F8440075
:1044E0000298016AB1F9001000EE101AB8EEC00A85
:1044F00090ED011A20EE010A016991ED091A20EEF2
:10450000010A80ED120A0298016AB1F9021000EE68
:10451000101AB8EEC00A90ED011A20EE010A0169E6
:1045200091ED091A20EE010A80ED130A0020019096
:10453000FFE701980D2827D8FFE7019946F24810B8
:10454000C0F60100405C8DF8030002989DF803104E
:10455000FFF7ECF898B1FFE702989DF80410FFF719
:1045600053F858B1FFE7019940F20400C2F200008D
:1045700000EBC100416802988847FFE7FFE7FFE7CB
:10458000019801300190D4E700208DF80F00FFE77B
:104590009DF90F0004B080BD80B584B002900298F0
:1045A00020B9FFE7FF208DF80F004AE002990020B4
:1045B00081F854000190FFE701980D2827D8FFE704
:1045C000019946F24810C0F60100405C8DF80300E6
:1045D00002989DF80310FFF7A9F898B1FFE7029839
:1045E0009DF80410FFF710F858B1FFE7019940F269
:1045F0000400C2F2000000EBC10041680298884745
:10460000FFE7FFE7FFE7019801300190D4E7029848
:10461000016A406A083008311222FBF7F7FE02995E
:10462000086A496A807900F0010088710299086A75
:10463000496AC07900F00100C87100208DF80F00B0
:10464000FFE79DF90F0004B080BD000081B000902D
:10465000009900200870009A41F25811C2F200013E
:104660005160009A41F27211C2F20001916041F270
:104670000071C2F200010978009A01F00101117085
:1046800001B0704781B000900098016991ED0B1A5C
:1046900090ED0D0A20EE010A80ED0D0A00980169E7
:1046A00091ED0B1A90ED0E0A20EE010A80ED0E0A34
:1046B000002001B07047000081B00090002001B0E0
:1046C0007047000081B000900098016991ED0A1ACE
:1046D00090ED0E0A30EE410A80ED0E0A002001B086
:1046E0007047000081B00090002001B070470000CA
:1046F00081B000900098016991ED0C1A90ED0D0ABF
:1047000020EE010A80ED0D0A0098016991ED0C1A66
:1047100090ED0E0A20EE010A80ED0E0A002001B095
:104720007047000081B000900099012081F854008A
:10473000002001B07047000081B00090009991F80E
:104740005200013081F85200009991F8520000F0B7
:10475000030081F85200002001B0704781B0009042
:104760000099032081F83000002001B0704700005C
:1047700081B000900098016991ED0A1A90ED0E0A3F
:1047800030EE010A80ED0E0A002001B070470000F3
:1047900081B000900098016991ED0A1A90ED0D0A20
:1047A00030EE410A80ED0D0A002001B07047000094
:1047B00081B00090002001B07047000081B00090EF
:1047C000002001B07047000081B00090009801699E
:1047D00091ED0A1A90ED0D0A30EE010A80ED0D0AF6
:1047E000002001B07047000081B0009000990420C3
:1047F00081F830000099022081F83100002001B0DA
:104800007047000083B00190019820B9FFE7FF20B6
:104810008DF80B0034E00198806990F8390001466A
:104820000091012812D0FFE70098022804D0FFE78A
:104830000098032805D00EE00199042081F830008B
:104840000EE00199022081F8300009E00199002072
:1048500081F8300004E00199002081F83000FFE782
:1048600001998869806A486301998869406A886308
:1048700001998869C06AC86300208DF80B00FFE7C2
:104880009DF90B0003B0704783B00190019820B9E7
:10489000FFE7FF208DF80B0059E00198806990F840
:1048A00039000146009101282BD0FFE7009802282B
:1048B00004D0FFE7009803280AD03BE001990120CB
:1048C00081F844000199002088640199C8643AE0A5
:1048D0000199012081F844000198816991ED091A3C
:1048E000B1EE410A30EE410A80ED120A0198816969
:1048F00091ED0A0ABFEE081A20EE010A80ED130AB4
:1049000021E00199002081F844000198816991ED2E
:10491000091AB1EE410A30EE410A80ED120A0198FF
:10492000816991ED0A0ABFEE081A20EE010A80EDB6
:10493000130A08E00199002081F844000199886475
:104940000199C864FFE700208DF80B00FFE79DF98F
:104950000B0003B07047000083B00190019820B9AC
:10496000FFE7FF208DF80B003BE00199087D00F088
:10497000010081F851000198806990F838000146E3
:104980000091012819D0FFE70098022804D0FFE722
:104990000098032808D018E00199012081F85300FD
:1049A000019981F8540018E00199012081F8530021
:1049B0000199002081F854000FE00199002081F84E
:1049C0005300019981F8540007E00199002081F813
:1049D0005300019981F85400FFE700208DF80B0087
:1049E000FFE79DF90B0003B07047000080B582B06F
:1049F000019041F20070C2F2000000900BF0FCF94F
:104A000000980199486000F13C0141F25810C2F24F
:104A100000001A22FBF7FAFC01994868007800F0C0
:104A20000100087001990020487002B080BD0000AC
:104A300082B00090009820B9FFE7FF208DF80700B2
:104A400003E000208DF80700FFE79DF9070002B0A2
:104A50007047000082B00090009820B9FFE7FF2067
:104A60008DF8070003E000208DF80700FFE79DF9AF
:104A7000070002B07047000082B00090009820B993
:104A8000FFE7FF208DF8070003E000208DF8070006
:104A9000FFE79DF9070002B07047000081B0009069
:104AA00000990020087001B07047000081B00090AC
:104AB000009890F8280000F0010001B07047000055
:104AC00081B000900098007F00F0010001B07047B5
:104AD00081B000900098007D00F0010001B07047A7
:104AE00081B00090009890F8290000F0010001B01A
:104AF0007047000040F28400C2F2000070470000DE
:104B000080B540F6D450C2F2000002F041F880BDFA
:104B100080B540F6B440C2F2000002F039F880BD22
:104B200080B540F63460C2F2000002F031F880BD7A
:104B300080B540F61450C2F2000002F029F880BDA2
:104B400080B540F67450C2F2000002F021F880BD3A
:104B500080B540F69460C2F2000002F019F880BD02
:104B600082B001900198007810384AF6AB21CAF65D
:104B7000AA21A0FB011000090090009945F6C07021
:104B8000C0F60100405C0199C8650098042807D36D
:104B9000FFE701990868042262F30900886506E0CE
:104BA0000199086840F2FF3290438865FFE7019859
:104BB000806D02B07047000086B0059000208DF82F
:104BC00013000598806A03900598806910BBFFE781
:104BD0000398029003281BD80299DFE801F0020D28
:104BE0000218059890F82F00C00720B1FFE70120B8
:104BF0008DF81300FFE70CE00598C06AB0F1C07FA4
:104C000004D1FFE701208DF81300FFE701E000E089
:104C1000FFE745E005988069B0F5005F25D1FFE723
:104C20000398019003281ED80199DFE801F00206DD
:104C3000021101208DF8130016E0059890F82F005E
:104C4000C00720B1FFE701208DF81300FFE70BE05C
:104C50000598C06AB0F1C07F04D1FFE701208DF84C
:104C60001300FFE700E0FFE719E003980090032836
:104C700004D3FFE70098032804D00EE001208DF84C
:104C800013000BE0059890F82F00C00720B1FFE754
:104C900001208DF81300FFE700E0FFE7FFE7FFE7E3
:104CA0009DF8130006B0704784B003900291019202
:104CB000009303980168086820F480200860009839
:104CC00003990968486003988068402809D1FFE784
:104CD0000198039909688860029803990968C86077
:104CE00008E00298039909688860019803990968A7
:104CF000C860FFE704B0704782B00090009820B908
:104D0000FFE701208DF8070074E00098008A6FF338
:104D1000DF20B0F5B67F09D3FFE70098008A6FF374
:104D2000DF2040F29561884204D3FFE701208DF82F
:104D300007005FE000980069C0F3CA20B0F5B67FB5
:104D400009D3FFE700980069C0F3CA2040F29561DB
:104D5000884204D3FFE701208DF807004AE000985D
:104D6000818A0069800D40EA81206FF3DF20B0F571
:104D7000B67F0DD3FFE70098818A0069800D40EA75
:104D800081206FF3DF2040F29561884204D3FFE772
:104D900001208DF807002DE00098808AC0F34A00BA
:104DA000B0F5B67F09D3FFE70098808AC0F34A00C8
:104DB00040F29561884204D3FFE701208DF8070097
:104DC00018E00098818A0020B0EB913F04D1FFE702
:104DD00001208DF807000DE00098808A000B800705
:104DE00020B9FFE701208DF8070003E000208DF8CF
:104DF0000700FFE79DF8070002B0704780B584B058
:104E00000290029820B9FFE7FE208DF80F002BE0FA
:104E100041F24A10C2F200000078C00720B1FFE75B
:104E2000FD208DF80F001FE00BF072FD41F6B86118
:104E3000C2F20001086020B9FFE7FE208DF80F00E4
:104E400012E045F26102C0F6000200200190032149
:104E5000FEF72EFB019841F24A12C2F20002012134
:104E600011708DF80F00FFE79DF90F0004B080BDB1
:104E700080B584B00290029820B9FFE7FE208DF83B
:104E80000F000CE002990020019008700298243075
:104E90003421FBF73AFB01988DF80F00FFE79DF9ED
:104EA0000F0004B080BD000080B586B00490049867
:104EB00020B9FFE7FE208DF81700C9E00498FFF73E
:104EC0001BFF20B1FFE7FF208DF81700C0E0049919
:104ED00001200870FEF740FA0A460499CA6088600B
:104EE000049824303421FBF710FB0020C4F2A540C5
:104EF00003900498018A6FF3DF2100EE101AB8EED8
:104F0000400A9FED551A30EE410A30EE000A9DED41
:104F1000032A80EE020A80ED0B0A04980169C1F3AE
:104F2000CA2100EE101AB8EE400A30EE410A30EE07
:104F3000000A9DED032A80EE020A80ED0C0A049817
:104F4000828A0169890D41EA82216FF3DF2100EE37
:104F5000101AB8EE400A30EE410A30EE000A9DED1C
:104F6000032A80EE020A80ED090A0498818AC1F3BF
:104F70004A0100EE101AB8EE400A30EE410A30EE57
:104F8000000A9DED031A80EE010A80ED0A0A0499D9
:104F9000888A800B81F839000499888AC0F301302F
:104FA00081F838000499C88A88870499088BC887D3
:104FB0000499488BA1F840000499087F002818BF85
:104FC000012081F842000499487F002818BF012081
:104FD00081F843000498C08BADF80A0000200190CE
:104FE000FFE701980F280FDCFFE7BDF80A00019AE0
:104FF000D04000F001000499114481F84400FFE71B
:10500000019801300190ECE7049991F8420000F01A
:10501000010081F85400049991F8430000F0010068
:1050200081F855000498018C00EE101AB8EE400A81
:105030009FED0A1A30EE010A30EE000A9DED031AC8
:1050400080EE010A80ED0D0A00208DF81700FFE7C1
:105050009DF9170006B080BD00008044000080C4A8
:1050600080B541F6B860C2F20000006801210BF083
:105070006FFB80BD80B582B000900020FEF7C2F9C2
:1050800000991031122205F07FFC20B9FFE70020C3
:105090008DF8070003E0FF208DF80700FFE79DF97A
:1050A000070002B080BD000080B582B00190019A77
:1050B000012108460BF09EFB0138B0FA80F0400950
:1050C00002B080BD7047000080B5012002F060F89A
:1050D00080BD000080B5082002F05AF880BD0000B5
:1050E00080B5102002F054F880BD000080B520206B
:1050F00002F04EF880BD000072B6FFE7FEE7000048
:1051000080B592B010900F91109818B1FFE70F98EA
:1051100020B9FFE7FF208DF84700C0E1FEF71CF93A
:10512000109A049213685268C01A914110F053FE0D
:105130000146049800EE101A9FEDDB1A80EE010A7A
:1051400080ED020AFEF708F90A4610994A600860E5
:1051500010980F99097800F07DFA0F9890ED010AE8
:10516000109890ED021A20EE010AB7EE081A20EE10
:10517000010A8DED0E0A1098C06890ED280AB5EE70
:10518000400AF1EE10FA72DDFFE7109890ED5D1A1B
:1051900090ED600A30EE410A8DED0D0A9DED0D0A8D
:1051A0009FEDC21AB4EE410AF1EE10FA09DDFFE7F5
:1051B0009DED0D0A9FEDBE1A30EE010A8DED0D0A30
:1051C000FFE79DED0D0A9FEDBB1AB4EE410AF1EE2B
:1051D00010FA09DAFFE79DED0D0A9FEDB71A30EEE0
:1051E000010A8DED0D0AFFE7109890ED051A90ED7C
:1051F000440A9DED0D2A31EE021A9DED0E2A71EE44
:10520000020A9FEDAD1A8DED031AFEF737FF9DEDF3
:10521000031A8DED0C0A109890ED052A90ED450AC1
:105220009DED0D3A32EE032A9DED0E3A72EE030A21
:10523000FEF724FF8DED0B0A9DED0E0A9DED0C1A75
:10524000B4EE410AF1EE10FA03DDFFE70C980E9080
:10525000FFE79DED0E0A9DED0B1AB4EE410AF1EE4B
:1052600010FA03DAFFE70B980E90FFE7FFE71098BC
:1052700014309DED0E0ADFED900AFEF7BDFE0F988B
:1052800090ED020A109890ED021A20EE010A8DEDC1
:105290000A0A1098C06890ED290AB5EE400AF1EEAE
:1052A00010FA6BDDFFE7002009909DED090A9FEDE4
:1052B0007F1AB4EE410AF1EE10FA09DDFFE79DED29
:1052C000090A9FED7B1A30EE010A8DED090AFFE70E
:1052D0009DED090A9FED771AB4EE410AF1EE10FA3E
:1052E00009DAFFE79DED090A9FED731A30EE010A16
:1052F0008DED090AFFE7109890ED061A90ED460A29
:105300009DED092A31EE021A9DED0A2A71EE020A7C
:105310009FED691A8DED021AFEF7B0FE9DED021A9F
:105320008DED080A109890ED062A90ED470A9DED44
:10533000093A32EE032A9DED0A3A72EE030AFEF7AD
:105340009DFE8DED070A9DED0A0A9DED081AB4EE4B
:10535000410AF1EE10FA03DDFFE708980A90FFE733
:105360009DED0A0A9DED071AB4EE410AF1EE10FA1E
:1053700003DAFFE707980A90FFE7FFE71098183075
:105380009DED0A0ADFED4C0AFEF736FE0F9890ED10
:10539000020AB0EE081A80EE010A9FED481A30EEBC
:1053A000010A9FED471A30EE010A109880ED060AB7
:1053B0001098007C0146019140B1FFE70198012857
:1053C0000CD0FFE7019802285DD064E0109900201E
:1053D000C1F860011099C1F864015CE0109901F115
:1053E0002000D1ED021A91ED050AD1ED5D0A9FED85
:1053F000351A8DED001A07F02DFA9DED001A8DED8E
:10540000060A109901F1D4009DED060AD1ED021AA9
:10541000D1ED5C0A07F01EFA9DED001A109880EDA0
:10542000580A109901F19800D1ED021A91ED060A7F
:10543000D1ED640A07F00EFA9DED001A8DED050A14
:10544000109901F1D4009DED050AD1ED021AD1EDBC
:105450005A0A07F0FFF9109880ED590A109901F5E2
:10546000907091ED580A05F077FB109880ED580A7E
:10547000109901F5A07091ED590A05F06DFB109897
:1054800080ED590A07E010990020C1F860011099D9
:10549000C1F86401FFE700208DF84700FFE79DF9A0
:1054A000470012B080BD00BF00247449DB0F4940A3
:1054B000DB0FC9C0DB0F49C0DB0FC94052B83E400B
:1054C000ABAAAA3E0000000080B586B0049003910C
:1054D0008DED020A049820B9FFE7FF208DF8170030
:1054E0007BE003980499C86004980021019101743D
:1054F000049A02F120009DED020AD268303207F0D2
:1055000021FB049901F15C009DED020AC96801F1DB
:1055100010020121009107F015FB0199049A02F194
:1055200098009DED020AD268703207F00BFB0099DB
:10553000049A02F1D4009DED020AD268503207F0BD
:1055400001FB049901F590709DED020AC968D1ED47
:10555000240A05F05DFB049901F5A0709DED020A97
:10556000C968D1ED240A05F053FB0498C16891ED98
:10557000260A91ED281A30EE010A80ED440A0499BA
:10558000C868D0F89800C1F814010498C16891ED7A
:10559000270A91ED291A30EE010A80ED460A049996
:1055A000C868D0F89C00C1F81C01FCF7BFFF049844
:1055B000C06805F0CBFD0498C068083005F0C6FD52
:1055C0000498C06805F058FC0498C068083005F0DD
:1055D00053FC01988DF81700FFE79DF9170006B0FE
:1055E00080BD000080B58CB00B90002000900A9028
:1055F00009900890079006900B9890ED590AB1EE2B
:10560000041A20EE010A8DED060A4FF07E500A9032
:105610000B98C06806A905F0C9FC00980590049095
:105620000390029001900B9890ED580AB2EE001A88
:1056300020EE010A8DED010A49F69A10C3F6996031
:1056400005900B98C068083001A905F0AFFC0CB0BC
:1056500080BD000080B584B002908DF807100298DC
:1056600020B9FFE7FF208DF80F0047E09DF8070005
:105670000299097C884204D1FFE700208DF80F00D1
:105680003CE00298203007F029FB02985C3007F0DC
:1056900025FB0298983007F021FB0298D43007F0E0
:1056A0001DFB029800F590709FED160A8DED000A23
:1056B00005F04CFB9DED000A029800F5A07005F086
:1056C00045FB0298C068083005F0D6FB0298C06818
:1056D00005F0D2FB02981430FBF77AF90299D1F861
:1056E000900188610299D1F8740148619DF8070022
:1056F0000299087400208DF80F00FFE79DF90F0054
:1057000004B080BD0000000080B584B00290029813
:1057100020B9FFE7FF208DF80F0045E00298C06830
:1057200005F04CFE0298C06805F0FCFB0190019862
:10573000A0B1FFE70299DDF804C0DCF81C00DCF83A
:105740002020DCF82430DCF828C0C1F89CC1C1F866
:105750009831C1F89421C1F89001FFE70298C06820
:10576000083005F02BFE0298C068083005F0DAFB1F
:1057700000900098A0B1FFE70299DDF800C0DCF8C6
:105780001C00DCF82020DCF82430DCF828C0C1F84C
:105790008CC1C1F88831C1F88421C1F88001FFE7CC
:1057A00000208DF80F00FFE79DF90F0004B080BDC9
:1057B00083B001900091019820B9FFE7FF208DF898
:1057C0000B0019E00199009B18685A689B68C1F8A2
:1057D0007031C1F86C21C1F868010199009BD8684B
:1057E0001A695B69C1F87C31C1F87821C1F874018C
:1057F00000208DF80B00FFE79DF90B0003B0704708
:1058000084B002900191029890F820008DF8030076
:105810009DF80300012805D0FFE79DF8030002284A
:105820000AD1FFE7019A029801684869104348616C
:1058300000208DF80F0008E00299486A40F48020AB
:10584000486201208DF80F00FFE79DF80F0004B0BB
:105850007047000088B00690059104920393069863
:1058600090F820008DF80700069800688068009086
:105870000598806808B9FFE700E0FFE79DF807009A
:10588000012806D0FFE79DF80700022840F080803D
:10589000FFE79DF80300400700280CD4FFE79DF8C0
:1058A00003000007002806D4FFE79DF80300C006A8
:1058B000002864D5FFE70098C0F3016002900299C8
:1058C00001208840039908600598806868B9FFE75F
:1058D00005980168C06840EA415006990968029A33
:1058E00001EB0211C1F880010EE005994A68886851
:1058F000C96840EAC200084306990968029A01EBA8
:105900000211C1F88001FFE705980069069909684E
:10591000029A01EB0211C1F884010598007D01286B
:105920000CD1FFE706980068029900EB0111D1F84D
:10593000840140F48070C1F88401FFE70498406856
:1059400006990968029A01EB0211C1F88C010498CA
:10595000006806990968029A01EB0211C1F88801F2
:1059600006980068029900EB0111D1F8800140F01F
:105970000100C1F8800100208DF81F0011E0069998
:10598000486A40F40010486201208DF81F0008E0CA
:105990000699486A40F48020486201208DF81F0073
:1059A000FFE79DF81F0008B07047000086B0049024
:1059B0000391049890F820008DF803009DF80300EF
:1059C000012806D0FFE79DF80300022840F0B080D0
:1059D000FFE746F20040C4F2000001900199D1F8BF
:1059E000000240F00100C1F800020199D1F8000264
:1059F00020F47C50C1F800020398426A0199D1F862
:105A0000000240EA0220C1F800020398406900F059
:105A10001F01012088400290029A0199D1F81C02CE
:105A20009043C1F81C020398C069F0B9FFE7029ADD
:105A30000199D1F80C029043C1F80C02039A9088A6
:105A4000D168526940EA0140019901EBC201C1F8F5
:105A50004002039A10889168526940EA0140019916
:105A600001EBC201C1F84402FFE70398C0690128B5
:105A70001ED1FFE7029A0199D1F80C021043C1F838
:105A80000C02039A90881168526940EA014001991A
:105A900001EBC201C1F84002039A908991685269F2
:105AA00040EA0140019901EBC201C1F84402FFE75D
:105AB0000398806940B9FFE7029A0199D1F804027E
:105AC0009043C1F8040207E0029A0199D1F8040258
:105AD0001043C1F80402FFE70398006940B9FFE7EB
:105AE000029A0199D1F814029043C1F8140207E018
:105AF000029A0199D1F814021043C1F81402FFE789
:105B00000398006A012808D1FFE7029A0199D1F8A9
:105B10001C021043C1F81C02FFE70199D1F80002F2
:105B200020F00100C1F8000200208DF8170008E005
:105B30000499486A40F48020486201208DF81700DB
:105B4000FFE79DF8170006B07047000080B582B0EF
:105B500001900198FDF710FD8DF803009DF80300FA
:105B6000032819D0FFE79DF8030040F2B442C2F2C7
:105B70000002342110FB0120006B60B1FFE79DF8AB
:105B8000030040F2B442C2F20002342110FB0120B3
:105B9000006B8047FFE7FFE702B080BD84B0039051
:105BA000029100200190039890F820008DF80300E6
:105BB0009DF80300012805D0FFE79DF803000228A7
:105BC00012D1FFE7029838B9FFE703980068C06870
:105BD00000F00300019006E003980068006900F0FF
:105BE00003000190FFE7FFE7019804B07047000051
:105BF00086B00490039102920193049890F82000DB
:105C00008DF803009DF80300012806D0FFE79DF8FA
:105C10000300022840F0E880FFE7039880B9FFE71F
:105C200004980068C068800748B9FFE70499486A8B
:105C300040F40010486201208DF81700DDE00FE00D
:105C4000049800680069800748B9FFE70499486A2A
:105C500040F40010486201208DF81700CDE0FFE706
:105C600004980068039900EB0110D0F8B00100F02F
:105C70000400029988600298806858B9FFE7049888
:105C80000068039900EB0110D0F8B001400D0299B3
:105C900008600AE004980068039900EB0110D0F84E
:105CA000B001C00802994860FFE7049800680399B2
:105CB00000EB0110D0F8B00100F002000299C860BA
:105CC00004980068039900EB0110D0F8B40100F0CB
:105CD0000F00082804D3FFE70299082008610BE0B1
:105CE00004980068039900EB0110D0F8B40100F0AB
:105CF0000F0002990861FFE704980068039900EB20
:105D00000110D0F8B40180B2000A029988610498A9
:105D10000068039900EB0110D0F8B401000C02995F
:105D2000486104980068039900EB0110D0F8B801AD
:105D30000199087004980068039900EB0110D0F8ED
:105D4000B801000A0199487004980068039900EBB3
:105D50000110D0F8B801000C01998870049800680F
:105D6000039900EB0110D0F8B801000E0199C8703A
:105D700004980068039900EB0110D0F8BC01019968
:105D8000087104980068039900EB0110D0F8BC0179
:105D9000000A0199487104980068039900EB01100A
:105DA000D0F8BC01000C019988710498006803992F
:105DB00000EB0110D0F8BC01000E0199C8710398E6
:105DC00038B9FFE704980168C86840F02000C8604F
:105DD00006E004980168086940F020000861FFE7C8
:105DE00000208DF8170008E00499486A40F48020EC
:105DF000486201208DF81700FFE79DF8170006B0F4
:105E00007047000083B0029000200190029890F843
:105E100020008DF803009DF80300012805D0FFE75E
:105E20009DF80300022822D1FFE7029800688068ED
:105E30004001002804D5FFE7019801300190FFE7F9
:105E40000298006880680001002804D5FFE70198E7
:105E500001300190FFE7029800688068C0000028C8
:105E600004D5FFE7019801300190FFE7FFE70198B3
:105E700003B0704780B58AB0099000200890099857
:105E80000068406907900998006840680690099882
:105E900000688068059009980068C06804900998B7
:105EA00000680069039009980068806902909DF875
:105EB0001C00C007002800F09480FFE79DF8140044
:105EC000C00758B3FFE709980168012088609DF872
:105ED00014008007002804D5FFE7099800F0D2FCE1
:105EE0001BE09DF814004007002805D5FFE708983F
:105EF00040F4006008900FE09DF8140000070028AF
:105F000005D5FFE7089840F48050089003E0099811
:105F100000F090FCFFE7FFE7FFE7FFE79DF81500C3
:105F2000C00760B3FFE7099801684FF4807088608C
:105F30009DF815008007002804D5FFE7099800F0B8
:105F4000EFFC1BE09DF815004007002805D5FFE792
:105F5000089840F4005008900FE09DF815000007E5
:105F6000002805D5FFE7089840F48040089003E03A
:105F7000099800F0ADFCFFE7FFE7FFE7FFE79DF8BA
:105F80001600C00760B3FFE7099801684FF480303E
:105F900088609DF816008007002804D5FFE709985F
:105FA00000F00EFD1BE09DF816004007002805D507
:105FB000FFE7089840F4004008900FE09DF81600B5
:105FC0000007002805D5FFE7089840F480300890C6
:105FD00003E0099800F0CCFCFFE7FFE7FFE7FFE7ED
:105FE000FFE79DF81C000007002810D5FFE79DF88B
:105FF0001000C006002809D5FFE7089840F400709B
:106000000890099801681020C860FFE7FFE79DF835
:106010001C00400700280FD5FFE79DF8100000077F
:10602000002808D5FFE7099801680820C86009988A
:1060300000F0F2FAFFE7FFE79DF81C008007002858
:106040000BD5FFE709980068C068800720B1FFE71B
:10605000099800F009FBFFE7FFE79DF81C004006E8
:10606000002810D5FFE79DF80C00C006002809D5D0
:10607000FFE7089840F480600890099801681020B4
:106080000861FFE7FFE79DF81C00800600280FD598
:10609000FFE79DF80C000007002808D5FFE70998E6
:1060A000016808200861099800F006FBFFE7FFE798
:1060B0009DF81C00C00600280BD5FFE70998006872
:1060C0000069800720B1FFE7099800F01DFBFFE79A
:1060D000FFE79DF81E00800700280FD5FFE79DF819
:1060E0001800C006002808D5FFE7099801681020AD
:1060F0004860099800F030FBFFE7FFE79DF81E00BD
:10610000C00778B1FFE79DF818000007002808D500
:10611000FFE70998016808204860099800F078FCBA
:10612000FFE7FFE79DF81D000006002840F18D8085
:10613000FFE79DF818004007002840F18180FFE745
:106140009DF81D00C00750B1FFE79DF80800C0078B
:1061500028B1FFE7089840F001000890FFE79DF89C
:106160001D00800700280BD5FFE79DF80800800779
:10617000002805D5FFE7089840F002000890FFE7E7
:106180009DF81D00400700280BD5FFE79DF808008B
:106190004007002805D5FFE7089840F00400089064
:1061A000FFE79DF81D000007002848D5FFE79DF890
:1061B000080010F0700F42D0FFE7029800F0700066
:1061C00001460191102814D0FFE70198202815D02E
:1061D000FFE70198302816D0FFE70198402817D034
:1061E000FFE70198502818D0FFE70198602819D0E0
:1061F0001DE0089840F00800089019E0089840F069
:106200001000089014E0089840F0200008900FE07B
:10621000089840F0400008900AE0089840F080009C
:10622000089005E0089840F48070089000E0FFE7CF
:1062300009980168886920F070008861FFE7FFE72E
:106240000998016804204860FFE7089848B1FFE713
:10625000089A0999486A104348620998FFF776FC42
:10626000FFE70AB080BD000080B584B002900298BC
:1062700020B9FFE701208DF80F00E0E0029890F8C8
:10628000200020B9FFE7029800F0DEF8FFE702984F
:106290000168086840F00100086001F0A1F9019070
:1062A000FFE7029800684068C007A8B9FFE701F05F
:1062B00097F90199401A0B280DD3FFE70299486A14
:1062C00040F4003048620299052081F82000012046
:1062D0008DF80F00B3E0E4E702980168086820F049
:1062E0000200086001F07CF90190FFE70298006865
:1062F00040688007002815D5FFE701F071F9019982
:10630000401A0B280DD3FFE70299486A40F4003089
:1063100048620299052081F8200001208DF80F00C5
:106320008DE0E3E70298007E012807D1FFE702989D
:106330000168086840F08000086006E00298016883
:10634000086820F080000860FFE70298407E01287E
:1063500007D1FFE702980168086840F04000086034
:1063600006E002980168086820F040000860FFE736
:106370000298807E012807D1FFE70298016808682B
:1063800040F02000086006E002980168086820F0EC
:1063900020000860FFE70298C07E012807D1FFE7D0
:1063A00002980168086820F01000086006E0029872
:1063B0000168086840F010000860FFE70298007F5D
:1063C000012807D1FFE702980168086840F008003B
:1063D000086006E002980168086820F0080008607C
:1063E000FFE70298407F012807D1FFE70298016884
:1063F000086840F00400086006E002980168086838
:1064000020F004000860FFE7029B19685A6898684A
:10641000D3F80CC040EA0C00D3F810C040EA0C00DE
:106420005B691843013A1043C86102990020486231
:10643000029A012182F820108DF80F00FFE79DF8E5
:106440000F0004B080BD000080B596B0159000200C
:10645000149013901290119010901598006846F2C5
:106460000041C4F2000188425CD1FFE740F25C5079
:10647000C2F200000168013101600068012812D1F8
:10648000FFE7FFE700200F9043F64000C4F2020050
:10649000016841F000710160006800F000700F9029
:1064A0000F98FFE7FFE7FFE700200E9043F630006C
:1064B000C4F20200016841F008010160006800F0C8
:1064C00008000E900E98FFE7032010900221119112
:1064D00000210991129113900920149040F6004078
:1064E000C4F2020010A900F06FFE099A1320069072
:1064F0000521089101F00CFB069801F0FFFA0899BC
:10650000099A1420079001F003FB079801F0F6FAAE
:106510000899099A15200A9001F0FAFA0A9801F0F0
:10652000EDFA77E01598006846F60001C4F2000124
:1065300088426ED1FFE7FFE700200D9043F6400050
:10654000C4F20200016841F080610160006800F05F
:1065500080600D900D98FFE740F25C50C2F20000A1
:106560000168013101600068012812D1FFE7FFE7EF
:1065700000200C9043F64000C4F20200016841F094
:1065800000710160006800F000700C900C98FFE74B
:10659000FFE7FFE700200B9043F63000C4F2020053
:1065A000016841F002010160006800F002000B90F8
:1065B0000B98FFE7602010900220119000200490BB
:1065C0001290032013900920149040F20040C4F26E
:1065D000020010A900F0F8FD049A3F200190052167
:1065E000039101F095FA019801F088FA0399049A51
:1065F0004020029001F08CFA029801F07FFA039992
:10660000049A4120059001F083FA059801F076FA8A
:10661000FFE7FFE716B080BD80B582B0019001981A
:10662000FCF7AAFF8DF803009DF80300032819D09A
:10663000FFE79DF8030040F2B442C2F200023421A9
:1066400010FB0120C06960B1FFE79DF8030040F234
:10665000B442C2F20002342110FB0120C06980471D
:10666000FFE7FFE702B080BD80B582B001900198DE
:10667000FCF782FF8DF803009DF80300032819D072
:10668000FFE79DF8030040F2B442C2F20002342159
:1066900010FB0120806960B1FFE79DF8030040F224
:1066A000B442C2F20002342110FB0120806980470D
:1066B000FFE7FFE702B080BD80B582B0019001988E
:1066C000FCF75AFF8DF803009DF80300032819D04A
:1066D000FFE79DF8030040F2B442C2F20002342109
:1066E00010FB0120406A60B1FFE79DF8030040F213
:1066F000B442C2F20002342110FB0120406A8047FC
:10670000FFE7FFE702B080BD80B582B0019001983D
:10671000FCF732FF8DF803009DF80300032819D021
:10672000FFE79DF8030040F2B442C2F200023421B8
:1067300010FB0120006A60B1FFE79DF8030040F202
:10674000B442C2F20002342110FB0120006A8047EB
:10675000FFE7FFE702B080BD80B582B001900198ED
:10676000FCF70AFF8DF803009DF80300032819D0F9
:10677000FFE79DF8030040F2B442C2F20002342168
:1067800010FB0120806A60B1FFE79DF8030040F232
:10679000B442C2F20002342110FB0120806A80471B
:1067A000FFE7FFE702B080BD80B584B00290029899
:1067B00090F8200001282FD1FFE70299022081F8EC
:1067C000200002980168086820F00100086000F0CD
:1067D00007FF0190FFE7029800684068C007A8B172
:1067E000FFE700F0FDFE0199401A0B280DD3FFE7EB
:1067F0000299486A40F4003048620299052081F805
:10680000200001208DF80F000FE0E4E7029900203E
:1068100048628DF80F0008E00299486A40F40020B1
:10682000486201208DF80F00FFE79DF80F0004B0CB
:1068300080BD000080B582B001900198FCF79CFEFD
:106840008DF803009DF80300032819D0FFE79DF899
:10685000030040F2B442C2F20002342110FB0120D6
:10686000C06860B1FFE79DF8030040F2B442C2F295
:106870000002342110FB0120C0688047FFE7FFE7DA
:1068800002B080BD80B582B001900198FCF774FE23
:106890008DF803009DF80300032817D0FFE79DF84B
:1068A00003003421414340F2B440C2F2000040589A
:1068B00058B1FFE79DF803003421414340F2B44052
:1068C000C2F2000040588047FFE7FFE702B080BDFA
:1068D00080B582B001900198FCF74EFE8DF8030060
:1068E0009DF80300032819D0FFE79DF8030040F24C
:1068F000B442C2F20002342110FB0120006960B1F1
:10690000FFE79DF8030040F2B442C2F200023421D6
:1069100010FB012000698047FFE7FFE702B080BD60
:1069200080B582B001900198FCF726FE8DF8030037
:106930009DF80300032819D0FFE79DF8030040F2FB
:10694000B442C2F20002342110FB0120406860B161
:10695000FFE79DF8030040F2B442C2F20002342186
:1069600010FB012040688047FFE7FFE702B080BDD1
:1069700080B582B001900198FCF7FEFD8DF8030010
:106980009DF80300032819D0FFE79DF8030040F2AB
:10699000B442C2F20002342110FB0120406960B110
:1069A000FFE79DF8030040F2B442C2F20002342136
:1069B00010FB012040698047FFE7FFE702B080BD80
:1069C00080B582B001900198FCF7D6FD8DF80300E8
:1069D0009DF80300032819D0FFE79DF8030040F25B
:1069E000B442C2F20002342110FB0120806860B181
:1069F000FFE79DF8030040F2B442C2F200023421E6
:106A000010FB012080688047FFE7FFE702B080BDF0
:106A100080B582B001900198FCF7AEFD8DF80300BF
:106A20009DF80300032819D0FFE79DF8030040F20A
:106A3000B442C2F20002342110FB0120C06A60B1EE
:106A4000FFE79DF8030040F2B442C2F20002342195
:106A500010FB0120C06A8047FFE7FFE702B080BD5E
:106A600080B584B002900298806D019000F0B8FD6E
:106A70000090029890F8350002280DD0FFE70299A7
:106A800080204865FFE70299002081F83400FFE785
:106A900001208DF80F0055E002980168086820F089
:106AA0001600086002980168486920F0800048617B
:106AB0000298006C20B9FFE70298806C38B1FFE7BC
:106AC00002980168086820F008000860FFE7029853
:106AD0000168086820F001000860FFE7029800687C
:106AE0000068C007C8B1FFE700F07AFD0099401ABE
:106AF000062811D3FFE70299202048650299032058
:106B000081F83500FFE70299002081F83400FFE7A3
:106B100003208DF80F0015E0E0E70298C16D3F20DB
:106B20008840019988600299012081F83500FFE7CB
:106B30000299002081F83400FFE7FFE700208DF87C
:106B40000F00FFE79DF80F0004B080BD82B00090F9
:106B5000009890F83500022807D0FFE700998020C0
:106B6000486501208DF807000EE00099052081F8A6
:106B7000350000980168086820F001000860FFE710
:106B800000208DF80700FFE79DF8070002B070476E
:106B900080B586B005900020039040F20000C2F25C
:106BA0000000006848F2B511C1F64E31A0FB01109B
:106BB000800A02900598806D019001980068049009
:106BC00004980599C96DC840000700281AD5FFE749
:106BD0000598006800684007002812D5FFE705986F
:106BE0000168086820F0040008600598C16D08205D
:106BF0008840019988600599486D40F0010048651A
:106C0000FFE7FFE704980599C96DC840C007A0B128
:106C1000FFE7059800684069000600280CD5FFE7EB
:106C20000598C16D01208840019988600599486DDB
:106C300040F002004865FFE7FFE704980599C96D39
:106C4000C8404007002814D5FFE705980068006891
:106C5000800700280CD5FFE70598C16D0420884007
:106C6000019988600599486D40F004004865FFE788
:106C7000FFE704980599C96DC840C006002847D5AC
:106C8000FFE7059800680068000700283FD5FFE788
:106C90000598C16D102088400199886005980068AA
:106CA0000068400300281AD5FFE7059800680068CF
:106CB0000003002809D4FFE70598006C20B1FFE726
:106CC0000598016C8847FFE708E00598806C20B1C3
:106CD000FFE70598816C8847FFE7FFE716E0059816
:106CE00000680068C005002807D4FFE70598016820
:106CF000086820F008000860FFE70598006C20B1E4
:106D0000FFE70598016C8847FFE7FFE7FFE7FFE72C
:106D100004980599C96DC8408006002840F18D800F
:106D2000FFE7059800680068C006002840F18480ED
:106D3000FFE70598C16D202088400199886005987B
:106D400090F83500052834D1FFE7059801680868F8
:106D500020F01600086005980168486920F080005E
:106D600048610598006C20B9FFE70598806C38B140
:106D7000FFE705980168086820F008000860FFE751
:106D80000598C16D3F2088400199886005990120D0
:106D900081F83500FFE70599002081F83400FFE70E
:106DA0000598006D20B1FFE70598016D8847FFE762
:106DB0007BE0059800680068400300281AD5FFE7CB
:106DC0000598006800680003002809D4FFE70598CB
:106DD000406C20B1FFE70598416C8847FFE708E069
:106DE0000598C06B20B1FFE70598C16B8847FFE7A6
:106DF000FFE720E0059800680068C005002811D46E
:106E0000FFE705980168086820F010000860059900
:106E1000012081F83500FFE70599002081F8340052
:106E2000FFE7FFE70598C06B20B1FFE70598C16B4E
:106E30008847FFE7FFE7FFE7FFE70598406DA0B34E
:106E4000FFE70598406DC00730B3FFE705990520BF
:106E500081F8350005980168086820F00100086095
:106E6000FFE70398013003900299884201D9FFE7B8
:106E700007E0FFE7059800680068C0070028F0D128
:106E8000FFE70599012081F83500FFE7059900200B
:106E900081F83400FFE7FFE70598C06C20B1FFE7F9
:106EA0000598C16C8847FFE7FFE706B080BD00008A
:106EB00080B586B004900020039000F091FB029012
:106EC000049820B9FFE701208DF81700A3E004988B
:106ED000406A08B1FFE7FFE70499022081F8350016
:106EE000FFE70499002081F83400FFE70498016867
:106EF000086820F001000860FFE704980068006857
:106F0000C00790B1FFE700F06BFB0299401A06281A
:106F10000AD3FFE70499202048650499032081F8EB
:106F200035008DF8170076E0E7E704980068006800
:106F30000390039848F23F01CFF2100108400390FC
:106F4000049900914868D1F808C0CB680A6940EA02
:106F50000C00184310434A6910438A691043CA69F8
:106F60001043096A01430398084303900498406A58
:106F7000042808D1FFE70499C86A096B0143039804
:106F800008430390FFE70398049909680860049890
:106F9000006840690390039820F00700039004986C
:106FA000416A0398084303900498406A04281AD160
:106FB000FFE70498816A0398084303900498C06A25
:106FC00080B1FFE70498FDF7F7FD50B1FFE70499A2
:106FD000402048650499012081F835008DF817009C
:106FE00019E0FFE7FFE703980499096848610498EE
:106FF000FDF7B6FD01900498C16D3F2088400199CE
:107000008860049900204865049A012182F83510AF
:107010008DF81700FFE79DF8170006B080BD00004F
:1070200080B588B0069005910492039300208DF8F6
:107030000B000698806D0190FFE7069890F83400E9
:10704000012804D1FFE702208DF81F0045E00699D2
:10705000012081F83400FFE7FFE7069890F835003B
:1070600001282BD1FFE70699022081F83500069907
:107070000020486506980599049A039BFDF714FEC5
:107080000698C16D3F208840019988600698016884
:10709000086840F0160008600698006C38B1FFE7F9
:1070A00006980168086840F008000860FFE7069845
:1070B0000168086840F00100086009E0FFE70699F0
:1070C000002081F83400FFE702208DF80B00FFE775
:1070D0009DF80B008DF81F00FFE79DF81F0008B01A
:1070E00080BD000080B584B0039000F079FA029072
:1070F000039801900198013048B1FFE740F26430F5
:10710000C2F200000178019808440190FFE7FFE710
:1071100000F066FA0299401A0199884201D2FFE70D
:10712000F6E704B080BD000080B582B0ADF806007F
:1071300000208DF80500FFE79DF805000F2824DCEE
:10714000FFE7BDF806009DF80510C840C007A8B1CC
:10715000FFE79DF8051040F21C50C2F2000050F805
:10716000210050B1FFE79DF8051040F21C50C2F21B
:10717000000050F821008047FFE7FFE7FFE79DF898
:10718000050001308DF80500D6E702B080BD000093
:1071900080B582B0ADF8060043F61440C4F2010099
:1071A0000068BDF8061008420CD0FFE7BDF80600E5
:1071B00043F61441C4F201010860BDF80600FFF770
:1071C000B3FFFFE702B080BD8EB00D900C910020A0
:1071D0000A90099008900B90FFE70B980F2800F297
:1071E000CC81FFE70B99012088400A900C98006839
:1071F0000A990840099009980A99884240F0B88194
:10720000FFE70C98406800F00300012807D0FFE773
:107210000C98406800F0030002282FD1FFE70D987A
:10722000806808900B984100032000FA01F108984B
:10723000884308900C98C0680B99490000FA01F146
:1072400008980843089008980D9988600D98406840
:1072500008900B99012000FA01F1089888430890E2
:107260000C984068C0F300100B9900FA01F10898DF
:107270000843089008980D994860FFE70C9840680B
:1072800000F00300032818D0FFE70D98C0680890AD
:107290000B984100032000FA01F1089888430890F8
:1072A0000C9880680B99490000FA01F1089808438E
:1072B000089008980D99C860FFE70C98406800F0A6
:1072C0000300022826D1FFE70D980B996FF0030207
:1072D00002EA51010844006A08900B9800F0070088
:1072E00081000F2000FA01F10898884308900C985B
:1072F00000690B9901F00701890000FA01F1089873
:107300000843089008980D990B9B02EA5302114418
:107310000862FFE70D98006808900B984100032071
:1073200000FA01F10898884308900C98406800F032
:1073300003000B99490000FA01F1089808430890EE
:1073400008980D9908600C9880798007002800F053
:107350000E81FFE7FFE70020079043F64400C4F2E8
:107360000200016841F480410160006800F480403F
:1073700007900798FFE70B9820F0030043F60801F9
:10738000C4F20101405808900B9800F003008100FE
:107390000F2000FA01F10898884308900D98002109
:1073A000C4F20201884203D1FFE7002006905EE0AC
:1073B0000D9840F20041C4F20201884203D1FFE778
:1073C0000120059050E00D9840F60001C4F2020142
:1073D000884203D1FFE70220049042E00D9840F676
:1073E0000041C4F20201884203D1FFE70320039069
:1073F00034E00D9841F20001C4F20201884203D149
:10740000FFE70420029026E00D9841F20041C4F20B
:107410000201884203D1FFE70520019018E00D9892
:1074200041F60001C4F20201884203D1FFE70620C1
:1074300000900AE00D9941F60042C4F202020820D1
:10744000914208BF07200090FFE700980190FFE7F6
:1074500001980290FFE702980390FFE703980490D9
:10746000FFE704980590FFE705980690FFE7069868
:10747000C0B20B9901F00301890000FA01F10898EC
:107480000843089008980B9921F0030143F608027D
:10749000C4F20102885043F60840C4F201000068BB
:1074A000089009990898884308900C988079C0063C
:1074B000002805D5FFE70999089808430890FFE7D9
:1074C000089843F60841C4F20101086043F60C40F5
:1074D000C4F2010000680890099908988843089050
:1074E0000C9880798006002805D5FFE7099908984F
:1074F00008430890FFE7089843F60C41C4F20101E5
:10750000086043F60440C4F201000068089009993D
:107510000898884308900C9880798007002805D542
:10752000FFE70999089808430890FFE7089843F691
:107530000441C4F20101086043F60040C4F20100B6
:107540000068089009990898884308900C988079F9
:10755000C00728B1FFE70999089808430890FFE79A
:10756000089843F60041C4F201010860FFE7FFE715
:10757000FFE70B9801300B902FE60EB0704700002C
:1075800082B00190ADF8021001980069BDF80210B8
:10759000084204D0FFE701208DF8010003E000203D
:1075A0008DF80100FFE79DF8010002B07047000070
:1075B00082B00190ADF802108DF801209DF8010015
:1075C00028B1FFE7BDF802000199886105E0BDF828
:1075D0000200000401998861FFE702B070470000D3
:1075E00048F2D460C2F200000068704780B58EB0E7
:1075F0000C900C9820B9FFE701208DF8370043E18B
:107600000C9890F83D0040B9FFE70C99002081F8F4
:107610003C000C9800F03CF9FFE70C99242081F81D
:107620003D000C980168086820F0010008600C9883
:107630000168086840F4004008600C980168086818
:1076400020F40040086000F0BDFB0A900C984068F0
:1076500048F2A061C0F2010188420BD8FFE70A9905
:1076600048F28042C0F21E020020914238BF012041
:1076700009900AE00A9940F60012C0F23D0200208B
:10768000914238BF01200990FFE70998012804D1F1
:10769000FFE701208DF83700F6E00A984DF6836188
:1076A000C4F21B31A0FB0110800C0B900C980068F9
:1076B000406820F03F000B9908430C990968486026
:1076C0000C980068006A20F03F0008900C98406811
:1076D00048F2A061C0F20101884204D8FFE70B988C
:1076E000013007900EE00B984FF49671484344F632
:1076F000D351C1F26201A0FB0101012000EB911006
:107700000790FFE70898079908430C9909680862F1
:107710000C980068C0694CF6FF71884306900C987D
:10772000406848F2A061C0F2010188421FD8FFE71B
:107730000A9801380C9949684900B0FBF1F0013012
:107740006FF31F30032803D8FFE7042005900BE0F8
:107750000A9801380C9949684900B0FBF1F00130F2
:107760006FF31F300590FFE7059804904CE00C98EC
:10777000806868B9FFE70A9801380C99496801EBFD
:107780004101B0FBF1F001306FF31F3003900DE0C9
:107790000A9801380C99496819225143B0FBF1F05D
:1077A0000130042161F31F300390FFE703980005C7
:1077B00018B9FFE70120029023E00C98806868B9AF
:1077C000FFE70A9801380C99496801EB4101B0FBC9
:1077D000F1F001306FF31F3001900DE00A9801388D
:1077E0000C99496819225143B0FBF1F00130042192
:1077F00061F31F300190FFE7019840F400400290D0
:10780000FFE702980490FFE70698049908430C9953
:107810000968C8610C980068006820F0C0000C9BE3
:107820001968DA691B6A1A43104308600C980068EB
:10783000806848F2FF3188430C9A1168D368126956
:107840001A43104388600C980068C06820F0FF005D
:107850000C9B19685A699B691A431043C8600C98BD
:107860000168086840F0010008600C990020086475
:107870000C9A202182F83D100C9908630C9981F82C
:107880003E008DF83700FFE79DF837000EB080BD51
:1078900080B590B00F9000200E900D900C900B9042
:1078A0000A900F98006845F60041C4F20001884232
:1078B00040F08980FFE7FFE70020099043F63000A1
:1078C000C4F20200016841F004010160006800F0A8
:1078D000040009900998FFE7FFE70020089043F6AD
:1078E0003000C4F20200016841F00101016000684B
:1078F00000F0010008900898FFE74FF400700A902C
:10790000122002900B90002003900C900320049012
:107910000D90042005900E9040F60000C4F2020085
:107920000AA90691FFF750FCDDF808C0039B049AF2
:10793000059806994FF4807ECDF828E0CDF82CC04C
:107940000C930D920E900020C4F20200FFF73CFC55
:10795000FFE70020079043F64000C4F202000168F0
:1079600041F400010160006800F4000007900798EE
:10797000FFE740F6B440C2F20000019046F2400139
:10798000C4F2020101604FF0C061416000218160DA
:10799000C1604FF48062026141618161C161016235
:1079A0004162FFF785FA18B1FFE7FDF7A5FBFFE796
:1079B000FFE70F9840F6B441C2F2000181630F98CF
:1079C0008863FFE7FFE710B080BD000040F264303D
:1079D000C2F20000027848F2D461C2F200010868E5
:1079E000104408607047000080B543F60041C4F2BF
:1079F0000201086840F400700860086840F4806084
:107A00000860086840F480700860032000F09AF86D
:107A10000F2000F005F800F03BF8002080BD0000CA
:107A200080B582B0009040F20000C2F20000006811
:107A300040F26431C2F200010A784FF47A71B1FB6E
:107A4000F2F1B0FBF1F001F0F3FE20B1FFE701200D
:107A50008DF8070018E000980F280DD8FFE700996F
:107A60004FF0FF30002200F053F8009840F26831E8
:107A7000C2F20001086003E001208DF8070003E076
:107A800000208DF80700FFE79DF8070002B080BDD9
:107A900080B582B0FFE70020019043F64400C4F2B5
:107AA0000200016841F480410160006800F48040F8
:107AB00001900198FFE7FFE70020009043F64000A7
:107AC000C4F20200016841F080510160006800F0DA
:107AD000805000900098FFE76FF001000F21002216
:107AE00000F016F802B080BD80B582B08DF80700B6
:107AF0009DF9070008F0E2F802B080BD80B582B0C1
:107B00008DF807009DF9070008F0F4F802B080BD79
:107B100080B586B08DF81700049103920020029082
:107B200008F000F902909DF917000190029804995D
:107B3000039A04F059FE0146019808F0FBF806B0DC
:107B400080BD000080B582B00190019808F036F940
:107B500002B080BD80B584B002900191029820B936
:107B6000FFE701208DF80F0021E1019843F6004165
:107B7000C4F20201096801F00701884212D9FFE747
:107B8000019943F60040C4F202000170006800F061
:107B900007000199884204D0FFE701208DF80F000B
:107BA00005E1FFE702980078800700282AD5FFE763
:107BB000029800784007002809D5FFE743F608013E
:107BC000C4F20201086840F4E0500860FFE7029840
:107BD00000780007002809D5FFE743F60801C4F242
:107BE0000201086840F460400860FFE743F60801BE
:107BF000C4F20201086820F0F000029A9268104373
:107C00000860FFE702980078C00700286ED0FFE701
:107C100002984068012811D1FFE743F60000C4F242
:107C20000200006800F400310020B0EB514F04D195
:107C3000FFE701208DF80F00B9E02CE002984068C2
:107C4000022805D0FFE702984068032811D1FFE71A
:107C500043F60000C4F20200006800F0007100204A
:107C6000B0EB516F04D1FFE701208DF80F009EE0CB
:107C700010E043F60000C4F20200006800F00201C8
:107C80000020B0EB510F04D1FFE701208DF80F0069
:107C90008DE0FFE7FFE743F60801C4F20201086840
:107CA00020F00300029A526810430860FFF798FC26
:107CB0000090FFE743F60800C4F20200006800F0FD
:107CC0000C0002994968B0EB810F0ED0FFE7FFF777
:107CD00087FC0099401A41F28931884204D3FFE7BA
:107CE00003208DF80F0062E0E4E7FFE7019843F618
:107CF0000041C4F20201096801F00701884212D272
:107D0000FFE7019943F60040C4F2020001700068E9
:107D100000F007000199884204D0FFE701208DF8A8
:107D20000F0044E0FFE702980078400700280CD5D8
:107D3000FFE743F60801C4F20201086820F4E050AE
:107D4000029AD26810430860FFE7029800780007A3
:107D500000280DD5FFE743F60801C4F202010868C8
:107D600020F46040029A126940EAC2000860FFE70E
:107D700000F04CF843F60801C4F202010968C9B2E8
:107D80000A0945F6A871C0F60101895CC84040F2B5
:107D90000001C2F20001086040F26830C2F2000047
:107DA0000068FFF73DFE00208DF80F00FFE79DF80B
:107DB0000F0004B080BD000040F20000C2F20000DD
:107DC0000068704780B5FFF7F7FF43F60801C4F27B
:107DD00002010968C1F3822245F6B871C0F60101BB
:107DE000895CC84080BD000080B5FFF7E5FF43F621
:107DF0000801C4F20201096889B24A0B45F6B8715C
:107E0000C0F60101895CC84080BD000080B586B025
:107E10000020059004900390029043F60800C4F2FD
:107E20000200006800F00C000146019140B1FFE73C
:107E3000019804280AD0FFE7019808280CD04FE0E9
:107E400042F20040C0F2F40002904FE041F60030F0
:107E5000C0F2B700029049E043F60400C4F2020009
:107E6000016801F03F01059100684002002813D528
:107E7000FFE743F60400C4F202000068C0F3881074
:107E800041F60031C0F2B701A0FB0101059A0023C1
:107E9000F8F726FA049012E043F60400C4F2020058
:107EA0000068C0F3881042F20041C0F2F401A0FB68
:107EB0000101059A0023F8F713FA0490FFE743F64F
:107EC0000400C4F20200006800F44031022000EB1C
:107ED000D130039004980399B0FBF1F0029005E0D3
:107EE00042F20040C0F2F4000290FFE7029806B0B0
:107EF00080BD000080B586B00490049820B9FFE7EB
:107F000001208DF8170050E304980078C00700287E
:107F100000F0A580FFE743F60800C4F20200006805
:107F200000F00C00042813D0FFE743F60800C4F269
:107F30000200006800F00C0008281ED1FFE743F69D
:107F40000400C4F2020000684002002815D5FFE7D3
:107F500043F60000C4F20200006800F40031002083
:107F6000B0EB514F08D0FFE70498406820B9FFE715
:107F700001208DF8170018E370E0FFE704984068CF
:107F8000B0F5803F09D1FFE743F60001C4F20201DA
:107F9000086840F48030086020E004984068B0F53C
:107FA000A02F0DD1FFE743F60001C4F202010868DB
:107FB00040F480200860086840F4803008600CE0DD
:107FC00043F60001C4F20201086820F48030086022
:107FD000086820F480200860FFE7FFE7FFE70498C7
:107FE0004068E8B1FFE7FFF7FBFA0390FFE743F6CD
:107FF0000000C4F20200006800F400310020B0EB81
:10800000514F0CD1FFE7FFF7EBFA0399401A6528AF
:1080100004D3FFE703208DF81700C6E2E7E71CE072
:10802000FFF7DEFA0390FFE743F60000C4F2020018
:10803000006800F400310020B0EB514F0CD0FFE796
:10804000FFF7CEFA0399401A652804D3FFE703200F
:108050008DF81700A9E2E7E7FFE7FFE7FFE70498DD
:1080600000788007002840F19680FFE743F608007B
:10807000C4F20200006810F00C0F13D0FFE743F6C3
:108080000800C4F20200006800F00C0008282CD19F
:10809000FFE743F60400C4F2020000684002002833
:1080A00023D4FFE743F60000C4F20200006800F0AA
:1080B00002010020B0EB510F09D0FFE70498C0681F
:1080C000012804D0FFE701208DF817006DE243F688
:1080D0000001C4F20201086820F0F800049A126955
:1080E00040EAC2000860FFE754E00498C06870B33B
:1080F000FFE70021C4F2472101200860FFF770FA72
:108100000390FFE743F60000C4F20200006800F0AD
:1081100002010020B0EB510F0CD1FFE7FFF760FA2E
:108120000399401A032804D3FFE703208DF81700B2
:108130003BE2E7E743F60001C4F20201086820F0E1
:10814000F800049A126940EAC200086021E00021A8
:10815000C4F2472100200860FFF742FA0390FFE7CE
:1081600043F60000C4F20200006800F002010020A3
:10817000B0EB510F0CD0FFE7FFF732FA0399401A2A
:10818000032804D3FFE703208DF817000DE2E7E78B
:10819000FFE7FFE7FFE704980078000700284BD5CA
:1081A000FFE70498406918B3FFE740F68061C4F226
:1081B000472101200860FFF713FA0390FFE743F619
:1081C0007400C4F20200006800F002010020B0EB6D
:1081D000510F0CD1FFE7FFF703FA0399401A032868
:1081E00004D3FFE703208DF81700DEE1E7E722E084
:1081F00040F68061C4F2472100200860FFF7F0F9E3
:108200000390FFE743F67400C4F20200006800F038
:1082100002010020B0EB510F0CD0FFE7FFF7E0F9AF
:108220000399401A032804D3FFE703208DF81700B1
:10823000BBE1E7E7FFE7FFE7049800784007002885
:1082400040F1CE80FFE700208DF8070043F64000A4
:10825000C4F202000068C000002815D4FFE7FFE761
:108260000020009043F64000C4F20200016841F093
:1082700080510160006800F0805000900098FFE796
:1082800001208DF80700FFE747F20000C4F200006C
:108290000068C005002822D4FFE747F20001C4F2BD
:1082A0000001086840F480700860FFF799F90390B6
:1082B000FFE747F20000C4F200000068C005002894
:1082C0000CD4FFE7FFF78CF90399401A032804D375
:1082D000FFE703208DF8170067E1EAE7FFE7FFE714
:1082E00004988068012809D1FFE743F67001C4F2C1
:1082F0000201086840F0010008601FE004988068EF
:1083000005280DD1FFE743F67001C4F202010868A9
:1083100040F004000860086840F0010008600CE0CC
:1083200043F67001C4F20201086820F00100086001
:10833000086820F004000860FFE7FFE7FFE7049803
:108340008068F8B1FFE7FFF74BF90390FFE743F6CA
:108350007000C4F20200006800F002010020B0EBDF
:10836000510F0ED1FFE7FFF73BF90399401A41F295
:108370008931884204D3FFE703208DF8170014E108
:10838000E5E71EE0FFF72CF90390FFE743F67000E6
:10839000C4F20200006800F002010020B0EB510FAF
:1083A0000ED0FFE7FFF71CF90399401A41F289311B
:1083B000884204D3FFE703208DF81700F5E0E5E7D6
:1083C000FFE79DF80700012809D1FFE743F64001C8
:1083D000C4F20201086820F080500860FFE7FFE760
:1083E00004988069002800F0DC80FFE743F608006D
:1083F000C4F20200006800F00C00082800F085803C
:10840000FFE70498806902285CD1FFE76021C4F28D
:10841000472100200860FFF7E3F80390FFE743F6E9
:108420000000C4F20200006800F000710020B0EB10
:10843000516F0CD0FFE7FFF7D3F80399401A0328D8
:1084400004D3FFE703208DF81700AEE0E7E70499B7
:10845000C869D1F820C04B6A8A6A40EA0C0040EA39
:108460008310D2034FF6FF739A43A2F58032104374
:10847000C96A40EA016043F60401C4F202010860DF
:108480006021C4F2472101200860FFF7A9F803909A
:10849000FFE743F60000C4F20200006800F000713C
:1084A0000020B0EB516F0CD1FFE7FFF799F803996B
:1084B000401A032804D3FFE703208DF8170074E067
:1084C000E7E721E06021C4F2472100200860FFF7C0
:1084D00087F80390FFE743F60000C4F2020000684B
:1084E00000F000710020B0EB516F0CD0FFE7FFF7F8
:1084F00077F80399401A032804D3FFE703208DF887
:10850000170052E0E7E7FFE74AE004988069012896
:1085100004D1FFE701208DF8170046E043F6040080
:10852000C4F202000068029004988069012831D0EA
:10853000FFE7029800F480000499C969884229D1B4
:10854000FFE7029800F03F000499096A884221D1B0
:10855000FFE7029847F6C07108400499496AB0EBFA
:10856000811F17D1FFE7029800F440300499896A0F
:10857000C9034FF6FF729143A1F58031884209D1BA
:10858000FFE7029800F070600499C96AB0EB016FD0
:1085900004D0FFE701208DF8170006E0FFE7FFE7B2
:1085A000FFE700208DF81700FFE79DF8170006B0E1
:1085B00080BD000080B582B00190019804F0FAFD02
:1085C0008DF803009DF8030002281BD0FFE70198F7
:1085D00004F0F0FD014640F26450C2F2000000EBEE
:1085E0004110806968B1FFE7019804F0E3FD01469E
:1085F00040F26450C2F2000000EB411080698047F5
:10860000FFE7FFE702B080BD80B584B0029002981A
:1086100020B9FFE701208DF80F0071E00298406A51
:1086200060B9FFE702984068B0F5827F01D1FFE7AB
:1086300003E002990020C861FFE705E002990020ED
:10864000086102994861FFE7029900208862029858
:1086500090F8510040B9FFE70299002081F85000DE
:10866000029800F051F8FFE70299022081F85100CA
:1086700002980168086820F040000860029A0192A0
:1086800011685068D2F808C0D36800F482700CF406
:10869000044C604403F400631844136903F00203BC
:1086A0001844536903F001031844936903F40073F9
:1086B0001844D36903F038031844136A03F08003A5
:1086C0001843926A02F4005210430860029A508BD9
:1086D00000F004001168526A02F010021044486071
:1086E00002980168C86920F40060C86102990020FE
:1086F0004865029A012182F851108DF80F00FFE7BA
:108700009DF80F0004B080BD80B590B00F900020A0
:108710000E900D900C900B900A900F98006843F209
:108720000001C4F20101884240F0B280FFE7FFE798
:108730000020099043F64400C4F20200016841F4AD
:1087400080510160006800F4805009900998FFE7AB
:10875000FFE70020089043F63000C4F202000168F1
:1087600041F002010160006800F0020008900898E2
:10877000FFE7FFE70020079043F63000C4F2020055
:10878000016841F001010160006800F001000790FC
:108790000798FFE718200A90022001900B90002014
:1087A00005900C90032002900D90052003900E90F0
:1087B00040F20040C4F202000AA90491FEF704FD51
:1087C000DDF804C0029A03980499059B4FF0800ECF
:1087D000CDF828E0CDF82CC00C930D920E9000201F
:1087E000C4F20200FEF7F0FC059940F61450C2F204
:1087F0000000069046F24042C4F2020202604FF0CE
:10880000C06242608160C1604FF480620261416178
:108810008161C16101624162FEF74AFB18B1FFE765
:10882000FCF76AFCFFE7FFE70F9840F61451C2F22D
:108830000001C1640F988863FFE740F67450C2F2EC
:108840000000009046F25841C4F2020101604FF06E
:10885000C0614160402181600021C1604FF48062AD
:10886000026141618161C16101624162FEF720FBE9
:1088700018B1FFE7FCF740FCFFE7FFE70F9840F671
:108880007451C2F2000181640F988863FFE7FFE72B
:1088900010B080BD80B588B006900591ADF812206B
:1088A0000393069890F85100012804D0FFE70220B6
:1088B0008DF81F0011E1059820B1FFE7BDF8120007
:1088C00020B9FFE701208DF81F0006E106984068F7
:1088D000B0F5827F16D1FFE70698806890B9FFE770
:1088E0000699042081F851000698059ABDF81230C7
:1088F0000399EC46CCF80010114600F065FB8DF8AA
:108900001F00EAE0FEF76CFE0290FFE7069890F881
:108910005000012804D1FFE702208DF81F00DCE0A1
:108920000699012081F85000FFE7FFE7069904202F
:1089300081F851000699002048650599069A9163CF
:10894000BDF81210069A9187BDF81210069AD187C9
:1089500006990863069988860699C8860699086468
:108960000699486406988068B0F5004F0DD1FFE77E
:1089700006980168086820F04000086006980168C1
:10898000086820F480400860FFE7069800680068E7
:1089900000F04000402807D0FFE70698016808680B
:1089A00040F040000860FFE70698C068D0BBFFE7D2
:1089B000FFE70698C08FA0B3FFE7069800688068BD
:1089C000C00778B1FFE706980068007B0699896BBD
:1089D00008700699886B013088630699C88F013842
:1089E000C8871DE0FEF7FCFD0299401A03998842F2
:1089F00004D3FFE70398013018B9FFE7039870B973
:108A0000FFE70699012081F85100FFE70699002051
:108A100081F85000FFE703208DF81F005DE0FFE7BD
:108A2000C7E739E0FFE70698C08FA0B3FFE70698D5
:108A300000688068C00778B1FFE706980068C068E2
:108A40000699896B08800699886B023088630699BD
:108A5000C88F0138C8871DE0FEF7C2FD0299401A91
:108A60000399884204D3FFE70398013018B9FFE760
:108A7000039870B9FFE70699012081F85100FFE7DC
:108A80000699002081F85000FFE703208DF81F00B1
:108A900023E0FFE7C7E7FFE706980399029A04F08F
:108AA000B1FA20B1FFE7069920204865FFE7069953
:108AB000012081F85100FFE70699002081F850005D
:108AC000FFE70698406D20B1FFE701208DF81F00F9
:108AD00003E000208DF81F00FFE79DF81F0008B09D
:108AE00080BD000080B584B002900191ADF80220F5
:108AF000029890F85100012804D0FFE702208DF879
:108B00000F00B7E0019820B1FFE7BDF8020020B9DF
:108B1000FFE701208DF80F00ACE002988068A0B953
:108B2000FFE702984068B0F5827F0ED1FFE7029917
:108B3000042081F851000298019ABDF802301146D4
:108B400000F014FC8DF80F0094E0FFE7029890F815
:108B50005000012804D1FFE702208DF80F0089E0C2
:108B60000299012081F85000FFE7FFE702990420F5
:108B700081F851000299002048650199029A916399
:108B8000BDF80210029A9187BDF80210029AD187AF
:108B90000299086402994864029988860299C886F5
:108BA00002988068B0F5004F0DD1FFE70298016888
:108BB000086820F04000086002980168086820F406
:108BC00080400860FFE70298C16C4CF6E950C0F69F
:108BD000000008640298C16C4CF63160C0F60000D9
:108BE000C8630298C16C4CF6B550C0F60000C8646A
:108BF0000298C16C00200865029B19689A6BD86CBA
:108C00000C31DB8FFEF70CFA78B1FFE70299486D63
:108C100040F010004865FFE70299002081F85000FD
:108C2000FFE701208DF80F0024E00298006800683B
:108C300000F04000402807D0FFE70298016808686C
:108C400040F040000860FFE7FFE70299002081F84C
:108C50005000FFE702980168486840F02000486033
:108C600002980168486840F00100486000208DF8D3
:108C70000F00FFE79DF80F0004B080BD80B582B003
:108C80000190019804F096FA8DF803009DF8030016
:108C900002281BD0FFE7019804F08CFA014640F24D
:108CA0006450C2F2000000EB4110406868B1FFE779
:108CB000019804F07FFA014640F26450C2F20000CD
:108CC00000EB411040688047FFE7FFE702B080BD3E
:108CD00080B582B00190019804F06CFA8DF8030021
:108CE0009DF8030002281BD0FFE7019804F062FA08
:108CF000014640F26450C2F2000000EB41100069EE
:108D000068B1FFE7019804F055FA014640F264505B
:108D1000C2F2000000EB411000698047FFE7FFE767
:108D200002B080BD80B588B006900591ADF81220E4
:108D30000393FEF755FC0290BDF81200ADF8060053
:108D4000069890F85100012804D0FFE702208DF822
:108D50001F0034E1059820B1FFE7BDF8120020B9EB
:108D6000FFE701208DF81F0029E1FFE7069890F842
:108D70005000012804D1FFE702208DF81F001EE1FA
:108D80000699012081F85000FFE7FFE706990320CC
:108D900081F851000699002048650599069A1163EB
:108DA000BDF81210069A9186BDF81210069AD18667
:108DB00006998863069988870699C8870699486442
:108DC0000699086406988068B0F5004F0DD1FFE75A
:108DD00006980168086820F040000860069801685D
:108DE000086840F480400860FFE706980068006863
:108DF00000F04000402807D0FFE7069801680868A7
:108E000040F040000860FFE70698C068B0F5006FCA
:108E100051D1FFE70698406828B1FFE7BDF806008A
:108E200001280ED1FFE706980168006B0088C86032
:108E30000699086B023008630699C88E0138C88607
:108E4000FFE7FFE70698C08EA0B3FFE7069800682B
:108E50008068800700280ED5FFE706980168006B40
:108E60000088C8600699086B023008630699C88EAE
:108E70000138C8861DE0FEF7B3FB0299401A03993A
:108E8000884204D3FFE70398013018B9FFE703983D
:108E900070B9FFE70699012081F85100FFE70699B4
:108EA000002081F85000FFE703208DF81F0086E0C6
:108EB000FFE7C7E750E00698406828B1FFE7BDF834
:108EC000060001280ED1FFE706980168006B0078C4
:108ED00008730699086B013008630699C88E01383B
:108EE000C886FFE7FFE70698C08EA0B3FFE70698A5
:108EF00000688068800700280ED5FFE706980168A3
:108F0000006B007808730699086B013008630699B6
:108F1000C88E0138C8861DE0FEF762FB0299401A30
:108F20000399884204D3FFE70398013018B9FFE79B
:108F3000039870B9FFE70699012081F85100FFE717
:108F40000699002081F85000FFE703208DF81F00EC
:108F500035E0FFE7C7E7FFE706980399029A04F0B8
:108F6000C3F820B1FFE7069920204865FFE706987F
:108F7000806870B9FFE7FFE700200090069800685E
:108F8000C068009006980068806800900098FFE72D
:108F9000FFE70699012081F85100FFE706990020BC
:108FA00081F85000FFE70698406D20B1FFE70120EF
:108FB0008DF81F0003E000208DF81F00FFE79DF8EB
:108FC0001F0008B080BD000080B58CB0DDF838C04F
:108FD0000A9009910892ADF81E3001200390FEF727
:108FE000FFFA04900A9890F851008DF817000A983B
:108FF00040680690BDF81E00ADF81C009DF81700F3
:10900000012812D0FFE70698B0F5827F09D1FFE76B
:109010000A98806828B9FFE79DF81700042804D053
:10902000FFE702208DF82F009BE1099838B1FFE798
:10903000089820B1FFE7BDF81E0020B9FFE7012026
:109040008DF82F008DE1FFE70A9890F85000012875
:1090500004D1FFE702208DF82F0082E10A99012058
:1090600081F85000FFE7FFE70A9890F851000428C4
:1090700005D0FFE70A99052081F85100FFE70A991A
:109080000020486508990A9A9163BDF81E100A9A53
:10909000D187BDF81E100A9A918709990A9A11631F
:1090A000BDF81E100A9AD186BDF81E100A9A918644
:1090B0000A9908640A9948640A980068006800F0F0
:1090C0004000402807D0FFE70A980168086840F090
:1090D00040000860FFE70A98C068B0F5006F40F0F4
:1090E0008180FFE70A98406828B1FFE7BDF81C00BF
:1090F00001280ED1FFE70A980168006B0088C8605C
:109100000A99086B023008630A99C88E0138C8862C
:10911000FFE7FFE70A98C18E0120019039B9FFE708
:109120000A98C08F002818BF01200190FFE701981E
:10913000C007002855D0FFE70A98006880688007BC
:10914000002818D5FFE70A98C08EA0B1FFE7039862
:10915000012810D1FFE70A980168006B0088C860F9
:109160000A99086B023008630A99C88E0138C886CC
:1091700000200390FFE70A9800688068C007A8B144
:10918000FFE70A98C08F88B1FFE70A980068C068B7
:109190000A99896B08800A99886B023088630A995A
:1091A000C88F0138C88701200390FFE7FEF718FA3F
:1091B0000499401A0E99884212D3FFE70E980130A5
:1091C00070B1FFE70A99012081F85100FFE70A9981
:1091D000002081F85000FFE703208DF82F00C0E049
:1091E00098E782E00A98406828B1FFE7BDF81C00C4
:1091F00001280ED1FFE70A980168006B0078087318
:109200000A99086B013008630A99C88E0138C8862C
:10921000FFE7FFE70A98C18E0120009039B9FFE708
:109220000A98C08F002818BF01200090FFE700981F
:10923000C007002858D0FFE70A98006880688007B8
:10924000002818D5FFE70A98C08EA0B1FFE7039861
:10925000012810D1FFE70A980168006B00780873B5
:109260000A99086B013008630A99C88E0138C886CC
:1092700000200390FFE70A9800688068C007A8B143
:10928000FFE70A98C08F88B1FFE70A980068C068B6
:109290000A99896B08700A99886B013088630A996A
:1092A000C88F0138C88701200390FFE7FEF798F9BF
:1092B0000499401A0E99884204D3FFE70E980130B2
:1092C00018B9FFE70E9870B9FFE70A99012081F8F5
:1092D0005100FFE70A99002081F85000FFE70320C2
:1092E0008DF82F003DE095E7FFE70A980E99049A64
:1092F00003F0FAFE68B1FFE70A9920204865FFE70E
:109300000A99002081F85000FFE701208DF82F0016
:1093100027E00A98806870B9FFE7FFE70020029015
:109320000A980068C06802900A98006880680290F5
:109330000298FFE7FFE70A99012081F85100FFE753
:109340000A99002081F85000FFE70A98406D20B18B
:10935000FFE701208DF82F0003E000208DF82F009B
:10936000FFE79DF82F000CB080BD000080B588B0ED
:10937000069005910492ADF80E30069890F85100D1
:109380008DF807000698406802909DF807000128B4
:1093900012D0FFE70298B0F5827F09D1FFE7069867
:1093A000806828B9FFE79DF80700042804D0FFE78C
:1093B00002208DF81F00DFE0059838B1FFE7049820
:1093C00020B1FFE7BDF80E0020B9FFE701208DF8BE
:1093D0001F00D1E0FFE7069890F85000012804D163
:1093E000FFE702208DF81F00C6E00699012081F8F2
:1093F0005000FFE7FFE7069890F85100042805D0D9
:10940000FFE70699052081F85100FFE70699002043
:1094100048650599069A1163BDF80E10069A918663
:10942000BDF80E10069AD1860499069A9163BDF88C
:109430000E10069A9187BDF80E10069AD1870699EC
:10944000086406994864069890F8510004280FD1E2
:10945000FFE70698C16C4CF6E950C0F600000864BE
:109460000698C16C4CF63160C0F60000C8630EE08F
:109470000698C16C4CF61960C0F6000008640698A6
:10948000C16C4CF67D70C0F60000C863FFE706981B
:10949000C16C4CF6B550C0F60000C8640698C16CAB
:1094A00000200865069B19689A6BD86C0C31DB8F1D
:1094B000FDF7B6FD78B1FFE70699486D40F0100062
:1094C0004865FFE70699002081F85000FFE701207A
:1094D0008DF81F0050E006980168486840F00100D0
:1094E00048600698816C002008640699896CC863FE
:1094F0000699896CC8640699896C0865069B1A6888
:10950000196B986C0C32DB8EFDF78AFD78B1FFE7A2
:109510000699486D40F010004865FFE70699002065
:1095200081F85000FFE701208DF81F0024E0069825
:109530000068006800F04000402807D0FFE7069868
:109540000168086840F040000860FFE7FFE70699FF
:10955000002081F85000FFE706980168486840F055
:109560002000486006980168486840F002004860A2
:1095700000208DF81F00FFE79DF81F0008B080BD98
:1095800080B584B002900191ADF80220029890F865
:109590005100012804D0FFE702208DF80F00A1E060
:1095A000019820B1FFE7BDF8020020B9FFE70120D4
:1095B0008DF80F0096E0FFE7029890F85000012820
:1095C00004D1FFE702208DF80F008BE00299012003
:1095D00081F85000FFE7FFE70299032081F851006E
:1095E0000299002048650199029A1163BDF80210A2
:1095F000029A9186BDF80210029AD1860299886378
:109600000299486402990864029988870299C88778
:1096100002988068B0F5004F0DD1FFE7029801680D
:10962000086820F04000086002980168086840F46B
:1096300080400860FFE70298816C4CF60160C0F63C
:10964000000008640298816C4CF6D560C0F60000FA
:10965000C8630298816C4CF6B550C0F60000C8642F
:109660000298816C00200865029B1A68196B986C3F
:109670000C32DB8EFDF7D4FC78B1FFE70299486D20
:1096800040F010004865FFE70299002081F8500083
:10969000FFE701208DF80F0024E0029800680068C1
:1096A00000F04000402807D0FFE7029801680868F2
:1096B00040F040000860FFE7FFE70299002081F8D2
:1096C0005000FFE702980168486840F020004860B9
:1096D00002980168486840F00200486000208DF858
:1096E0000F00FFE79DF80F0004B080BD80B582B089
:1096F0000190019803F05EFD8DF803009DF80300D2
:10970000022815D0FFE79DF80300410140F26450A4
:10971000C2F20000405850B1FFE79DF8030041013C
:1097200040F26450C2F2000040588047FFE7FFE774
:1097300002B080BD80B582B00190019803F03AFD7F
:109740008DF803009DF8030002281BD0FFE7019865
:1097500003F030FD014640F26450C2F2000000EB1D
:109760004110C06868B1FFE7019803F023FD01468E
:1097700040F26450C2F2000000EB4110C068804724
:10978000FFE7FFE702B080BD80B582B0019001988D
:1097900003F010FD8DF803009DF8030002281BD094
:1097A000FFE7019803F006FD014640F26450C2F263
:1097B000000000EB4110806868B1FFE7019803F0FA
:1097C000F9FC014640F26450C2F2000000EB411087
:1097D00080688047FFE7FFE702B080BD80B582B0B8
:1097E0000190019803F0E6FC8DF803009DF803005A
:1097F00002281BD0FFE7019803F0DCFC014640F291
:109800006450C2F2000000EB4110406968B1FFE70C
:10981000019803F0CFFC014640F26450C2F2000010
:1098200000EB411040698047FFE7FFE702B080BDD1
:1098300080B582B00190019804F0ACFD02B080BD0B
:1098400085B003900291FFE7039890F83C0001284F
:1098500004D1FFE702208DF813007EE00399012078
:1098600081F83C00FFE7FFE70399022081F83D0003
:109870000398006840680190039800688068009031
:10988000019820F070000190029801680198084347
:1098900001900198039909684860039800680021C5
:1098A000C4F2010188423CD0FFE703980068B0F1A0
:1098B000804F36D0FFE70398006840F20041C4F2C1
:1098C000000188422DD0FFE70398006840F60001B0
:1098D000C4F20001884224D0FFE70398006840F6F4
:1098E0000041C4F2000188421BD0FFE703980068E2
:1098F00040F20041C4F20101884212D0FFE7039810
:10990000006844F20001C4F20101884209D0FFE777
:109910000398006841F60001C4F2000188420ED1AC
:10992000FFE7009820F080000090029841680098BE
:10993000084300900098039909688860FFE703993D
:10994000012081F83D00FFE70399002081F83C00E9
:10995000FFE700208DF81300FFE79DF8130005B026
:109960007047000080B582B00090009820B9FFE7F2
:1099700001208DF807003FE0009890F83D0040B9C5
:10998000FFE70099002081F83C00009800F038F8CB
:10999000FFE70099022081F83D00009951F8040B7F
:1099A00004F096FD0099012081F84600FFE7009938
:1099B000012081F83E00009981F83F00009981F86C
:1099C0004000009981F84100FFE7FFE7009901207E
:1099D00081F84200009981F84300009981F8440021
:1099E000009981F84500FFE70099012081F83D00CA
:1099F00000208DF80700FFE79DF8070002B080BD4A
:109A000083B002900298006840F60041C4F2000161
:109A1000884212D1FFE7FFE70020019043F64000A3
:109A2000C4F20200016841F008010160006800F022
:109A3000080001900198FFE71BE00298006844F2DB
:109A40000041C4F20101884212D1FFE7FFE7002084
:109A5000009043F64400C4F20200016841F4003172
:109A60000160006800F4003000900098FFE7FFE715
:109A7000FFE703B07047000080B586B00490039103
:109A800000208DF80B00FFE7049890F83C000128B7
:109A900004D1FFE702208DF81700ABE00499012004
:109AA00081F83C00FFE7FFE70499022081F83D00C0
:109AB0000498006880680190019820F07700019078
:109AC000019820F47F40019001980499096888600A
:109AD000039800680090002872D0FFE700981028D3
:109AE0006ED0FFE7009820286AD0FFE70098302862
:109AF00066D0FFE70098402855D0FFE7009850282F
:109B000037D0FFE70098602840D0FFE70098702822
:109B10000BD0FFE70098B0F5805F05D0FFE7009815
:109B2000B0F5005F16D052E055E004980068039B42
:109B30005A689968DB6804F0B9FD04980068806889
:109B40000190019840F0770001900198049909680C
:109B5000886040E004980068039B5A689968DB6855
:109B600004F0A4FD04980168886840F4804088608F
:109B700031E004980068039A5168D26804F082FFCB
:109B800004980068502104F0ABFD24E004980068BC
:109B9000039A5168D26804F09DFF04980068602120
:109BA00004F09EFD17E004980068039A5168D2689B
:109BB00004F068FF04980068402104F091FD0AE079
:109BC000049800680399096804F08AFD03E0012005
:109BD0008DF80B00FFE70499012081F83D00FFE7B5
:109BE0000499002081F83C00FFE79DF80B008DF8F8
:109BF0001700FFE79DF8170006B080BD80B58AB05A
:109C0000099000200890079006900590049009980C
:109C1000006840F60001C4F20001884223D1FFE74A
:109C2000FFE70020039043F63000C4F20200016811
:109C300041F008010160006800F0080003900398FB
:109C4000FFE74FF480400490022005900121069127
:109C500003210791089040F60040C4F2020004A9D5
:109C6000FDF7B2FA56E00998006840F60041C4F2E8
:109C70000001884222D1FFE7FFE70020029043F66F
:109C80003000C4F20200016841F080010160006808
:109C900000F0800002900298FFE74FF4E05004903B
:109CA00002200590012106910790089041F600409E
:109CB000C4F2020004A9FDF787FA2AE009980068B7
:109CC00044F20041C4F20101884221D1FFE7FFE7DD
:109CD0000020019043F63000C4F20200016841F018
:109CE00020010160006800F0200001900198FFE76A
:109CF00040200490022005900690079003200890D1
:109D000041F20040C4F2020004A9FDF75DFAFFE74A
:109D1000FFE7FFE70AB080BD80B586B004900391ED
:109D2000029200208DF80700FFE7049890F83C00AD
:109D3000012804D1FFE702208DF8170089E004997B
:109D4000012081F83C00FFE7FFE7029800900C2813
:109D500000F270800099DFE801F0076D6D6D206DF5
:109D60006D6D3A6D6D6D530004980068039904F0B1
:109D7000CDFC04980168886940F008008861049867
:109D80000168886920F004008861039802690498DA
:109D9000016888691043886150E00498006803995D
:109DA00004F02AFD04980168886940F40060886125
:109DB00004980168886920F48060886103980269CA
:109DC00004980168886940EA0220886136E00498B6
:109DD0000068039904F08AFD04980168C86940F09E
:109DE0000800C86104980168C86920F00400C861CF
:109DF0000398026904980168C8691043C8611DE0AE
:109E000004980068039904F0EBFD04980168C869A0
:109E100040F40060C86104980168C86920F480605B
:109E2000C8610398026904980168C86940EA022081
:109E3000C86103E001208DF80700FFE7FFE7049900
:109E4000002081F83C00FFE79DF807008DF817001F
:109E5000FFE79DF8170006B080BD000080B582B016
:109E60000090009820B9FFE701208DF807003FE03F
:109E7000009890F83D0040B9FFE70099002081F874
:109E80003C00009800F038F8FFE70099022081F8C4
:109E90003D00009951F8040B04F01AFB00990120D1
:109EA00081F84600FFE70099012081F83E00009903
:109EB00081F83F00009981F84000009981F8410045
:109EC000FFE7FFE70099012081F84200009981F83F
:109ED0004300009981F84400009981F84500FFE7AC
:109EE0000099012081F83D0000208DF80700FFE770
:109EF0009DF8070002B080BD82B001900198006813
:109F000040F60001C4F20001884212D1FFE7FFE7EA
:109F10000020009043F64000C4F20200016841F0C6
:109F200004010160006800F0040000900098FFE761
:109F3000FFE702B07047000080B58CB00A9009912D
:109F4000099828B9FFE70A9890F83E0007901CE0AE
:109F50000998042805D1FFE70A9890F83F00069079
:109F600010E00998082805D1FFE70A9890F840000A
:109F7000059004E00A9890F841000590FFE70598E5
:109F80000690FFE706980790FFE70798012804D09E
:109F9000FFE701208DF82F00AFE0099828B9FFE70F
:109FA0000A99022081F83E001EE00998042806D193
:109FB000FFE70A99022081F83F00049012E0099817
:109FC000082806D1FFE70A99022081F84000039093
:109FD00005E00A99022081F841000390FFE7039809
:109FE0000490FFE70498FFE70A98006809990122A6
:109FF000019204F03FFB01980A9909680022C4F21B
:10A000000102914202900CD0FFE70A9800684FF6D7
:10A010000041CBF6FE710844B0FA80F0400902908E
:10A02000FFE70298C00738B1FFE70A980168486C5B
:10A0300040F400404864FFE70A9800680021C4F239
:10A04000010188423CD0FFE70A980068B0F1804FD8
:10A0500036D0FFE70A98006840F20041C4F20001E0
:10A0600088422DD0FFE70A98006840F60001C4F24C
:10A070000001884224D0FFE70A98006840F60041BA
:10A08000C4F2000188421BD0FFE70A98006840F242
:10A090000041C4F20101884212D0FFE70A9800682B
:10A0A00044F20001C4F20101884209D0FFE70A9896
:10A0B000006841F60001C4F20001884212D1FFE7B6
:10A0C0000A980068806800F0070008900898062841
:10A0D00007D0FFE70A980168086840F001000860AF
:10A0E000FFE706E00A980168086840F00100086090
:10A0F000FFE700208DF82F00FFE79DF82F000CB040
:10A1000080BD000080B586B0059004910598006878
:10A110000499002204F0AEFA05980168012000229B
:10A12000C4F20102914203900CD0FFE70598006849
:10A130004FF60041CBF6FE710844B0FA80F04009BA
:10A140000390FFE70398C007D8B1FFE7FFE7059842
:10A150000068006A41F21111084210D1FFE705982A
:10A160000068006A40F24441084207D1FFE70598C1
:10A170000168486C20F400404864FFE7FFE7FFE710
:10A18000FFE7FFE705980068006A41F211110842F5
:10A1900010D1FFE705980068006A40F24441084288
:10A1A00007D1FFE705980168086820F00100086002
:10A1B000FFE7FFE7FFE7049828B9FFE705990120CB
:10A1C00081F83E001EE00498042806D1FFE70599B7
:10A1D000012081F83F00029012E00498082806D17F
:10A1E000FFE70599012081F84000019005E00599FD
:10A1F000012081F841000190FFE701980290FFE7FC
:10A200000298FFE7002006B080BD000082B00190F8
:10A21000ADF8021002B0704780B582B0019001988D
:10A2200005F068FA8DF803009DF8030003281BD0A1
:10A23000FFE79DF8030000EBC00140F28850C2F236
:10A24000000000EB8100006968B1FFE79DF80300A2
:10A2500000EBC00140F28850C2F2000000EB810028
:10A2600000698047FFE7FFE702B080BD80B592B08C
:10A270001190119800680068109011980068C068EB
:10A280000F901198006840690E9000200D900C907E
:10A29000109800F00F000D900D9888B9FFE79DF819
:10A2A0004000800600280AD5FFE79DF83C008006A4
:10A2B000002804D5FFE7119805F040FA02E2FFE715
:10A2C0000D98002800F0C280FFE79DF83800C00715
:10A2D00038B9FFE7BDF83C0010F4907F00F0B6807D
:10A2E000FFE79DF84000C00758B1FFE79DF83D002B
:10A2F000C00730B1FFE71199486C40F00100486495
:10A30000FFE79DF84000400700280BD5FFE79DF8C8
:10A310003800C00730B1FFE71199486C40F00200E7
:10A320004864FFE79DF84000800700280BD5FFE751
:10A330009DF83800C00730B1FFE71199486C40F034
:10A3400004004864FFE79DF840000007002811D58D
:10A35000FFE79DF83C008006002805D4FFE79DF844
:10A360003800C00730B1FFE71199486C40F0080091
:10A370004864FFE71198406C002866D0FFE79DF81D
:10A380004000800600280AD5FFE79DF83C008006C3
:10A39000002804D5FFE7119805F0D0F9FFE71198E0
:10A3A00000684069C0F380100C901198406C000761
:10A3B000002804D4FFE70C9800283ED0FFE711984E
:10A3C00005F01EF9119800684069400600282FD555
:10A3D000FFE7FFE7FFE71198006850E8050F20F05E
:10A3E00040000B90FFE70B991198026842E80510B6
:10A3F0000028F0D1FFE7FFE71198C06B98B1FFE7A5
:10A400001198C16B4FF24140C0F6000008651198E9
:10A41000C06BFCF79BFB28B1FFE71198C06B016D87
:10A420008847FFE703E01198FFF7F6FEFFE703E038
:10A430001198FFF7F1FEFFE706E01198FFF7ECFE39
:10A44000119900204864FFE7FFE73BE11198006B9A
:10A45000012840F01781FFE79DF84000C006002862
:10A4600040F11081FFE79DF83C00C006002840F154
:10A470000981FFE7FFE700200A9011980068006853
:10A480000A901198006840680A900A98FFE71198AE
:10A49000006840694006002840F19A80FFE7119863
:10A4A000C06B00684068ADF82600BDF826000028A3
:10A4B00075D0FFE7BDF826001199898D88426EDAC4
:10A4C000FFE7BDF826001199C8851198C06BC069D7
:10A4D000B0F5807F58D0FFE7FFE7FFE711980068ED
:10A4E00050E8030F20F480700890FFE70899119856
:10A4F000026842E803100028F0D1FFE7FFE7FFE71A
:10A50000FFE71198006850E8050F20F00100079060
:10A51000FFE707991198026842E805100028F0D17A
:10A52000FFE7FFE7FFE7FFE71198006850E8050F36
:10A5300020F040000690FFE706991198026842E873
:10A5400005100028F0D1FFE7FFE71199202081F8DE
:10A550004200119900200863FFE7FFE711980068A7
:10A5600050E8030F20F010000590FFE705991198BF
:10A57000026842E803100028F0D1FFE7FFE71198D6
:10A58000C06BFCF76DFAFFE7119902204863119840
:10A59000818DC28D891A89B2FFF738FE17E0BDF8A8
:10A5A00026001199898D884210D1FFE71198C06B60
:10A5B000C069B0F5807F08D1FFE711990220486398
:10A5C0001198818DFFF722FEFFE7FFE7FFE779E0B3
:10A5D0001199888DC98D401AADF812001198C08D5F
:10A5E00000284ED0FFE7BDF81200002849D0FFE751
:10A5F000FFE7FFE71198006850E8030F20F4907020
:10A600000390FFE703991198026842E803100028BD
:10A61000F0D1FFE7FFE7FFE7FFE71198006850E898
:10A62000050F20F001000290FFE7029911980268DF
:10A6300042E805100028F0D1FFE7FFE7119920203C
:10A6400081F84200119900200863FFE7FFE71198A5
:10A65000006850E8030F20F010000190FFE7019917
:10A660001198026842E803100028F0D1FFE7FFE7E5
:10A670001199022048631198BDF81210FFF7C6FD2A
:10A68000FFE71FE09DF84000000600280AD5FFE71D
:10A690009DF83C000006002804D5FFE7119805F05E
:10A6A00037FA0FE09DF84000400600280AD5FFE782
:10A6B0009DF83C004006002804D5FFE7119804F0FF
:10A6C000E9FFFFE712B080BD80B582B0009000982E
:10A6D00020B9FFE701208DF8070040E0009880696D
:10A6E00008B1FFE700E0FFE7009890F8410040B9AB
:10A6F000FFE70099002081F84000009800F034F84E
:10A70000FFE70099242081F8410000980168C8689B
:10A7100020F40050C860009805F0C4F80098016863
:10A72000086920F49040086100980168486920F0A9
:10A730002A00486100980168C86840F40050C86069
:10A74000009900204864009A202182F84110009A64
:10A7500082F84210009948638DF80700FFE79DF8E2
:10A76000070002B080BD000080B590B00F900020BF
:10A770000E900D900C900B900A900F98006844F684
:10A780000001C4F2000188425FD1FFE7FFE700202B
:10A79000099043F64000C4F20200016841F48021B0
:10A7A0000160006800F4802009900998FFE7FFE746
:10A7B0000020089043F63000C4F20200016841F026
:10A7C00004010160006800F0040008900898FFE7A9
:10A7D0004FF440600A9002200B90002004900C90EF
:10A7E00003200D9007200E9040F60000C4F20200F6
:10A7F0000AA9FCF7E9FC049940F6D450C2F2000023
:10A80000059046F22802C4F2020202604FF0006294
:10A8100042608160C1604FF4806202614161816188
:10A82000C16101624162FCF743FB18B1FFE7FAF72F
:10A8300063FCFFE7FFE70F9840F6D451C2F2000136
:10A84000C1630F988863FFE79CE00F98006841F2AE
:10A850000041C4F20101884240F09380FFE7FFE726
:10A860000020079043F64400C4F20200016841F062
:10A8700020010160006800F0200007900798FFE7C2
:10A88000FFE70020069043F63000C4F202000168A2
:10A8900041F040010160006800F040000690069819
:10A8A000FFE74FF484400A9002200B9000200290B2
:10A8B0000C9003200D9008200E9041F60000C4F289
:10A8C00002000AA9FCF780FC029940F63460C2F24B
:10A8D0000000039046F22842C4F2020202604FF0E8
:10A8E000206242608160C1604FF480620261416118
:10A8F0008161C16101624162FCF7DAFA18B1FFE7D8
:10A90000FAF7FAFBFFE7FFE70F9840F63461C2F26F
:10A910000001C1630F988863FFE740F69460C2F2BC
:10A920000000019046F2A041C4F2020101604FF024
:10A9300020614160402181600021C1604FF480624C
:10A94000026141618161C16101624162FCF7B0FA5B
:10A9500018B1FFE7FAF7D0FBFFE7FFE70F9840F6E3
:10A960009461C2F2000181630F988863FFE747207A
:10A97000009005210022FDF7CBF80098FDF7BEF806
:10A98000FFE7FFE710B080BD80B584B00290019171
:10A99000ADF80220029890F84200202817D1FFE776
:10A9A000019820B1FFE7BDF8020020B9FFE70120C0
:10A9B0008DF80F000FE002990020086302980199BA
:10A9C000BDF8022005F00CF88DF80F0003E002201E
:10A9D0008DF80F00FFE79DF80F0004B080BD000068
:10A9E00080B582B00190019804F084FE8DF80300D8
:10A9F0009DF8030003281BD0FFE79DF8030000EB40
:10AA0000C00140F28850C2F2000000EB8100C06833
:10AA100068B1FFE79DF8030000EBC00140F28850E9
:10AA2000C2F2000000EB8100C0688047FFE7FFE74B
:10AA300002B080BD80B582B00190019804F05AFE4A
:10AA40008DF803009DF8030003281BD0FFE79DF855
:10AA5000030000EBC00140F28850C2F2000000EB9E
:10AA60008100806868B1FFE79DF8030000EBC0013A
:10AA700040F28850C2F2000000EB810080688047FD
:10AA8000FFE7FFE702B080BD80B582B0019001987A
:10AA900004F030FE8DF803009DF8030003281BD05E
:10AAA000FFE79DF8030000EBC00140F28850C2F2BE
:10AAB000000000EB8100406868B1FFE79DF80300EB
:10AAC00000EBC00140F28850C2F2000000EB8100B0
:10AAD00040688047FFE7FFE702B080BDFFE7FEE781
:10AAE00084B08DED030A9DED030AB6EE001A20EE48
:10AAF000010A8DED020A03980190019800900099D7
:10AB000045F6DF10C5F63770A0EB610000900098A5
:10AB100001909DED010A9DED021A21EE001A21EE31
:10AB2000002AB7EE081A31EE422A20EE020A8DED15
:10AB3000010A9DED010A9DED022A22EE002A22EE75
:10AB4000002A31EE421A20EE010A8DED010A9DED38
:10AB5000010A04B07047000080B586B004908DED06
:10AB6000030A049818B9FFE7002005904CE09DED1A
:10AB7000030A049890ED014A90ED022A90ED063AFE
:10AB800090ED071A23EE043A30EE430A21EE021A42
:10AB900030EE410A8DED020A002028B9FFE7029845
:10ABA00005F07EF858B90DE002980BF0E9F841EC99
:10ABB000100B51EC100B05F059F818B1FFE7039892
:10ABC0000290FFE79DED020A049890ED034A90ED94
:10ABD000043A90ED052A90ED061A20EE040A21EEC3
:10ABE000031A30EE010A90ED071A21EE021A30EE38
:10ABF000010A8DED010A04998869C86102980499D7
:10AC0000886101980590FFE79DED050A06B080BDBB
:10AC100080B588B007908DED060ACDED050A07983E
:10AC200008B9FFE78BE005980799086007990020AD
:10AC300088610799C861079890ED000AB5EE400A4F
:10AC4000F1EE10FA0EDCFFE707994FF07E50C86076
:10AC5000079900200861079948610799486007999A
:10AC600088606CE09DED060A079890ED001A80EE72
:10AC7000010A8DED040A9DED041A9FED320A80EE63
:10AC8000010A0AF06BF98DED030A9FED2F0A8DED95
:10AC9000000A09F0F3FFB0EE401A9DED000A31EE14
:10ACA000011A9DED033A21EE031AB7EE002A8DED4D
:10ACB000012A31EE021A23EE033A31EE031A8DED2A
:10ACC000021A9DED031A21EE011A9DED023A81EE62
:10ACD000031A079880ED031A079890ED031A31EED6
:10ACE000011A80ED041A0799C86848619DED031A9E
:10ACF00021EE011A31EE421A31EE011A9DED022ABF
:10AD000081EE021A079880ED011A09F0B7FFB0EE44
:10AD1000401A9DED010A31EE012A9DED031A22EE43
:10AD2000012A30EE420A21EE011A30EE010A9DEDB1
:10AD3000021A80EE010A079880ED020AFFE708B0C8
:10AD400080BD00BFDB0F4940DB0F493F80B584B0B9
:10AD500002908DED010A029818B9FFE700200390D8
:10AD600039E09DED010A029890ED031A90ED043A46
:10AD700090ED052A31EE031A31EE021A80EE010A37
:10AD80008DED000A002028B9FFE7009804F04AFF83
:10AD900058B911E000980AF0F3FF41EC100B51ECA8
:10ADA000100B04F00FFF38B1FFE70098029988619B
:10ADB00000980299C86106E001980299886101989B
:10ADC0000299C861FFE702989DED010AFFF7C4FEF2
:10ADD0008DED030AFFE79DED030A04B080BD00007E
:10ADE00080B582B08DF806009DF80600022804DBCD
:10ADF000FFE7FF208DF8070039E09DF8061040F2CC
:10AE00002460C2F2000050F8210020B1FFE70020CA
:10AE10008DF807002BE08820F8F7B4F801469DF87C
:10AE2000062040F22460C2F2000040F822109DF893
:10AE3000061050F8210020B9FFE7FF208DF8070029
:10AE400015E09DF8061040F22460C2F20000009068
:10AE500050F821008821F5F758FB00999DF806006D
:10AE600051F82010087000208DF80700FFE79DF9C9
:10AE7000070002B080BD000080B588B0069006983B
:10AE800020B9FFE7FE208DF81F002EE0069800F0A5
:10AE900049F80590059820B9FFE7FC208DF81F00C0
:10AEA00023E005988088019008208DF80800FF2095
:10AEB0008DF809008DF80A008DF80B008DF80C0054
:10AEC0008DF80D008DF80E008DF80F00FC208DF828
:10AED00010000598007801A9F7F708FE002818BFB0
:10AEE0004FF0FF308DF81F00FFE79DF91F0008B0FD
:10AEF00080BD000082B08DF803009DF80300022899
:10AF000003DBFFE70020019009E09DF8031040F209
:10AF10002460C2F2000050F821000190FFE7019880
:10AF200002B0704780B586B00490049818B9FFE766
:10AF30000020059036E004980078FFF7DBFF0390CF
:10AF4000039818B9FFE7002005902BE0002002903D
:10AF5000FFE70298039991F8841088421FDAFFE70F
:10AF60000398029900EB810040680190019888B134
:10AF7000FFE7019800780499097888420AD1FFE731
:10AF80000198408804994988884203D1FFE70198D5
:10AF9000059007E0FFE7029801300290D9E7002012
:10AFA0000590FFE7059806B080BD000080B584B02D
:10AFB00002900191029818B1FFE7019820B9FFE7CC
:10AFC000FE208DF80F0011E00298FFF7ABFF009014
:10AFD000009820B9FFE7FC208DF80F0006E00098EC
:10AFE000019900F049F98DF80F00FFE79DF90F0076
:10AFF00004B080BD80B586B004900391049818B168
:10B00000FFE7039820B9FFE7FE208DF8170090E0D6
:10B0100003984178807840EA0120ADF80A00BDF835
:10B020000A009FED460ADFED460A102106F02AFECF
:10B03000049880ED070A0399C8780979000140EA6D
:10B040001110ADF80800BDF80800BBEE0E0AF3EED3
:10B050000E0A0C21009106F015FE0099049880ED6F
:10B06000080A03980279407902F00F0240EA0220B0
:10B07000ADF80600BDF80600BAEE080AF2EE080ABE
:10B0800006F000FE049880ED090A0398807900EE2E
:10B09000100AB8EE400A049880ED0A0AFFE7049807
:10B0A00090ED070AB5EE400AF1EE10FA0ADAFFE772
:10B0B000049890ED070A9FED231A30EE010A80ED07
:10B0C000070AECE7FFE7049890ED070A9FED1D1AC9
:10B0D000B4EE410AF1EE10FA0ADBFFE7049890EDB6
:10B0E000070A9FED191A30EE010A80ED070AEAE718
:10B0F0000498C079C007C0B1FFE7049890ED071A23
:10B100009FED100A30EE410A80ED070A049890ED99
:10B11000080AB1EE400A80ED080A049890ED090A89
:10B12000B1EE400A80ED090AFFE700208DF8170014
:10B13000FFE79DF9170006B080BD00BFDA0F49C1D7
:10B14000DA0F4941DB0FC940DB0FC9C080B586B0BB
:10B150000490049820B9FFE7FE208DF8170087E0DF
:10B1600004980078FFF73CFE20B1FFE7FF208DF840
:10B1700017007DE004980078FFF7BCFE0390039869
:10B1800020B9FFE7FF208DF8170071E00020029042
:10B19000FFE70298039991F8841088421BDAFFE7D1
:10B1A0000398029900EB8100406878B1FFE70398AB
:10B1B000029900EB810040684088049949888842E0
:10B1C00004D1FFE7FD208DF8170051E0FFE702985A
:10B1D00001300290DDE7039890F88400202804DB1A
:10B1E000FFE7FF208DF8170042E03020F7F7CAFE96
:10B1F0000190019820B9FFE7FF208DF8170037E094
:10B2000001983021F5F781F90199049A1068526884
:10B210004A6008600199002008720498C079019979
:10B2200000F00100087604984088ADF80200049808
:10B230000078BDF802100322F7F796FA38B1FFE75D
:10B240000198F7F7A9FDFF208DF8170010E001988D
:10B25000039991F8842001EB82014860039991F8E9
:10B260008400013081F8840000208DF81700FFE78A
:10B270009DF9170006B080BD80B58EB00C900B9183
:10B280000C9818B1FFE70B9820B9FFE7FE208DF866
:10B29000370087E00C988088ADF818000B9890ED87
:10B2A000020ADFED420A9FED421A102004F03EFE32
:10B2B000ADF822000B9890ED010AFBEE0E0AB3EEFA
:10B2C0000E1A0C20019004F031FE01460198ADF8F1
:10B2D00020100B9991ED030ADFED360ACDED000A3F
:10B2E0009FED351A04F022FEDDED000A01460198BB
:10B2F000ADF81E100B9991ED040AB1EE041A04F09A
:10B3000015FE01460198ADF81C100B9991ED000A4D
:10B31000FAEE080AB2EE081A04F008FEADF81A00B8
:10B320009DF823008DF824009DF822008DF825005B
:10B33000BDF8200000098DF82600BDF820109DF80A
:10B340001F0040EA01108DF827009DF81E008DF8BF
:10B350002800BDF81C0000098DF82900BDF81C105C
:10B360009DF81B0040EA01108DF82A009DF81A0094
:10B370008DF82B000C988088029008208DF80C0026
:10B3800009980A99CDF81110CDF80D000C980078A5
:10B3900002A9F7F7ABFB002818BF4FF0FF308DF87C
:10B3A0003700FFE79DF937000EB080BDDA0F49C1C5
:10B3B000DA0F4941000000000000FA4380B590B068
:10B3C0000E900E9820B9FFE7FE208DF83F0077E041
:10B3D0000E980078FFF78EFD0D900D9820B9FFE7CD
:10B3E000FC208DF83F006BE000200C900B90FFE7F5
:10B3F0000B980D9991F8841088421EDAFFE70D989A
:10B400000B9900EB8100406890B1FFE70D980B9914
:10B4100000EB8100406840880E994988884207D136
:10B42000FFE70D980B9900EB810040680C9004E059
:10B43000FFE70B9801300B90DAE70C9820B9FFE793
:10B44000FC208DF83F003BE00E984088ADF82A00C4
:10B450000E980078BDF82A1003AA0023F7F716F813
:10B46000E0B1FFE7F7F778FF0191009000990198AC
:10B470000C9A13695269C91A904148F2A162C0F24C
:10B480000102891A70F1000004D3FFE70C99002033
:10B490000872FFE7FF208DF83F0011E00C990120B2
:10B4A0000872F7F759FF0A460C994A6108610C982F
:10B4B00003A90D31FFF79EFD00208DF83F00FFE747
:10B4C0009DF93F0010B080BD80B582B08DF80600B8
:10B4D0009DF80600022804DBFFE7FF208DF8070037
:10B4E00039E09DF8061040F22C60C2F2000050F8DE
:10B4F000210020B1FFE700208DF807002BE0482055
:10B50000F7F740FD01469DF8062040F22C60C2F29C
:10B51000000040F822109DF8061050F8210020B9D4
:10B52000FFE7FF208DF8070015E09DF8061040F2B8
:10B530002C60C2F20000009050F821004821F4F77E
:10B54000E4FF00999DF8060051F8201008700020D3
:10B550008DF80700FFE79DF9070002B080BD0000ED
:10B5600080B58EB00C900C9820B9FFE7FE208DF8C6
:10B570003700A9E00C98007800F0AAF80B900B981F
:10B5800020B9FFE7FC208DF837009DE00B980230D2
:10B590000A900C984088ADF81600BDF81610A1F27C
:10B5A0000120019104280CD3FFE70198A0F20520A7
:10B5B000042829D3FFE70198A0F20920032849D3E2
:10B5C00072E04FF40070069008208DF81C000020F7
:10B5D0000490FFE70498032815DCFFE70A98049A13
:10B5E00000EB4200407806A9053101F812000A98E4
:10B5F000049A30F8120001EB42014870FFE704980A
:10B6000001300490E6E753E040F2FF100690082076
:10B610008DF81C0004200390FFE70398072818DC2E
:10B62000FFE70A98039A00EB4200407806A905312B
:10B6300001EB420202F8080C0A98039A30F8120053
:10B6400001EB420101F8070CFFE70398013003907A
:10B65000E3E72DE040F2FF20069008208DF81C0063
:10B660000290FFE702980A2818DCFFE70A98029A7E
:10B6700000EB4200407806A9053101EB420202F8D6
:10B68000100C0A98029A30F8120001EB420101F8FE
:10B690000F0CFFE7029801300290E3E700208DF8DD
:10B6A00023008DF8240003E0FF208DF837000BE025
:10B6B0000C98007806A9F7F719FA002818BF4FF080
:10B6C000FF308DF83700FFE79DF937000EB080BDE1
:10B6D00082B08DF803009DF80300022803DBFFE72A
:10B6E0000020019009E09DF8031040F22C60C2F2A6
:10B6F000000050F821000190FFE7019802B0704768
:10B7000082B08DF805009DF805000146009140B11A
:10B71000FFE70098012809D0FFE7009802280AD027
:10B720000EE042F21070ADF806000EE04FF48040DB
:10B73000ADF8060009E047F23050ADF8060004E02D
:10B740004FF6FF70ADF80600FFE7BDF9060002B046
:10B750007047000083B0ADF808008DF807109DF821
:10B76000070001460091022804D3FFE70098022851
:10B7700013D026E0BDF80800B0F5007F0CDDFFE730
:10B78000BDF80800B0F5027F06DAFFE7BDF8080053
:10B7900001388DF80B0019E014E0BDF80800B0F591
:10B7A000017F0DDDFFE7BDF8080040F20A21884265
:10B7B00006DCFFE7BDF8080001388DF80B0005E056
:10B7C00000E0FFE7FF208DF80B00FFE79DF90B007D
:10B7D00003B0704780B586B00490049818B9FFE7AD
:10B7E000002005902FE004980078FFF771FF039088
:10B7F000039818B9FFE70020059024E0002002908C
:10B80000FFE70298039991F84410884218DAFFE79D
:10B810000398029900EB810080690190019850B172
:10B82000FFE70198408804994988884203D1FFE7DF
:10B830000198059007E0FFE7029801300290E0E7E9
:10B8400000200590FFE7059806B080BD83B08DF815
:10B8500007009DF807000146009140B1FFE70098FE
:10B86000012809D0FFE7009802280BD00EE0002045
:10B87000C4F2102002900DE04AF22C00C4F299109C
:10B88000029007E04FF07E50029003E04FF07E50B0
:10B890000290FFE79DED020A03B0704780B586B0C5
:10B8A0000490049820B9FFE7FE208DF8170081E08E
:10B8B00004980078FFF708FE20B1FFE7FF208DF81D
:10B8C000170077E004980078FFF702FF03900398D1
:10B8D00020B9FFE7FF208DF817006BE000200290F1
:10B8E000FFE70298039991F8441088421BDAFFE7BA
:10B8F0000398029900EB8100806978B1FFE7039813
:10B90000029900EB81008069408804994988884247
:10B9100004D1FFE7FD208DF817004BE0FFE7029808
:10B9200001300290DDE7039890F844000B2804DB17
:10B93000FFE7FF208DF817003CE05020F7F722FBCF
:10B940000190019820B9FFE7FF208DF8170031E042
:10B950000199049A106852684A600860019818308A
:10B960002821F4F7D2FD04984079019900F00100F4
:10B9700081F828000499087849880322F6F7F4FE34
:10B9800038B1FFE70198F7F707FAFF208DF81700A5
:10B9900010E00198039991F8442001EB820188613D
:10B9A000039991F84400013081F8440000208DF89B
:10B9B0001700FFE79DF9170006B080BD80B582B083
:10B9C000019001989FED020A00F004F802B080BDDA
:10B9D0000000000080B58AB007A9019101460198D6
:10B9E000089180ED000A089820B9FFE7FE208DF845
:10B9F000270078E008980078FFF76AFE069006981E
:10BA000020B9FFE7FC208DF827006CE0019890ED4D
:10BA1000000AB7EE001AB4EE410AF1EE10FA04DDA6
:10BA2000FFE74FF07E500790FFE7019890ED000A86
:10BA3000BFEE001AB4EE410AF1EE10FA05DAFFE7A4
:10BA40000020CBF680700790FFE708984079C00788
:10BA500040B1FFE7019890ED000AB1EE400A80ED99
:10BA6000000AFFE70898FFF7B5FE0590059820B992
:10BA7000FFE7FC208DF8270035E008994888097910
:10BA8000FFF768FE8DF813009DF91300B0F1FF3F3A
:10BA900004DCFFE7FF208DF8270024E001980699D9
:10BAA0000231039190ED000A8DED000A08980079AB
:10BAB000FFF726FE9DED000A01EE100AB8EEC11A4E
:10BAC00020EE010ABDEEC00A10EE100AADF80A0021
:10BAD000BDF80A0003999DF9132021F812000020F7
:10BAE0008DF82700FFE79DF927000AB080BD000010
:10BAF00080B590B00E900E9820B9FFE7FE208DF82B
:10BB00003F0072E00E980078FFF7E2FD0D900D986F
:10BB100020B9FFE7FC208DF83F0066E000200C9084
:10BB2000FFE70C980D9991F84410884259DAFFE725
:10BB30000D980C9900EB810080690B900B98002800
:10BB40004AD0FFE70B9840880E994988884243D134
:10BB5000FFE70E990878498804AA0023F6F796FCB7
:10BB6000E8B1FFE7F7F7F8FB039102900299039819
:10BB70000B9A136A526AC91A904140F2E932891A43
:10BB800070F1000007D3FFE70B9900200876FC2036
:10BB90008DF83F0029E0FF208DF83F0025E00B994C
:10BBA00001200876F7F7D8FB0A460B994A6208622B
:10BBB0000B9804A900F008FD0B9901918868CA68E8
:10BBC0000B69D1F814C0C1F838C04B630A63C8626E
:10BBD00000208DF83F0008E0FFE70C9801300C9042
:10BBE0009FE7FC208DF83F00FFE79DF93F0010B074
:10BBF00080BD000080B582B040F66440C2F2000013
:10BC0000019046F20041C4F200010160032141604D
:10BC100000218160C1604FF4102202614FF40012D4
:10BC200042610176417681760122C27601774177C1
:10BC3000FAF71AFB18B1FFE7F9F75EFAFFE702B06F
:10BC400080BD000080B582B040F68C40C2F200009A
:10BC5000019046F60001C4F2000101600321416039
:10BC600000218160C1604FF4102202614FF4001284
:10BC700042610176417681760122C2760177417771
:10BC8000FAF7F2FA18B1FFE7F9F736FAFFE702B070
:10BC900080BD000080B58AB0FFE70020099043F620
:10BCA0003000C4F20200016841F400110160006834
:10BCB00000F4001009900998FFE7FFE700200890C2
:10BCC00043F63000C4F20200016841F480010160D3
:10BCD000006800F4800008900898FFE70C200090AE
:10BCE0000521059100220692FBF712FF0098FBF751
:10BCF00005FF0599069A0D200190FBF709FF0198B1
:10BD0000FBF7FCFE0599069A39200290FBF700FF2D
:10BD10000298FBF7F3FE0599069A3A200390FBF789
:10BD2000F7FE0398FBF7EAFE0599069A3B2004907C
:10BD3000FBF7EEFE0498FBF7E1FE0599069A452015
:10BD40000790FBF7E5FE0798FBF7D8FE0AB080BD29
:10BD500080B582B04EF28130C0F6000046F2581233
:10BD6000C0F601020021019104F0DAFD019940F6CC
:10BD7000A012C2F2000210604EF62930C0F6000098
:10BD800046F20012C0F6010204F0CAFD02B080BD06
:10BD900080B59AB0002019901890179016901590C1
:10BDA000FFE70020149043F63000C4F2020001685F
:10BDB00041F002010160006800F002001490149844
:10BDC000FFE7FFE70020139043F63000C4F20200C3
:10BDD000016841F040010160006800F040001390EC
:10BDE0001398FFE7FFE70020129043F63000C4F2FB
:10BDF0000200016841F001010160006800F00100EB
:10BE000012901298FFE7FFE70020119043F63000F0
:10BE1000C4F20200016841F008010160006800F00E
:10BE2000080011901198FFE7FFE70020109043F6FB
:10BE30003000C4F20200016841F0040101600068B2
:10BE400000F0040010901098FFE7FFE700200F902B
:10BE500043F63000C4F20200016841F08001016045
:10BE6000006800F080000F900F98FFE7FFE70020C8
:10BE70000E9043F63000C4F20200016841F0200148
:10BE80000160006800F020000E900E98FFE741F678
:10BE90000000C4F2020001904021009100220C92A7
:10BEA000FBF786FB0020C4F20200039010210291F0
:10BEB00001220592FBF77CFB059A40F20040C4F298
:10BEC000020006901146FBF773FB009A0198059952
:10BED000159216911791189115A90791FBF774F90E
:10BEE0000198059A0799082315934FF404130493B6
:10BEF00016931792FBF768F90398049B059A079924
:10BF0000159216931792FBF75FF9029B0398059A17
:10BF100007991593169217921892FBF755F9049A00
:10BF200005980799302315931692179040F6000054
:10BF3000C4F20200FBF748F9059A06980799159292
:10BF4000169217921892FBF73FF90C9A0620089068
:10BF500005210B91FBF7DCFD0898FBF7CFFD0B9952
:10BF60000C9A09200990FBF7D3FD0998FBF7C6FD51
:10BF70000B990C9A0A200A90FBF7CAFD0A98FBF766
:10BF8000BDFD0B990C9A17200D90FBF7C1FD0D9884
:10BF9000FBF7B4FD1AB080BD80B582B040F6F46006
:10BFA000C2F20000019045F60041C4F200010160B8
:10BFB00041F68021C0F20601416000218160C1602C
:10BFC0004FF48042026141618161C1610162FBF70E
:10BFD0000DFB18B1FFE7F9F78FF8FFE702B080BD5E
:10BFE00080B582B040F64870C2F20000019043F282
:10BFF0000001C4F2010101604FF48271416000212F
:10C000008160C16002220261012242614FF400722C
:10C0100082611822C2610162416281620A21C162A9
:10C02000FCF7F2FA18B1FFE7F9F766F8FFE702B09C
:10C0300080BD000080B588B0002100910791069175
:10C040000591049103910291019140F6A070C2F212
:10C05000000044F20042C4F20102026041608160CB
:10C0600041F28732C26001618161FDF77BFC18B14A
:10C07000FFE7F9F741F8FFE740F6A070C2F20000D1
:10C08000FDF7ECFE18B1FFE7F9F736F8FFE760209F
:10C090000190002202920392059240F6A070C2F233
:10C0A000000001A9FDF738FE18B1FFE7F9F724F801
:10C0B000FFE740F6A070C2F20000FDF79FFD08B058
:10C0C00080BD000080B58AB00021009109910891DF
:10C0D000079106910591049103910291019140F617
:10C0E000E870C2F2000040F60002C4F200020260F2
:10C0F000416081604FF6FF72C26001618161FDF7AE
:10C10000ADFE18B1FFE7F8F7F7FFFFE70020089052
:10C11000099040F6E870C2F2000008A9FDF790FB14
:10C1200018B1FFE7F8F7E8FFFFE760200190002073
:10C1300002900390059040F6E870C2F2000001A959
:10C140000822FDF7E9FD18B1FFE7F8F7D5FFFFE793
:10C1500040F6E870C2F20000FDF750FD0AB080BD65
:10C1600080B58EB0002100910D910C910B910A9138
:10C17000099108910791069105910491039102910B
:10C18000019141F23000C2F2000040F60042C4F2D8
:10C1900000020260416081604FF6FF72C26001617F
:10C1A0008161FDF7DFFB18B1FFE7F8F7A5FFFFE7B7
:10C1B0004FF480500A9041F23000C2F200000AA908
:10C1C000FDF75AFC18B1FFE7F8F796FFFFE741F2D9
:10C1D0003000C2F20000FDF741FE18B1FFE7F8F7AA
:10C1E0008BFFFFE700200890099041F23000C2F277
:10C1F000000008A9FDF724FB18B1FFE7F8F77CFF62
:10C20000FFE760200190002202920392059241F222
:10C210003000C2F2000001A9FDF77EFD18B1FFE772
:10C22000F8F76AFFFFE741F23000C2F2000001A90F
:10C230000422FDF771FD18B1FFE7F8F75DFFFFE796
:10C2400041F23000C2F2000001A90822FDF764FDAE
:10C2500018B1FFE7F8F750FFFFE741F23000C2F2F4
:10C260000000FDF7CBFC0EB080BD000080B582B0B1
:10C2700041F27800C2F20000019044F60001C4F2DD
:10C280000001016048F2A061C0F20101416000219B
:10C290008160C16001610C2242618161C161FEF770
:10C2A00013FA18B1FFE7F8F727FFFFE702B080BDE8
:10C2B00080B582B041F2C000C2F20000019041F2AC
:10C2C0000041C4F2010101604FF4E13141600021FD
:10C2D0008160C16001610C2242618161C161FEF730
:10C2E000F3F918B1FFE7F8F707FFFFE702B080BDE9
:10C2F000FFE7FEE780B58DB00DF1100CCDF808C05A
:10C3000084460298CDF82CC00A9109928DF823300A
:10C3100080ED030A0B9820B9FFE7FF208DF833006A
:10C3200035E10B98007801460191052800F28980DB
:10C330000199DFE801F00345658585799DF92300C2
:10C3400004283BD1FFE70A9890ED000A90ED012AFE
:10C3500090ED021A30EE420A30EE010A099880EDA3
:10C36000000A0A9890ED000A90ED012A90ED021A59
:10C3700030EE020A30EE010A099880ED010A0A98AF
:10C3800090ED002A90ED011A90ED020A31EE421A6A
:10C3900030EE010A099880ED020A0A9890ED000A31
:10C3A00090ED012A90ED021AB1EE400A30EE420AF9
:10C3B00030EE010A099880ED030A00E0CBE040E08E
:10C3C0009DF92300042819D1FFE70A9890ED000A8F
:10C3D000B1EE400A099880ED000A0A9800680999B0
:10C3E00048600A980068099988600A9890ED000AE8
:10C3F000B1EE400A099880ED030A00E0ABE0FFE7E8
:10C400009DF9230002280DD1FFE70A9890ED000A5C
:10C41000B1EE400A099880ED000A0A98006809996F
:10C42000486000E097E0FFE79DF92300012805D16F
:10C43000FFE70A9800680999086000E08BE0FFE7D1
:10C4400089E0002006908DF81700FFE79DF917009E
:10C450009DF9231088422EDAFFE7029809999DF989
:10C46000172001EB820191ED000AB0EEC00A80EDC9
:10C47000000A90ED000A90ED021AB4EE410AF1EEC6
:10C4800010FA06DDFFE7029890ED000A8DED000A34
:10C4900005E0029890ED020A8DED000AFFE7029890
:10C4A0009DED000A80ED020AFFE79DF817000130BC
:10C4B0008DF81700CAE7029890ED020AB7EE001A4D
:10C4C000B4EE410AF1EE10FA21DDFFE700208DF80D
:10C4D0000F00FFE79DF90F009DF92310884215DA40
:10C4E000FFE7029890ED021A09989DF90F1000EBF2
:10C4F000810090ED000A80EE010A80ED000AFFE75E
:10C500009DF80F0001308DF80F00E3E7FFE70020F2
:10C510008DF80E00FFE79DF90E009DF9231088426B
:10C5200015DAFFE7029890ED031A09989DF90E10AD
:10C5300000EB810090ED000A20EE010A80ED000A78
:10C54000FFE79DF80E0001308DF80E00E3E70020B4
:10C550008DF833001BE000208DF80D00FFE79DF8FB
:10C560000D009DF9231088420DDAFFE709999DF827
:10C570000D20002041F82200FFE79DF80D0001305A
:10C580008DF80D00EBE7FF208DF83300FFE79DF9F4
:10C5900033000DB080BD000083B001908DF8031012
:10C5A000019820B9FFE7FF208DF80B0007E09DF808
:10C5B00003000199087000208DF80B00FFE79DF93A
:10C5C0000B0003B07047000080B58AB00990089155
:10C5D0000898417B807B40EA0120ADF81E00089856
:10C5E000C17B007C40EA0120ADF81C000898417C2A
:10C5F000807C40EA0120ADF81A0009980079FFF725
:10C600007FF8ADF8180009980079FFF71FF98DED54
:10C61000050ABDF81E0000EE100AB8EEC00A9FED34
:10C620006D1A80EE010A9FED6C1A20EE010A8DED65
:10C63000040ABDF91C0000EE100AB8EEC00A8DED28
:10C64000030ABDF91A00BDF91810484300EE100A9C
:10C65000B8EEC00A9FED611A80EE010A8DED020A64
:10C6600009988079C00700284CD0FFE7BDF81E006C
:10C670000999B1F84010401A01900198B0F5805F17
:10C6800005DDFFE70999486C013848640AE0019824
:10C6900010F5805F05DAFFE70999486C01304864BE
:10C6A000FFE7FFE7BDF81E000999A1F840000498D4
:10C6B0000090099890ED110AB8EEC00A9FED461A55
:10C6C00020EE010A9DED001A30EE010A9DED051ADB
:10C6D00080EE010A80ED120A0999886C88609DED50
:10C6E000030A9DED051A80EE010A099880ED030A00
:10C6F0009DED020A9DED051A20EE010A099880EDD4
:10C70000040A13E0099900204864BDF81E10099A34
:10C71000A2F84010099988640498099988600398E0
:10C720000999C860029809990861FFE7FFE709982D
:10C7300090ED020AB5EE400AF1EE10FA0ADAFFE7D0
:10C74000099890ED020A9FED241A30EE010A80ED5F
:10C75000020AECE7FFE7099890ED020A9FED1E1A26
:10C76000B4EE410AF1EE10FA0ADBFFE7099890ED0A
:10C77000020A9FED1B1A30EE010A80ED020AEAE779
:10C78000099890F82800C007C0B1FFE7099890ED1C
:10C79000021A9FED110A30EE410A80ED020A099853
:10C7A00090ED030AB1EE400A80ED030A099890ED7E
:10C7B000040AB1EE400A80ED040AFFE70898C07C45
:10C7C00000EE100AB8EE400A099880ED050A0AB09A
:10C7D00080BD00BF00000046DB0FC940000080465E
:10C7E000DB0FC9C0FFE7FEE788B00790069105920E
:10C7F000079800F0070004900498C0F1070005288E
:10C8000003D3FFE70420019004E00498C0F107007F
:10C810000190FFE70198039004980430062803D89C
:10C82000FFE70020009003E0049803380090FFE742
:10C830000098029006980399012202FA01F1013949
:10C840000840029B984005999A40013A11400843DC
:10C8500008B0704780B590B00E908DED0D0ACDED0B
:10C860000C0A8DED0B1ACDED0A1A002028B9FFE74E
:10C870000D9803F0E3F958B943E00D9809F080FAF8
:10C8800041EC100B51EC100B03F0ACF9C8B3FFE70F
:10C89000002028B9FFE70C9803F0D0F958B930E030
:10C8A0000C9809F06DFA41EC100B51EC100B03F0F1
:10C8B00099F930B3FFE7002028B9FFE70B9803F0A0
:10C8C000BDF958B91DE00B9809F05AFA41EC100B6C
:10C8D00051EC100B03F086F998B1FFE7002028B95E
:10C8E000FFE70A9803F0AAF978B90AE00A9809F074
:10C8F00047FA41EC100B51EC100B03F073F920B91F
:10C90000FFE70E9880690F9016E19DED0D0ADDEDB1
:10C910000C0A0E98406890ED071AF7F7AFFB8DED03
:10C92000090A9DED090A0E98406890ED001A20EE64
:10C93000010A8DED080A0E98406890ED000A9DED01
:10C940000C1A20EE010A8DED070A0E981C309DEDA1
:10C95000070AFEF701F98DED060A0E9800780146E8
:10C96000019110B3FFE70198012804D0FFE7019877
:10C97000022817D01CE09DED060A0E9890ED021AD1
:10C9800090ED052A30EE420A9DED0A2AB4EE412AC6
:10C99000F1EE10FAC8BFB0EE421A80EE010A8DED3A
:10C9A000050A05E00B98059002E000200590FFE7DE
:10C9B00009980E99086106980E994861002028B9D7
:10C9C000FFE7059803F03AF970B90AE0059809F015
:10C9D000D7F941EC100B51EC100B03F003F918B927
:10C9E000FFE700200590FFE79DED080A0E984068DC
:10C9F00090ED011A90ED032A20EE010A9DED051A33
:10CA000021EE021A30EE410A8DED040A0E9890EDE7
:10CA1000030A9DED081A9DED0A2A21EE021A30EE56
:10CA2000010A8DED030A9DED030A0E98406890ED12
:10CA3000021A20EE010A8DED020A0E98406890ED70
:10CA4000020A9FED3F1AB4EE410AF1EE10FA39DD09
:10CA5000FFE7002028B9FFE7039803F0EFF858B983
:10CA60002FE0039809F08CF941EC100B51EC100BFE
:10CA700003F0B8F828B3FFE79DED040A9DED021A14
:10CA800030EE010AB0EEC00A0E98406890ED051A2B
:10CA9000B4EE410AF1EE10FA12DCFFE79DED030A55
:10CAA000B0EEC00A0E98406890ED041AB4EE410A48
:10CAB000F1EE10FA04DCFFE703980E99C860FFE777
:10CAC000FFE7FFE79DED021A9DED040A30EE010A33
:10CAD0008DED040A002028B9FFE7049803F0AEF8B2
:10CAE00058B925E0049809F04BF941EC100B51ECD2
:10CAF000100B03F077F8D8B1FFE70E98406890ED7F
:10CB0000050A9FED0F1AB4EE410AF1EE10FA0BDDA3
:10CB1000FFE79DED040A0E984068D0ED050AF5F791
:10CB200053F88DED040AFFE704980E998861FFE73A
:10CB30000E9880690F90FFE79DED0F0A10B080BD41
:10CB4000BD37863580B586B004908DF80F108DED19
:10CB5000020A0192049820B9FFE7FF208DF8170020
:10CB6000B7E0002030B9FFE70198406803F066F8AD
:10CB700080B90BE00198406809F002F941EC100B14
:10CB800051EC100B03F02EF820B9FFE7FF208DF8D1
:10CB900017009EE0002030B9FFE70198806803F09D
:10CBA0004DF880B90BE00198806809F0E9F841EC94
:10CBB000100B51EC100B03F015F820B9FFE7FF2024
:10CBC0008DF8170085E0002030B9FFE70198C068B4
:10CBD00003F034F880B90BE00198C06809F0D0F890
:10CBE00041EC100B51EC100B02F0FCFF20B9FFE7F9
:10CBF000FF208DF817006CE0002030B9FFE70198A6
:10CC0000006903F01BF880B90BE00198006909F096
:10CC1000B7F841EC100B51EC100B02F0E3FF20B918
:10CC2000FFE7FF208DF8170053E0002030B9FFE741
:10CC30000198406903F002F880B90BE0019840695F
:10CC400009F09EF841EC100B51EC100B02F0CAFFFA
:10CC500020B9FFE7FF208DF817003AE0019804990A
:10CC600048609DED021AB7EE000A80EE010A8DEDD4
:10CC7000000A002028B9FFE7009802F0DFFF58B94A
:10CC80000EE0009809F07CF841EC100B51EC100B11
:10CC900002F0A8FF20B1FFE700980499886003E044
:10CCA000FF208DF8170014E0049901F11C009DEDA0
:10CCB000020A4968D1ED060AFDF7AAFF9DF80F00A8
:10CCC00004990870049800F009F800208DF8170006
:10CCD000FFE79DF9170006B080BD000080B584B065
:10CCE0000290029820B9FFE7FF208DF80F0013E0B3
:10CCF000029900200190C860029908610299486178
:10CD00000299886102981C309FED050AFEF71EF813
:10CD100001988DF80F00FFE79DF90F0004B080BD6A
:10CD20000000000082B00090009820B9FFE7FF20CB
:10CD30008DF8070005E000990020C8608DF8070015
:10CD4000FFE79DF9070002B07047000000000000F7
:10CD5000EFF30980BFF36F8F154B1A681EF0100FA9
:10CD600008BF20ED108A20E9F04F10602DE909007E
:10CD70004FF0500080F31188BFF34F8FBFF36F8FD8
:10CD800005F0B4FC4FF0000080F31188BDE8090005
:10CD900019680868B0E8F04F1EF0100F08BFB0EC3B
:10CDA000108A80F30988BFF36F8F704700BF00BF00
:10CDB0008012002080B582B001900198806B0090B5
:10CDC00000980168486820F0030048600099486DA9
:10CDD00040F0100048650099012081F8510000984A
:10CDE000FBF7E8FB02B080BD80B582B001900198EE
:10CDF000806B00900098FBF76BFF02B080BD0000D5
:10CE000080B582B001900198806B00900098FCF78B
:10CE100091FC02B080BD000080B582B00190019805
:10CE2000806B00900098FCF7D9FC02B080BD000038
:10CE300080B584B003900398806B0290FAF7D0FB22
:10CE4000019003980068006800F48070B0F5807F5E
:10CE500039D0FFE702980168486820F02000486058
:10CE60000298806868B9FFE702984068B0F5827F51
:10CE700007D1FFE702980168486820F00300486086
:10CE800006E002980168486820F001004860FFE76A
:10CE90000298019A642100F0B5F820B1FFE70299E9
:10CEA00020204865FFE702990020C88702990120E9
:10CEB00081F851000298406D20B1FFE70298FBF71E
:10CEC00079FB04E0FFE70298FBF7D8FEFFE704B028
:10CED00080BD000080B584B003900398806B029001
:10CEE000FAF77EFB019003980068006800F48070F8
:10CEF000B0F5807F3BD0FFE702980168486820F0DA
:10CF00002000486002980168486820F002004860EC
:10CF10000298019A642100F0E7F830B1FFE7029926
:10CF2000486D40F020004865FFE70298806870B9BE
:10CF3000FFE7FFE70020009002980068C0680090BB
:10CF400002980068806800900098FFE7FFE7029968
:10CF50000020C8860299012081F851000298406D96
:10CF600020B1FFE70298FBF725FB04E0FFE70298FA
:10CF7000FCF7BCFBFFE704B080BD000080B584B0C7
:10CF800003900398806B0290FAF72AFB01900398B4
:10CF90000068006800F48070B0F5807F2BD0FFE758
:10CFA00002980168486820F0200048600298019AC1
:10CFB000642100F099F830B1FFE70299486D40F024
:10CFC00020004865FFE702980168486820F00300E8
:10CFD000486002990020C8860299C88702990120FA
:10CFE00081F851000298406D20B1FFE70298FBF7ED
:10CFF000E1FA04E0FFE70298FCF7C6FBFFE704B0A4
:10D0000080BD000080B586B0049003910292049820
:10D010004068B0F5827F13D1FFE704988068B0F5CF
:10D02000004F06D0FFE704988068B0F5806F07D105
:10D03000FFE704980168086820F040000860FFE7F7
:10D0400004984068B0F5827F31D1FFE7049880688A
:10D05000B0F5806F15D0FFE70498039B02996A46EC
:10D0600011608021002200F0BDF848B1FFE704996B
:10D07000486D40F02000486503208DF817002FE030
:10D0800014E00498039B02996A4611600121002272
:10D0900000F0A8F848B1FFE70499486D40F020007F
:10D0A000486503208DF817001AE0FFE714E00498A4
:10D0B000039B02996A4611600121002200F092F858
:10D0C00048B1FFE70499486D40F02000486503200F
:10D0D0008DF8170004E0FFE700208DF81700FFE748
:10D0E0009DF8170006B080BD80B586B0049003910E
:10D0F00002920498039B02996A4611600221012260
:10D1000000F070F848B1FFE70499486D40F0200046
:10D11000486503208DF8170048E040F20000C2F295
:10D12000000000684AF6AB21CAF6AA21A0FB011054
:10D1300000094DF68361C4F21B31A0FB0110800C85
:10D140004FF47A714843019004984068B0F5827FAB
:10D1500015D1FFE70498039B02996A46116080216C
:10D16000002200F03FF848B1FFE70499486D40F015
:10D170002000486503208DF8170017E012E0FFE754
:10D18000019808B9FFE70CE0019801380190FFE72A
:10D19000049800688068C1B20020B0EBD11FEFD1C5
:10D1A000FFE7FFE700208DF81700FFE79DF8170065
:10D1B00006B080BD82B000900098006843F2000184
:10D1C000C4F20101884204D1FFE700208DF8070076
:10D1D00003E002208DF80700FFE79DF8070002B08A
:10D1E0007047000080B58AB0DDF830C00890079124
:10D1F0008DF81B20059305980190FAF7F1F9024686
:10D2000001980C99891A08440390FAF7E9F90290F9
:10D21000039840F20001C2F200010968C1F3CB316A
:10D2200048430490FFE70898006880680799084021
:10D23000401AB0FA80F040099DF81B1088425FD078
:10D24000FFE705980130002859D0FFE7FAF7C8F941
:10D250000299401A0399884204D2FFE703980028F4
:10D2600042D1FFE708980168486820F0E000486074
:10D2700008984068B0F5827F13D1FFE7089880686E
:10D28000B0F5004F06D0FFE708988068B0F5806FD2
:10D2900007D1FFE708980168086820F0400008609F
:10D2A000FFE70898806AB0F5005F0FD1FFE7FFE75E
:10D2B00008980168086820F4005008600898016820
:10D2C000086840F400500860FFE7FFE70899012074
:10D2D00081F85100FFE70899002081F85000FFE72E
:10D2E00003208DF827000FE0049818B9FFE700200D
:10D2F000039003E0049801380490FFE7FFE792E70A
:10D3000000208DF82700FFE79DF827000AB080BDB8
:10D31000074B19680868B0E8F04F80F30988BFF33D
:10D320006F8F4FF0000080F31188704700BF00BF7F
:10D330008012002080B56FF00400002102F01CFD77
:10D3400080BD000084B003900291039890ED000A24
:10D35000029890ED001A30EE010A8DED010A9DED64
:10D36000010AB7EE001AB4EE410AF1EE10FA1BDD25
:10D37000FFE79DED011AB7EE000A80EE010A8DED80
:10D38000000A9DED001A039890ED000A20EE010AB4
:10D3900080ED000A9DED001A029890ED000A20EE43
:10D3A000010A80ED000AFFE704B0704780B586B03F
:10D3B00004900391049828B1FFE70498B0F82C0179
:10D3C00020B9FFE7FF208DF817004FE0049890ED9B
:10D3D000020A90ED4A1A30EE410A8DED020A0498D5
:10D3E000D0ED360A90ED680A9FED221AF6F746FE58
:10D3F0008DED010A9DED020A0498006A90ED072A5E
:10D40000B7EE001A81EE021AB4EE410AF1EE10FAFC
:10D4100028DBFFE70398C078C00718B3FFE79DED4E
:10D42000010AB7EE001AB4EE410AF1EE10FA19DC67
:10D43000FFE704998868C1F82801049901F5D070C4
:10D44000096A91ED060AB8EE400ADFED0A0A80EE9D
:10D45000800AF6F7D1FD0499B1F82C010138A1F842
:10D460002C01FFE700208DF81700FFE79DF917005A
:10D4700006B080BDDB0FC94080B586B00490039133
:10D48000049818B1FFE7039820B9FFE7FF208DF853
:10D49000170036E0F5F760FF08F09DFC00EE100A7B
:10D4A0009FED1A1A8DED011A80EE010A049880EDA5
:10D4B000020AF5F751FF049A029213695269C01AE1
:10D4C000914108F088FC9DED011A0146029800EE9A
:10D4D000101A80EE010A80ED060AF5F73DFF0A46B4
:10D4E00004994A61086103980078049900F00100EA
:10D4F00008700498039900F0E1F800208DF81700F7
:10D50000FFE79DF9170006B080BD00BF00247449F5
:10D5100080B58AB0089007918DED060A089858B139
:10D52000FFE7079840B1FFE79DED060AB5EE400A18
:10D53000F1EE10FA04DCFFE7FF208DF82700B9E0D8
:10D54000079840688DF81700079808990862F4F763
:10D55000EDFF00200490FFE704989DF81710884223
:10D5600048DAFFE70798049901EB810100EB4100DD
:10D570003030FEF793F908980499C1EB011100EBE4
:10D58000810000F5D2709DED060A079901F1740241
:10D5900001210391FFF7D6FA03990898049AC2EB88
:10D5A000021200EB820000F543709DED060A079A17
:10D5B0009432FFF7C7FA0899049801EB401000F283
:10D5C000EC409DED060A096AD1ED4D0AFDF720FBFE
:10D5D0000899049801EB401000F2AC509DED060A4A
:10D5E000096AD1ED4E0AFDF713FBFFE704980130FD
:10D5F0000490B1E707986C30FEF750F90898006A7C
:10D6000090F8700001460291E0B1FFE7029801280E
:10D610002FD1FFE7089800F274409DED060A0799A4
:10D6200001F1F40201210191FFF78CFA01990898A8
:10D6300000F596609DED060A079A02F58A72FFF7DB
:10D6400081FA1AE0089800F274409DED060A0799E5
:10D6500001F1B40201210091FFF774FA00990898D2
:10D6600000F596609DED060A079AD432FFF76AFA34
:10D6700003E0FC208DF827001CE0089901F26C60A3
:10D680009DED060A096AD1ED4F0AFDF7C1FA089926
:10D6900001F28C609DED060A096AD1ED500AFDF792
:10D6A000B7FA08990020C1F82C01C1F828018DF8BB
:10D6B0002700FFE79DF927000AB080BD80B584B040
:10D6C00002900191029820B9FFE7FF208DF80F002A
:10D6D000C2E00298006A90F82400C007002800F019
:10D6E000AB80FFE7029890F82401014600910328DF
:10D6F00000F29C800099DFE801F00220547102984A
:10D7000090ED260A9FED581A80EE010A006A90ED0E
:10D710000A1AB4EE410AF1EE10FA09DDFFE70299A8
:10D72000012081F8240102998868C1F82001FFE7EF
:10D730000298019900F090F97DE0029890ED260A98
:10D740009FED491A80EE010A006A90ED0A1AB4EEC4
:10D75000410AF1EE10FA05DAFFE70299002081F89C
:10D76000240168E0029890ED020A90ED481A30EE2C
:10D77000410A006A90ED0B1AB4EE410AF1EE10FA7C
:10D7800009DBFFE70299012081F81C0102990220C0
:10D7900081F824014FE0FFE70298019900F05CF95D
:10D7A00049E002990020A1F82C01029890ED360A78
:10D7B000016A91ED061AB8EE412A9FED291A81EE11
:10D7C000021A30EE010A80ED680A0299032081F8FE
:10D7D000240102998868C1F82001FFE702980199A5
:10D7E00000F03AF9029890ED020A90ED481A30EEF6
:10D7F000410A9FED1C1AB4EE410AF1EE10FA14DB57
:10D80000FFE7029890ED260A9FED171A80EE010AB5
:10D81000B3EE041AB4EE410AF1EE10FA05DAFFE7AE
:10D820000299002081F82401FFE704E0029900201A
:10D8300081F82401FFE70BE00299002081F8240120
:10D84000029981F81C010298019900F005F9FFE79F
:10D8500000208DF80F00FFE79DF90F0004B080BD98
:10D86000DB0FC9C09A99993E00007A4480B586B012
:10D870000490049820B9FFE7FF208DF817005AE0C4
:10D880000498006A40688DF80F0000200290FFE7BE
:10D8900002989DF80F1088422FDAFFE7049802994A
:10D8A000C1EB011100EB810000F5D270FFF716FA11
:10D8B00004980299C1EB011100EB810000F543705F
:10D8C000FFF70CFA0498029900EB411000F2EC40CB
:10D8D0009FED1B0A8DED010AFDF738FA9DED010A57
:10D8E0000498029900EB411000F2AC50FDF72EFABB
:10D8F000FFE7029801300290CAE7049800F27440F2
:10D90000FFF7ECF9049800F59660FFF7E7F9049843
:10D9100000F26C609FED0A0A8DED000AFDF716FA21
:10D920009DED000A049800F28C60FDF70FFA0020CC
:10D930008DF81700FFE79DF9170006B080BD00BF06
:10D940000000000080B584B00290029820B9FFE783
:10D95000FF208DF80F0034E00298006A40688DF8CF
:10D96000070000200090FFE700989DF8071088420C
:10D9700019DAFFE702980099C1EB011100EB810071
:10D9800000F5D270FFF7CEF902980099C1EB0111B2
:10D9900000EB810000F54370FFF7C4F9FFE7009842
:10D9A00001300090E0E7029800F27440FFF7BAF906
:10D9B000029800F59660FFF7B5F900208DF80F008A
:10D9C000FFE79DF90F0004B080BD000084B0029015
:10D9D000029820B9FFE7FF208DF80F0038E0029889
:10D9E000006A40688DF8070000200090FFE700986B
:10D9F0009DF8071088421EDAFFE70298009900EBB5
:10DA000081010020C1F830010299009A01EB8201E6
:10DA1000C1F848010299009A01EB8201C1F8600146
:10DA20000299009A01EB8201C1F87801FFE70098A2
:10DA300001300090DBE702990020C1F890010299C3
:10DA4000C1F894010299C1F898018DF80F00FFE721
:10DA50009DF90F0004B0704780B594B012901191F9
:10DA6000129818B1FFE7119820B9FFE7FF208DF851
:10DA70004F0008E31298006A40688DF8430012983E
:10DA80000078C007F0B9FFE700200F90FFE70F987C
:10DA90009DF8431088420FDAFFE71298006A0F9949
:10DAA00001EB810100EB41003030FDF787FFFFE71C
:10DAB0000F9801300F90EAE71298006A6C30FDF77A
:10DAC0007DFFBDE2129890F818010146079150B110
:10DAD000FFE70798012800F0AB80FFE707980228CE
:10DAE00000F0C681A6E200200E90FFE70E989DF898
:10DAF0004310884251DAFFE712980E99C1EB0111E9
:10DB000000EB810000F5D270FFF70CF912990E9A24
:10DB1000C2EB021001EB800000F5D27001EB820233
:10DB2000D2ED3E0AD1ED061A9FEDD81AB0EE410AA9
:10DB3000FEF790FE12980E9900EB810080ED4C0AE2
:10DB400012980E9900EB8101D1F83001C1F8600103
:10DB500012990E9A01EB421000F2AC5001EB8201D7
:10DB600091ED580AFCF7F8FF12980E9900EB81002E
:10DB700080ED5E0A1299086A0E9A02EB820300EBAE
:10DB80004300303001EB820191ED5E0AFDF722FF88
:10DB9000FFE70E9801300E90A8E7129901F2744049
:10DBA00040F28452C2F2000292ED000AD1ED061A50
:10DBB000D1ED360A9FEDB51A8DED061AFEF74AFE35
:10DBC0009DED061A129880ED640A129901F596608F
:10DBD000D1ED061AD1ED450A91ED640AFEF73AFE41
:10DBE000129880ED650A129901F28C6091ED650A38
:10DBF000FCF7B2FF129880ED660A1299086A6C3041
:10DC000091ED660AFDF7E6FE11988078C00770B1C5
:10DC1000FFE71298FFF72AFE1298FFF793FE12987B
:10DC2000FFF7D4FE1299012081F81801FFE706E200
:10DC300000200D90FFE70D989DF84310884280F278
:10DC40009680FFE71298006A90F8380001388DF846
:10DC500033001298016A9DF8332001EB820191EDA7
:10DC6000030A90ED671A20EE010A9FED891A80EEF3
:10DC7000010A8DED0B0A129890ED670A80EE010AF9
:10DC800040F2D050C2F2000080ED000A12990D9AC5
:10DC9000C2EB021001EB800000F5D2709DED0B0A83
:10DCA00001EB8202D2ED3E0AD1ED061A9FED771A02
:10DCB0008DED051AFEF7CEFD9DED051A12980D9912
:10DCC00000EB810080ED4C0A129A0D99C1EB011016
:10DCD00002EB800000F5437002EB8101D2ED061AE1
:10DCE00092ED440AD1ED3E0AFEF7B4FD12980D996B
:10DCF00000EB810080ED520A12980D9900EB810132
:10DD000001F5987001F5A471FFF71CFB12980D99AD
:10DD100000EB810090ED4C0A90ED521A30EE010AB2
:10DD200080ED580A12990D9A01EB421000F2AC50A6
:10DD300001EB820191ED580AFCF70EFF12980D9944
:10DD400000EB810080ED5E0A1299086A0D9A02EBE1
:10DD5000820300EB4300303001EB820191ED5E0A5B
:10DD6000FDF738FEFFE70D9801300D9063E712993B
:10DD700001F2744040F28452C2F2000292ED000AB5
:10DD8000D1ED061AD1ED360A9FEDC11A8DED041AB8
:10DD9000FEF760FD9DED041A129880ED640A129959
:10DDA00001F59660D1ED061AD1ED450A91ED640AB0
:10DDB000FEF750FD129880ED650A129901F28C6011
:10DDC00091ED650AFCF7C8FE129880ED660A12997B
:10DDD000086A6C3091ED660AFDF7FCFD11988078B9
:10DDE000C00758B9FFE71298FFF740FD1298FFF7F8
:10DDF000EDFD1299002081F8180138E041F24B1036
:10DE0000C2F200000078C00780BBFFE71198C0781D
:10DE1000C00758B3FFE71299022081F81801129841
:10DE200090F8240001460391012808D0FFE70398E9
:10DE3000022809D0FFE7039803280BD010E01299BD
:10DE40000120A1F82C0110E01299086A006AA1F8DB
:10DE50002C010AE0129941F60A20A1F82C0104E0F5
:10DE600012990020A1F82C01FFE7FFE7FFE7E6E0A9
:10DE700012981199FFF79AFA00200A90FFE70A9882
:10DE80009DF84310884280F28F8003E0000000007C
:10DE900000C0DA451298006A90F8380001388DF811
:10DEA00027001298016A9DF8272001EB820191ED6D
:10DEB000030A90ED671A20EE010A9FED761A80EEB4
:10DEC000010A8DED080A12990A9AC2EB021001EBC1
:10DED000800000F5D2709DED080A01EB8202D2EDC0
:10DEE0003E0AD1ED061A9FED6A1A8DED021AFEF771
:10DEF000B1FC9DED021A12980A9900EB810080EDA9
:10DF00004C0A129A0A99C1EB011002EB800000F54D
:10DF1000437002EB8101D2ED061A92ED440AD1ED75
:10DF20003E0AFEF797FC12980A9900EB810080EDFB
:10DF3000520A12980A9900EB810101F5987001F5D7
:10DF4000A471FFF7FFF912980A9900EB810090ED98
:10DF50004C0A90ED521A30EE010A80ED580A1299DF
:10DF60000A9A01EB421000F2AC5001EB820191EDF4
:10DF7000580AFCF7F1FD12980A9900EB810080ED38
:10DF80005E0A1299086A0A9A02EB820300EB4300C8
:10DF9000303001EB820191ED5E0AFDF71BFDFFE7DA
:10DFA0000A9801300A906AE7129901F27440D1EDA3
:10DFB000061AD1ED360A91ED680A9FED351A8DEDFE
:10DFC000011AFEF747FC9DED011A129880ED640AD4
:10DFD000129901F59660D1ED061AD1ED450A91ED41
:10DFE000640AFEF737FC129880ED650A129901F277
:10DFF0008C6091ED650AFCF7AFFD129880ED660A22
:10E000001299086A6C3091ED660AFDF7E3FC1198ED
:10E01000C078C00768B9FFE71299012081F818019C
:10E020001298D0F8D80040F28451C2F20001086082
:10E03000FFE704E01299002081F81801FFE7FFE7ED
:10E040001298006A3030FDF78BFA1298006A406827
:10E05000052806D3FFE71298006A5830FDF780FACA
:10E06000FFE71298006A6C30FDF77AFA1198C078D1
:10E0700000F0010041F24B11C2F2000108700020D3
:10E080008DF84F00FFE79DF94F0014B080BD00BF31
:10E090000000000000C0DA4583B001908DF8031045
:10E0A000019820B9FFE7FF208DF80B000BE09DF8E9
:10E0B0000300019981F8240001990020A1F82C01A6
:10E0C0008DF80B00FFE79DF90B0003B070470000CF
:10E0D00080B588B00690069820B9FFE7FF208DF83C
:10E0E0001F0041E1002005900699096A49688DF8F2
:10E0F00013100390FFE703989DF81310884280F2F5
:10E100008B80FFE70698006A039901EB810100EB21
:10E1100041003030FDF7ECFC0698006A039901EBF2
:10E12000810100EB41003030FDF754FB0290029872
:10E13000A0B1FFE70698039900EB0111DDF808C0D4
:10E14000DCF82C00DCF83020DCF83430DCF838C0A7
:10E15000C1F834C00B63CA628862FFE70699039A6C
:10E1600001EB421000F2EC4001EB021191ED0B0AC1
:10E17000FCF7F2FC0698039900EB810080ED370A6A
:10E180000698039900EB810090ED370A9FED7B1A0A
:10E1900080EE010A80ED3E0A0698039900EB8100AB
:10E1A00090ED3E0AB7EE001AB4EE410AF1EE10FA15
:10E1B00009DDFFE70698039900EB81014FF07E50DF
:10E1C000C1F8F800FFE70698039900EB810090ED95
:10E1D0003E0ABFEE001AB4EE410AF1EE10FA0ADA76
:10E1E000FFE70698039900EB81010020CBF68070D1
:10E1F000C1F8F800FFE70698039900EB810090ED65
:10E200003E1A9DED050A30EE010A8DED050AFFE785
:10E210000398013003906EE79DED050A9DF8130009
:10E2200001EE100AB8EEC11A80EE010A069880EDE0
:10E23000440A0698006A6C30FDF75AFC069800F113
:10E2400088010191006A6C30FDF7C4FA014601981B
:10E250005022F2F720F90698016A91ED050A90ED37
:10E26000341A20EE010A80ED360AFFE7069890ED99
:10E27000360AB5EE400AF1EE10FA0ADAFFE7069820
:10E2800090ED360A9FED3A1A30EE010A80ED360A1B
:10E29000ECE7FFE7069890ED360A9FED351AB4EEED
:10E2A000410AF1EE10FA0ADBFFE7069890ED360A14
:10E2B0009FED311A30EE010A80ED360AEAE7069842
:10E2C00090F8B000C00750B1FFE7069890ED361AFD
:10E2D0009FED270A30EE410A80ED360AFFE70699E6
:10E2E00001F26C6091ED250AFCF736FC069880ED92
:10E2F0003D0A069890ED250A9FED1E1A80EE010A50
:10E3000080ED450A069890ED450AB7EE001AB4EE86
:10E31000410AF1EE10FA06DDFFE706994FF07E5054
:10E32000C1F81401FFE7069890ED450ABFEE001A08
:10E33000B4EE410AF1EE10FA07DAFFE70699002081
:10E34000CBF68070C1F81401FFE7069890ED0B0A38
:10E3500090ED0F1A30EE410A00F2AC6080ED000A39
:10E3600000208DF81F00FFE79DF91F0008B080BD59
:10E37000DB0FC94000409C45DB0FC9C000C0DA4537
:10E3800080B582B0019002F0C3FA02F077FB02B0D0
:10E3900080BD000080B582B0009000980138B0F1D7
:10E3A000807F03D3FFE70120019019E00098013836
:10E3B0004EF21401CEF2000108604FF0FF300F2141
:10E3C00001F0B8FC4EF21801CEF200010020086006
:10E3D0004EF21002CEF20002072111600190FFE719
:10E3E000019802B080BD000080B5F9F7EFFA05F0A2
:10E3F00071FB012803D0FFE704F088FAFFE780BD36
:10E4000080B594B008A83021F2F77FF8002007907B
:10E410000690059004900390FFE70020029043F6D9
:10E420004000C4F20200016841F0805101600068C0
:10E4300000F0805002900298FFE7FFE70020019073
:10E4400047F20000C4F20000016841F4804101601D
:10E45000006800F4804001900198FFE701200890D7
:10E460004FF48030099002200E904FF480010F91FC
:10E4700006211091A821119112900420139008A850
:10E48000F9F738FD18B1FFE7F6F736FEFFE70F2082
:10E49000039002200490002005904FF4A0500690B5
:10E4A0004FF48050079003A80521F9F753FB18B1EA
:10E4B000FFE7F6F721FEFFE714B080BD4EF6885166
:10E4C000CEF20001086840F4700008607047000058
:10E4D00083B0029001910298006800900298002198
:10E4E000C4F20101884225D0FFE70298B0F1804FC5
:10E4F00020D0FFE7029840F20041C4F200018842B8
:10E5000018D0FFE7029840F60001C4F200018842EB
:10E5100010D0FFE7029840F60041C4F200018842A3
:10E5200008D0FFE7029840F20041C4F2010188429E
:10E530000AD1FFE7009820F0700000900198416830
:10E54000009808430090FFE702980021C4F20101FF
:10E55000884255D0FFE70298B0F1804F50D0FFE7D6
:10E56000029840F20041C4F20001884248D0FFE71F
:10E57000029840F60001C4F20001884240D0FFE753
:10E58000029840F60041C4F20001884238D0FFE70B
:10E59000029840F20041C4F20101884230D0FFE706
:10E5A000029844F20001C4F20101884228D0FFE73A
:10E5B000029844F20041C4F20101884220D0FFE7F2
:10E5C000029844F60001C4F20101884218D0FFE726
:10E5D000029841F60001C4F20001884210D0FFE722
:10E5E000029841F60041C4F20001884208D0FFE7DA
:10E5F000029842F20001C4F2000188420AD1FFE70A
:10E60000009820F4407000900198C1680098084379
:10E610000090FFE7009820F08000019949690843C5
:10E620000090019880680299C86201980068029978
:10E63000886202980021C4F20101884208D0FFE7F5
:10E64000029840F20041C4F20101884205D1FFE77F
:10E650000198006902990863FFE70299086840F091
:10E66000040008600299012048610098029908603E
:10E6700003B0704784B0039002910192029800F0B9
:10E680001F01012088400090009A0399086A904376
:10E6900008620198029901F01F0100FA01F2039942
:10E6A000086A1043086204B07047000085B0049007
:10E6B000039102920193049880680090009820F4DE
:10E6C0007F40009003980299019A41EA0221014398
:10E6D00000980843009000980499886005B070473E
:10E6E00083B002900191029880680090009820F019
:10E6F0007000009001980099084340F007000090D6
:10E7000000980299886003B07047000085B00490BB
:10E7100003910498006A01900499086A20F00100AE
:10E7200008620498406800900498806902900298FA
:10E7300020F070000290029820F0030002900398ED
:10E740000168029808430290019820F002000190AD
:10E750000398816801980843019004980021C4F24D
:10E760000101884208D0FFE7049840F20041C4F25A
:10E77000010188420ED1FFE7019820F008000190C6
:10E780000398C168019808430190019820F00400A3
:10E790000190FFE704980021C4F20101884208D0EB
:10E7A000FFE7049840F20041C4F20101884213D10E
:10E7B000FFE7009820F480700090009820F400702B
:10E7C000009003984169009808430090039881697C
:10E7D000009808430090FFE7009804994860029869
:10E7E00004998861039840680499486301980499E2
:10E7F000086205B07047000085B00490039104984A
:10E80000006A01900499086A20F0100008620498D8
:10E8100040680090049880690290029820F4E040DB
:10E820000290029820F440700290039801680298C8
:10E8300040EA01200290019820F020000190039806
:10E840008168019840EA0110019004980021C4F207
:10E850000101884208D0FFE7049840F20041C4F269
:10E86000010188420FD1FFE7019820F0800001905C
:10E870000398C168019840EA01100190019820F0C6
:10E8800040000190FFE704980021C4F20101884292
:10E8900008D0FFE7049840F20041C4F20101884229
:10E8A00015D1FFE7009820F480600090009820F4D4
:10E8B0000060009003984169009840EA8100009050
:10E8C00003988169009840EA81000090FFE7009872
:10E8D00004994860029804998861039840680499F3
:10E8E000886301980499086205B0704785B0049068
:10E8F00003910498006A01900499086A20F48070DA
:10E9000008620498406800900498C06902900298D8
:10E9100020F070000290029820F00300029003980B
:10E920000168029808430290019820F40070019059
:10E9300003988168019840EA012001900498002121
:10E94000C4F20101884208D0FFE7049840F2004178
:10E95000C4F2010188420FD1FFE7019820F4006062
:10E9600001900398C168019840EA01200190019844
:10E9700020F480600190FFE704980021C4F20101B7
:10E98000884208D0FFE7049840F20041C4F2010138
:10E99000884215D1FFE7009820F48050009000983D
:10E9A00020F40050009003984169009840EA01105B
:10E9B000009003988169009840EA01100090FFE7F9
:10E9C00000980499486002980499C86103984068C7
:10E9D0000499C86301980499086205B07047000063
:10E9E00085B0049003910498006A01900499086A24
:10E9F00020F4805008620498406800900498C06930
:10EA00000290029820F4E0400290029820F44070B6
:10EA1000029003980168029840EA01200290019850
:10EA200020F40050019003988168019840EA013079
:10EA3000019004980021C4F20101884208D0FFE748
:10EA4000049840F20041C4F2010188420BD1FFE773
:10EA5000009820F48040009003984169009840EAB3
:10EA600081100090FFE7009804994860029804998B
:10EA7000C861039840680499086401980499086281
:10EA800005B0704785B00490039102920498006A23
:10EA900000900499086A20F00100086204988069D7
:10EAA0000190019820F0F00001900299019840EA4D
:10EAB00001100190009820F00A000090039900983E
:10EAC00008430090019804998861009804990862AD
:10EAD00005B0704785B00490039102920498006AD3
:10EAE00000900499086A20F0100008620498806978
:10EAF0000190019820F4704001900299019840EA39
:10EB000001300190009820F0A00000900399009837
:10EB100040EA0110009001980499886100980499D6
:10EB2000086205B07047000080B588B0079001F01A
:10EB3000FBFA4FF29130C0F6000046F22412C0F604
:10EB400001020021049101F0EBFE049941F60C62F0
:10EB5000C2F20002069210604EF69140C0F600002C
:10EB600046F22802C0F6010201F0DAFE0499069A84
:10EB700050604EF63170C0F6000046F24C02C0F60E
:10EB8000010201F0CDFE0499069A90604FF209103F
:10EB9000C0F6000046F29402C0F6010201F0C0FE89
:10EBA0000499069AD0604FF2E910C0F6000046F2D0
:10EBB000B802C0F6010201F0B3FE0499069A106192
:10EBC0004FF2E120C0F6000046F2DC02C0F601027E
:10EBD00001F0A6FE0499069A50614EF6E170C0F667
:10EBE000000046F27002C0F6010201F099FE049A9C
:10EBF00006998861022005900A2101F083FB049A9E
:10EC00000699C861032002905821019101F07AFB16
:10EC10000199049ADDF818C003460298CCF8383000
:10EC200001F070FB049A069B01460598D963042104
:10EC3000039101F067FB049A069B014602989962D2
:10EC4000102101F05FFB049A069B0146059859626A
:10EC5000182101F057FB049A069B01460598D962DA
:10EC60000C2101F04FFB0399049ADDF818C003460C
:10EC70000598CCF8303001F045FB0699486301F067
:10EC8000A9FA01F045FE01F0F9FE08B080BD0000D0
:10EC900080B58CB00B9001F01FFA06F066FE41ECD7
:10ECA000100B9FED9D1B53EC112B51EC100B06F03C
:10ECB00099FC41EC100B51EC100B06F029FE0A9068
:10ECC0000020089001F084F901F0F2F9099040F277
:10ECD000D850C2F20000079040F27801C2F2000161
:10ECE000F2F7F2FF0798F2F7C7FF40F60840C2F2CA
:10ECF000000041F24C11C2F20001F1F727FD079824
:10ED0000F2F7BAFF0899B0EE401AB7EE000A80EEAB
:10ED1000010A41F20C10C2F2000046F27C12C0F669
:10ED20000102FDF70FFF0120F4F7D4F9089841F62E
:10ED30004D41C0F60101F4F7B5F80898F4F760F812
:10ED4000FFE70A99099808440990F3F7ADF9F2F73B
:10ED50007BFFF2F789FFF2F7A1FFF2F7ADFF01F0B9
:10ED6000E3F940F2D850C2F200000690F3F770F8D1
:10ED70000698F3F7E7F840F22060C2F2000000784E
:10ED8000012865D1FFE740F2D851C2F2000191EDB0
:10ED9000071A40F65840C2F2000090ED000A30EE2B
:10EDA000010A80ED000A91ED081A90ED010A30EE9B
:10EDB000010A80ED010A91ED091A90ED020A30EE88
:10EDC000010A80ED020A40F21E60C2F200000188D2
:10EDD00001310180008841F28831884237DBFFE74A
:10EDE00040F65840C2F2000090ED000A9FED4C1A28
:10EDF00080EE010A40F27801C2F2000181ED000AC2
:10EE000090ED010A80EE010A81ED010A90ED020AFF
:10EE100080EE010A81ED020A40F22062C2F2000295
:10EE20000020107040F2D850C2F200000590F2F7B6
:10EE30004BFF0598F2F720FF40F60840C2F20000B1
:10EE400041F24C11C2F20001F1F780FCFFE7FFE74D
:10EE500040F22060C2F20000007801281BD0FFE7DA
:10EE600040F2D850C2F2000000F1100100F11C0283
:10EE700040F60840C2F20000049041F24C13C2F286
:10EE80000003F1F7AFFD049940F65820C2F20000EC
:10EE9000F1F7AEFBFFE701F09DF940F65821C2F211
:10EEA000000108684A688B6840F64041C2F20001E0
:10EEB00001914B610A61C86040F2D853C2F200036D
:10EEC0000393D8691A6A5B6A8B604A60086041F6EE
:10EED0000C60C2F200000290C06A01F0F5FA0199DC
:10EEE0000298C06A00231A4601F08CFA0398D0ED0C
:10EEF0000A0A41F20C10C2F200009FED0A0ADFED8F
:10EF00000A1AB0EE611AFDF7A5FC0120F4F742F8E9
:10EF1000099801F077F814E70000000000407F40F6
:10EF200000409C450000204200000000000000005E
:10EF300080B586B0059001F0CFF806F016FD41ECE3
:10EF4000100B9FED231B53EC112B51EC100B06F013
:10EF500049FB41EC100B51EC100B06F0D9FC04906E
:10EF6000002001F035F801F0A3F803900420F4F735
:10EF7000D3F80220F4F7D0F8032001909FED160A91
:10EF8000F4F708F80198F4F7A5F8FFE70499039857
:10EF9000084403909DED030AB8EE400A9FED0F1A56
:10EFA00020EE010A05F012FFB7EE001A30EE010A5A
:10EFB000B6EE001A20EE010A8DED020A9DED020A5E
:10EFC0000320F3F7E7FF039801F01CF8DEE700BF2A
:10EFD000000000000000594000000000A69B443BD8
:10EFE00010B58AB0099001F077F806F0BEFC41EC4C
:10EFF000100B9FED431B53EC112B51EC100B06F043
:10F00000F1FA41EC100B51EC100B06F081FC08906A
:10F01000002000F0DDFF01F04BF80790F5F76AFDE6
:10F0200000F51B7140F62810C2F20000F5F798F9C0
:10F03000FFE7089907980844079041F60C60C2F270
:10F0400000000690806B40F60021C2F20001002310
:10F0500005931A4601F0F6F840F62810C2F20000B7
:10F060000190F5F7A5F8019A0698D2F8511040F6EC
:10F070009C13C2F2000303931960116BD2F834C0E1
:10F08000D2F838E0D46B40F68013C2F20003049348
:10F09000DC60C3F808E0C3F804C01960516C936CDD
:10F0A000D2F84CC040F69012C2F200020292C2F8AE
:10F0B00008C053601160006B01F006FA0299059BCD
:10F0C0000698006B1A4601F09DF90698406B01F016
:10F0D000FBF90399059B0698406B1A4601F092F9DB
:10F0E0000698406A01F0F0F90499059B0698406A79
:10F0F0001A4601F087F9079800F084FF99E700BFEE
:10F100000000000000407F4080B58AB0099000F008
:10F11000E3FF06F02AFC41EC100B9FED2F1B53EC94
:10F12000112B51EC100B06F05DFA41EC100B51EC79
:10F13000100B06F0EDFB0890002000F049FF00F0F6
:10F14000B7FF0790F5F7D6FC0690069800F5F67124
:10F1500040F23860C2F2000005909FED210AF4F7FA
:10F160001FFD059942F6F600C4F284000863FFE72C
:10F17000089907980844079041F60C60C2F2000015
:10F180000290806A40F23861C2F20001049101F5F8
:10F190003771002301931A4601F054F8019B02983D
:10F1A000406A40F61811C2F2000103911A4601F0BC
:10F1B00049F80498F4F7C4FE00F07AFF0399024678
:10F1C0000498F4F727FB0498F4F7ECFD079800F097
:10F1D00019FFCDE700BF00BF0000000000407F40E6
:10F1E0000000FA430000000080B588B0079000F0EE
:10F1F00073FF06F0BAFB41EC100B9FED351B53EC8F
:10F20000112B51EC100B06F0EDF941EC100B51EC09
:10F21000100B06F07DFB0690002000F0D9FE00F0F8
:10F2200047FF0590F5F766FC00F5A27140F66820EF
:10F23000C2F200009FED280AF6F746F9FFE70699AB
:10F2400005980844059041F60C60C2F20000C06ABF
:10F2500040F62841C2F2000100231A4600F0F2FFF6
:10F2600058B9FFE740F66820C2F2000040F6284196
:10F27000C2F20001F6F79CFAFFE741F60C60C2F219
:10F2800000000290006B40F61C41C2F200010391A5
:10F29000002301931A4600F0D5FF40F66820C2F221
:10F2A00000000490F6F730FA019B04990298806AF6
:10F2B00001F5C0711A4601F0A5F803990498F5F715
:10F2C0001FFF0498F6F78EF9059800F09BFEB6E74D
:10F2D0000000000000407F400000FA4300000000F2
:10F2E00080B586B0059000F0F7FE06F03EFB41ECDD
:10F2F000100B9FED231B53EC112B51EC100B06F060
:10F3000071F941EC100B51EC100B06F001FB04906D
:10F31000002000F05DFE00F0CBFE0390F5F7EAFB65
:10F32000014641F25870C2F2000002909FED160AA9
:10F33000FEF7EEF802980221FEF7AEFEFFE7049911
:10F3400003980844039041F60C60C2F20000406B41
:10F3500041F60861C2F20001009100231A4600F054
:10F3600071FF41F25870C2F200000190FEF7B0FE4A
:10F3700000990198FEF780F8039800F043FEDEE75D
:10F380000000000000407F400000FA430000000041
:10F3900080B584B0039000F09FFE06F0E6FA41ECE1
:10F3A000100B9FED251B53EC112B51EC100B06F0AD
:10F3B00019F941EC100B51EC100B06F0A9FA029070
:10F3C000002000F005FE00F073FE019040F6A8104A
:10F3D000C2F20000F5F712FDFFE702990198084418
:10F3E000019040F6A810C2F20000F5F743FE142089
:10F3F000F5F75AFE38B1FFE740F6A810C2F2000058
:10F40000F5F752FD06E040F6A810C2F20000F5F74D
:10F410002FFDFFE741F60C60C2F20000806B40F662
:10F42000A811C2F2000100231A4600F0EBFF019878
:10F4300000F0E8FDD1E700BF0000000000407F4081
:10F4400080B582B001900198806B009000990020F7
:10F45000C8850098FAF7E0FE02B080BD80B584B0A0
:10F460000390002002900398806B0190019800683F
:10F470004069C0B2C0090290019890F8410021286B
:10F480000AD1FFE7029838B1FFE701990020C8844C
:10F49000019800F013F9FFE7019800684069C0F394
:10F4A00080100290019890F8420022280AD1FFE7CC
:10F4B000029838B1FFE701990020C885019800F053
:10F4C0009FF8FFE70199486C40F0100048640198EC
:10F4D000FAF7A2FE04B080BD80B586B0059005980D
:10F4E000806B0490059800680068C00500285AD415
:10F4F000FFE704990020C885FFE7FFE7049800684C
:10F5000050E8030F20F480700390FFE703990498FC
:10F51000026842E803100028F0D1FFE7FFE7FFE7A9
:10F52000FFE70498006850E8050F20F00100029002
:10F53000FFE702990498026842E805100028F0D11C
:10F54000FFE7FFE7FFE7FFE70498006850E8050FD3
:10F5500020F040000190FFE701990498026842E81A
:10F5600005100028F0D1FFE7FFE70499202081F87B
:10F5700042000498006B012814D1FFE7FFE7FFE782
:10F580000498006850E8030F20F010000090FFE797
:10F5900000990498026842E803100028F0D1FFE7C0
:10F5A000FFE7FFE7FFE70499002048630498006B3A
:10F5B000012805D1FFE70498818DFAF727FE03E0C3
:10F5C0000498FBF70DFAFFE706B080BD80B582B066
:10F5D00001900198806B0090009901204863009889
:10F5E000006B012806D1FFE70098818D4908FAF7E2
:10F5F0000DFE03E00098FBF71DFAFFE702B080BDA7
:10F6000084B00390FFE7FFE70398006850E8030F1A
:10F6100020F490700290FFE702990398026842E894
:10F6200003100028F0D1FFE7FFE7FFE7FFE70398AB
:10F63000006850E8050F20F001000190FFE70199F4
:10F640000398026842E805100028F0D1FFE7FFE7C1
:10F650000398006B012814D1FFE7FFE7FFE7039849
:10F66000006850E8030F20F010000090FFE70099B9
:10F670000398026842E803100028F0D1FFE7FFE793
:10F68000FFE70399202081F84200039900200863D6
:10F6900004B0704780B582B0019001980168C868D5
:10F6A00020F04000C8600199202081F841000198B5
:10F6B000FBF7EAF9002002B080BD000082B00190A3
:10F6C000FFE7FFE70198006850E8030F20F0C00053
:10F6D0000090FFE700990198026842E803100028B3
:10F6E000F0D1FFE7FFE70199202081F8410002B047
:10F6F0007047000082B000900098006844F6000156
:10F70000C4F20001884204D1FFE700208DF8070011
:10F7100010E00098006841F20041C4F20101884203
:10F7200004D1FFE701208DF8070003E003208DF8E6
:10F730000700FFE79DF8070002B0704780B586B06C
:10F740000490002003900290049890F84200222830
:10F7500040F0A080FFE704988068B0F5805F13D187
:10F76000FFE70498006978B9FFE70498806A02907F
:10F770000498006840686FF35F200299088004993C
:10F78000886A0230886223E00498806A03900498B3
:10F790008068B0F5805F08D0FFE70498806850B9B2
:10F7A000FFE70498006930B9FFE7049800684068F3
:10F7B0000399087007E004980068406800F07F0033
:10F7C00003990870FFE70499886A01308862FFE7AF
:10F7D0000499C88D0138C8850004002856D1FFE778
:10F7E00004980168C86820F02000C8600498016887
:10F7F000C86820F48070C86004980168486920F0E7
:10F80000010048610499202081F8420004990020F9
:10F8100048630498006B012830D1FFE70499002069
:10F820000863FFE7FFE70498006850E8030F20F043
:10F8300010000190FFE701990498026842E8031064
:10F840000028F0D1FFE7FFE7049800680068C006D1
:10F8500000280ED5FFE7FFE700200090049800681D
:10F860000068009004980068406800900098FFE7E6
:10F87000FFE70498818DFAF7C9FC03E00498FBF7D1
:10F88000AFF8FFE700208DF8170007E000208DF8A3
:10F89000170003E002208DF81700FFE79DF817001E
:10F8A00006B080BD80B586B00590059800680069F7
:10F8B00020F44050059A1168D268104308610599F8
:10F8C00088680B694A69C969184310430843049062
:10F8D00005980068C06849F20C61884304990843A0
:10F8E00005990968C86005980068406920F440706F
:10F8F000059A11689269104348610598006841F2C1
:10F900000001C4F20101884209D0FFE705980068B0
:10F9100041F20041C4F20101884204D1FFE7F8F747
:10F9200063FA039003E0F8F74DFA0390FFE70598B8
:10F93000C069B0F5004F29D1FFE703981921A0FB5A
:10F940000101059A1368029353685A00DB0FF0F720
:10F95000C7FC0299864648F21F53C5F2EB13AEFB73
:10F960000320420910014FF0640C02FB1CEC322210
:10F9700002EBCC02A2FB0332F82303EA521300EBA2
:10F980004300C2F342121044886026E00398192114
:10F99000A0FB0101059A1368019353689A009B0F1D
:10F9A000F0F79EFC0199844648F21F52C5F2EB1213
:10F9B000ACFB02304309642003FB10CC322000EB87
:10F9C0000C10A0FB0202F02000EA521000EB031022
:10F9D000C2F3431210448860FFE706B080BD000008
:10F9E00080B58AB008900791ADF81A200798089959
:10F9F0008862BDF81A000899888508990020486433
:10FA0000089A222182F842100899CA6B4FF2D94114
:10FA1000C0F60001D1630899CA6B4FF2CD51C0F610
:10FA2000000111640899CA6B4FF25D41C0F60001F4
:10FA3000D1640899C96B086507A805900898016802
:10FA4000C06B0431059A1268BDF81A30F7F7E8FA6E
:10FA500058B1FFE70899102048640899202081F8E0
:10FA6000420001208DF827004EE0FFE700200490BF
:10FA7000089800680068049008980068406804903E
:10FA80000498FFE708980069A0B1FFE7FFE7FFE7E8
:10FA90000898006850E8030F40F480700390FFE777
:10FAA00003990898026842E803100028F0D1FFE7A4
:10FAB000FFE7FFE7FFE7FFE70898006850E8050F5A
:10FAC00040F001000290FFE702990898026842E8BE
:10FAD00005100028F0D1FFE7FFE7FFE7FFE70898F0
:10FAE000006850E8050F40F040000190FFE70199E1
:10FAF0000898026842E805100028F0D1FFE7FFE708
:10FB000000208DF82700FFE79DF827000AB080BD90
:10FB100083B00190019890F8410021283AD1FFE785
:10FB200001988068B0F5805F13D1FFE70198006904
:10FB300078B9FFE70198006A0090009800886FF399
:10FB40005F200199096848600199086A02300862DB
:10FB500008E0019A106A411C116200780199096855
:10FB60004860FFE70199C88C0138C884000468B96F
:10FB7000FFE701980168C86820F08000C86001981C
:10FB80000168C86840F04000C860FFE700208DF8B9
:10FB90000B0003E002208DF80B00FFE79DF80B003F
:10FBA00003B0704780B582B041F2C000C2F20000DD
:10FBB0000190FAF75BFB0198F3F744FC02B080BDBB
:10FBC000FFE7FEE782B041EC100B8DED000B0198D2
:10FBD000C0F30A5040F2FF71401A18BF012002B072
:10FBE0007047000082B041EC100B8DED000B0198C6
:10FBF000C0F30A5040F2FF71401A18BF012002B052
:10FC00007047000082B041EC100B8DED000B0198A5
:10FC1000C0F30A5040F2FF71401A18BF012002B031
:10FC20007047000081B000EE100A00900098C0F309
:10FC3000C750FF3818BF012001B0704781B000EEF7
:10FC4000100A00900098C0F3C750FF3818BF012079
:10FC500001B0704781B000EE100A00900098C0F328
:10FC6000C750FF3818BF012001B0704784B041EC85
:10FC7000100B8DED020B039A00200021CFF6E071EE
:10FC8000B1EB420F019006D1FFE70298B0FA80F085
:10FC900040090190FFE7019800F0010004B07047AF
:10FCA00081B000EE100A009000994FF0807000EBD8
:10FCB0004100B0FA80F0400901B0704781B08DF882
:10FCC00003009DF90300002812D4FFE79DF90310FB
:10FCD00001F01F02012090404A094EF28011CEF23D
:10FCE000000141F82200BFF34F8FBFF36F8FFFE792
:10FCF00001B0704781B08DF803009DF90300002822
:10FD00000ED4FFE79DF9031001F01F02012090407F
:10FD10004A094EF20011CEF2000141F82200FFE73D
:10FD200001B070474EF60C50CEF200000068C0F3F0
:10FD30000220704782B08DF8070000919DF90700FE
:10FD400000280AD4FFE7009800019DF907104EF241
:10FD50000042CEF2000288540BE0009800019DF8AA
:10FD6000071001F00F014EF61452CEF20002885433
:10FD7000FFE702B07047000082B08DF807000091E5
:10FD80009DF9070000280AD4FFE7009800019DF9BB
:10FD900007104EF20042CEF2000288540BE00098A9
:10FDA00000019DF8071001F00F014EF61452CEF23B
:10FDB00000028854FFE702B07047000083B0029051
:10FDC000029800F0070000904EF60C51CEF20001B0
:10FDD0000868019001984FF6FF02104001900198C9
:10FDE000009A40EA02200022C0F2FA521043019029
:10FDF0000198086003B0704780B582B00190019807
:10FE000040F60021C2F200015822F0F744FB02B094
:10FE100080BD000082B08DED010ACDED000A019891
:10FE20000099C90F61F3DF7001909DED010A02B0E6
:10FE30007047000080B588B0069006980190019840
:10FE400058B9FFE74FF0500080F31188BFF36F8F70
:10FE5000BFF34F8F0790FFE7FEE7019841F2802143
:10FE6000C2F200010968884204D1FFE700208DF842
:10FE7000170056E001F0FEFF01984069049041F23E
:10FE80008820C2F200000068039041F29020C2F284
:10FE900000000068029002F019F804980399884263
:10FEA00005D0FFE704980299884204D1FFE70220B9
:10FEB0008DF8170034E0049848F67861C2F200012A
:10FEC000884218D1FFE70198806A78B9FFE7019866
:10FED00090F85800012804D1FFE702208DF81700A0
:10FEE00003E003208DF81700FFE703E002208DF800
:10FEF0001700FFE713E0049848F68C61C2F2000196
:10FF0000884203D0FFE7049820B9FFE704208DF86A
:10FF1000170003E001208DF81700FFE7FFE7FFE778
:10FF2000FFE79DF8170008B080BD000086B08DED9A
:10FF3000050ACDED040A8DED031A02909DED030A2A
:10FF40009DED041A30EE410A8DED010A04980090EF
:10FF50009DED050A9DED001A30EE410A029901203F
:10FF60008840013801EE100AB8EEC11A20EE010AED
:10FF70009DED011A80EE010ABDEEC00A10EE100AD6
:10FF800006B0704780B582B000200190F7F72CFDD5
:10FF9000FEF736FAFBF7FCFEFBF77CFEFBF72AFECA
:10FFA000FBF750FEFBF7F8FFFCF744F8FCF718F8F6
:10FFB000FCF75CF9FCF77CF9FCF784F8FCF7D0F867
:10FFC00000F08EF8FBF7C4FE00F0DAF8FFE7FEE77A
:10FFD00080B584B00290EFF305800390039820B1C0
:10FFE000FFE76FF00500019009E000200190029802
:10FFF00020B1FFE7029802F0B7F8FFE7FFE70198AA
:020000040801F1
:1000000004B080BD80B586B00490EFF30580059004
:10001000059820B1FFE76FF0050001901BE000207C
:10002000019003F073FD039004980399401A029025
:10003000029858B1FFE702990020B0EBD17F05D1BB
:10004000FFE7029903A802F0C7F803E06FF003008E
:100050000190FFE7FFE7019806B080BD80B582B050
:1000600003F038FD0146009158B1FFE700980128E0
:100070000AD0FFE70098022807D1FFE7022001908D
:1000800012E0032001900FE0FFE740F26050C2F25F
:1000900000000068012803D1FFE70120019002E081
:1000A00000200190FFE7FFE7019802B080BD00004B
:1000B00080B582B0EFF305800190019820B1FFE791
:1000C00003F02EFD009003E003F020FD0090FFE719
:1000D000009802B080BD00004FF47A7070470000B5
:1000E00082B0EFF305800190019820B1FFE76FF037
:1000F0000500009014E040F26050C2F20000006879
:1001000048B9FFE740F26051C2F2000101200860E7
:100110000020009003E04FF0FF300090FFE7FFE782
:10012000009802B07047000080B584B0EFF30580FE
:100130000390039820B1FFE76FF0050002901BE0E9
:1001400003F0C8FC0146019140B1FFE70198012886
:100150000CD0FFE70198022803D008E001200290AC
:1001600009E002F0BBFA0020029004E0FFE74FF044
:10017000FF300290FFE7FFE7029804B080BD000067
:1001800080B582B0EFF305800190019820B1FFE7C0
:100190006FF00500009019E040F26050C2F20000DC
:1001A000006801280DD1FFE7FDF7C4F840F2605167
:1001B000C2F200010220086002F020FA0020009044
:1001C00003E04FF0FF300090FFE7FFE7009802B038
:1001D00080BD000080B584B0EFF3058003900398E4
:1001E00020B1FFE76FF00500029027E003F072FCFA
:1001F0000146019140B1FFE70198012818D0FFE7BF
:100200000198022811D014E00120029003F04CFF65
:10021000012809D0FFE703F05DFC20B9FFE74FF0AC
:10022000FF300290FFE7FFE707E00020029004E0C4
:10023000FFE74FF0FF300290FFE7FFE7029804B0BE
:1002400080BD000080B588B00690059104920393AC
:100250000698029000200190EFF305800790079820
:1002600068B3FFE7029830B1FFE7059818B1FFE7E0
:10027000039820B1FFE76FF0030001901EE000201B
:100280000090029805996A4602F08CFF012804D07C
:10029000FFE76FF0020001900FE0009860B1FFE708
:1002A0004EF60451CEF200014FF080500860BFF3CB
:1002B0004F8FBFF36F8FFFE7FFE7FFE71FE0029865
:1002C00018B1FFE7059820B9FFE76FF00300019030
:1002D00014E002980599039A02F076FE01280CD0EA
:1002E000FFE7039820B1FFE76FF00100019003E002
:1002F0006FF002000190FFE7FFE7FFE7FFE70198DB
:1003000008B080BD80B588B00690059104920020A9
:100310000390EFF305800790079800286ED1FFE760
:10032000069800286AD0FFE70598002866D0FFE706
:100330004FF0FF300290049868B3FFE7049880689C
:10034000A0B1FFE70498C06850280FD3FFE70498D6
:10035000006958B1FFE7049840690699059A51432E
:10036000884203D3FFE70120029013E004988068DD
:1003700078B9FFE70498C06858B9FFE704980069A6
:1003800038B9FFE70498406918B9FFE700200290E8
:10039000FFE7FFE702E000200290FFE70298012854
:1003A0000ED1FFE706980599049A93681269EE4604
:1003B0004FF0000CCEF800C002F02EFB03900AE0D4
:1003C000029838B9FFE706980599002202F0EAFA88
:1003D0000390FFE7FFE7039878B1FFE7049820B1A7
:1003E000FFE704980068019002E000200190FFE719
:1003F0000398019901F05CFEFFE7FFE7039808B05E
:1004000080BD000080B588B0069005918DF813205E
:1004100003930698029000200190EFF30580079067
:10042000079868B3FFE7029830B1FFE7059818B165
:10043000FFE7039820B1FFE76FF0030001901EE093
:1004400000230093029805996A4602F0E1FC012816
:1004500004D0FFE76FF0020001900FE0009860B158
:10046000FFE74EF60451CEF200014FF080500860D5
:10047000BFF34F8FBFF36F8FFFE7FFE7FFE720E08A
:10048000029818B1FFE7059820B9FFE76FF0030065
:10049000019015E002980599039A002302F0A2FB4F
:1004A00001280CD0FFE7039820B1FFE76FF00100AF
:1004B000019003E06FF002000190FFE7FFE7FFE724
:1004C000FFE7019808B080BD80B584B00290029823
:1004D0000190EFF305800390039820B1FFE76FF0E0
:1004E000050000900DE0019820B9FFE76FF00300D0
:1004F000009005E000210091019802F015FBFFE754
:10050000FFE7009804B080BD80B586B004900391E9
:10051000049820F001000290049800F0010000907F
:1005200000200190EFF305800590059820B1FFE7CA
:100530006FF00500019033E0029820B9FFE76FF0FB
:10054000030001902BE00098A0B1FFE70298039907
:1005500002F0C2FF01280CD0FFE7039820B1FFE7AB
:100560006FF00100019003E06FF002000190FFE7DF
:10057000FFE713E00298039902F098FE01280CD0DF
:10058000FFE7039820B1FFE76FF00100019003E05F
:100590006FF002000190FFE7FFE7FFE7FFE7FFE7EB
:1005A000019806B080BD000080B588B0069000209C
:1005B0000590EFF3058007900798002840F08580AC
:1005C000FFE7069820B1FFE706984068049002E034
:1005D00000200490FFE79DF81000C00718B1FFE766
:1005E0000120039002E000200390FFE7049800F050
:1005F0000800082868D0FFE74FF0FF300290069807
:10060000C8B1FFE70698806840B1FFE70698C06868
:10061000502803D3FFE7012002900BE00698806882
:1006200038B9FFE70698C06818B9FFE700200290C4
:10063000FFE7FFE702E000200290FFE702980128B1
:1006400012D1FFE7039838B1FFE7069881680420CC
:1006500002F08EF9059006E006988168012002F00C
:1006600087F90590FFE711E0029870B9FFE703985A
:1006700028B1FFE7042002F067F9059004E00120AB
:1006800002F062F90590FFE7FFE7FFE7059878B110
:10069000FFE7069820B1FFE706980068019002E0A6
:1006A00000200190FFE70598019901F001FDFFE7A7
:1006B000059840B1FFE7039828B1FFE7059840F09F
:1006C00001000590FFE7FFE7FFE7059808B080BD50
:1006D00080B586B00490049820F00100039004983F
:1006E00000F00100019000200290EFF305800590DA
:1006F000059820B1FFE76FF00500029024E0039811
:1007000020B9FFE76FF0030002901CE0019858B198
:10071000FFE7039802F022FC012804D0FFE76FF006
:1007200002000290FFE70DE00398002319461A46E5
:1007300002F058FA012804D0FFE76FF0020002909F
:10074000FFE7FFE7FFE7FFE7029806B080BD000084
:1007500080B58AB00890079108980690069830B145
:10076000FFE79DF81F000006002804D5FFE76FF0A3
:10077000030005903BE04FF0FF300590EFF305805C
:100780000990099820B3FFE7002303930493069888
:100790000799EC4604AACCF80020012203F0AEF839
:1007A000039A069869460A6005AB114603F0A6F85D
:1007B000049860B1FFE74EF60451CEF200014FF00D
:1007C00080500860BFF34F8FBFF36F8FFFE70DE0DE
:1007D0000698079901220023029302F0D3FF029AA0
:1007E000069805AB114602F0CDFFFFE7FFE705983D
:1007F0000AB080BD80B58CB00A9009910892EFF3E1
:1008000005800B900B9820B1FFE76FF00500079073
:100810007AE09DF82B000006002804D5FFE76FF072
:10082000030007906FE09DF824008007002803D59F
:10083000FFE70020059002E00A980590FFE70020FE
:1008400007900898029003F061F90490FFE705997A
:10085000029B002006AA03F055FA01900198012896
:100860003FD1FFE70A990798084007900699079833
:10087000084307909DF82400C00780B1FFE70A995C
:1008800007980840884201D1FFE73BE0089820B96B
:10089000FFE76FF00200079034E0FFE70EE00A98F0
:1008A0000799084201D0FFE72CE0089820B9FFE73C
:1008B0006FF00200079025E0FFE7FFE703F026F95D
:1008C0000499401A039003980299884203D9FFE7DC
:1008D0000020029004E003990298401A0290FFE77A
:1008E0000BE0089820B9FFE76FF00200079003E0E3
:1008F0006FF001000790FFE7FFE7FFE7019800288E
:10090000A5D1FFE7FFE7FFE707980CB080BD000027
:1009100080B582B003F0D4F80190019802B080BD98
:10092000B0B58EB00B900A91099200200690EFF3BB
:1009300005800D900D98002840F09980FFE70B98F6
:10094000002800F09480FFE7802007901820059091
:10095000002008904FF0FF300490099800284DD0F7
:10096000FFE70998006820B1FFE709980068089040
:10097000FFE70998806920B1FFE709988069059031
:10098000FFE7059848B1FFE70598382805D8FFE745
:1009900009980079C00718B1FFE700200C9069E0C2
:1009A0000998406928B1FFE70998406980080790D5
:1009B000FFE70998806880B1FFE70998C0685C2864
:1009C0000BD3FFE70998006938B1FFE70998406940
:1009D00018B1FFE7012004900FE00998806858B92A
:1009E000FFE70998C06838B9FFE70998006918B9A6
:1009F000FFE700200490FFE7FFE702E000200490FB
:100A0000FFE70498012817D1FFE70B980899079A88
:100A10000A9BDDF814C0DDF824E0DEF80850DEF8AB
:100A20001040EE46CEF80850CEF80440CEF800C094
:100A300002F040FE069019E00498B0B9FFE70B9869
:100A40000899BDF81C200A9BDDF814C0EE4606ACE0
:100A5000CEF80440CEF800C002F0DCFD012803D03F
:100A6000FFE700200690FFE7FFE7FFE7FFE70698B4
:100A70000C90FFE70C980EB0B0BD000080B586B0BA
:100A8000049004980390EFF305800590059820B139
:100A9000FFE76FF0050002901CE0039820B9FFE724
:100AA0006FF00300029014E00398FFF7C3F98DF88C
:100AB00007009DF80700042806D0FFE700200290F9
:100AC000039801F013FC03E06FF002000290FFE7CF
:100AD000FFE7FFE7029806B080BD000080B584B054
:100AE0000390029148F6A060C2F2000000680090F6
:100AF00041F28020C2F200000068043001F0ECF8FE
:100B000008B9FFE700E0FFE70398013080B9FFE78D
:100B1000029868B1FFE741F28020C2F2000000684D
:100B2000011D48F67860C2F2000001F07BF93DE05B
:100B30000098039908440190019841F28021C2F283
:100B40000001096848600198009988420ED2FFE7C9
:100B500041F29020C2F20000006841F28021C2F20E
:100B600000010968043101F027F91EE041F28820F4
:100B7000C2F20000006841F28021C2F2000109685F
:100B8000043101F019F9019848F60461C2F200013C
:100B90000968884207D2FFE7019848F60461C2F26B
:100BA0000001086000E0FFE7FFE7FFE704B080BD59
:100BB00080B582B0019001F05DF948F2D861C2F2CF
:100BC000000108680130086041F28020C2F2000094
:100BD000006898B9FFE7019841F28021C2F2000154
:100BE000086048F2D860C2F200000068012803D112
:100BF000FFE700F021FB00E0FFE71CE048F66C6037
:100C0000C2F200000068A0B9FFE741F28020C2F202
:100C100000000068C06A0199C96A884207D8FFE7E6
:100C2000019841F28021C2F20001086000E0FFE774
:100C300000E0FFE7FFE748F2E460C2F2000001686D
:100C4000013101600068019948640198C06A48F266
:100C5000E861C2F200010968884208D9FFE70198FB
:100C6000C06A48F2E861C2F200010860FFE701993A
:100C7000C86A00EB800241F29820C2F2000000EB4B
:100C80008200043101F0CEF801F020F948F66C60E2
:100C9000C2F200000068C8B1FFE741F28020C2F252
:100CA00000000068C06A0199C96A88420CD2FFE757
:100CB0004EF60451CEF200014FF080500860BFF3B1
:100CC0004F8FBFF36F8F00E0FFE700E0FFE702B058
:100CD00080BD000080B584B001F0CCF848F6A46077
:100CE000C2F200000068002840D1FFE748F6A45097
:100CF000C2F20000029001F03FF848F6B850C2F28C
:100D00000000039001F038F80299039841F2842220
:100D1000C2F20002116041F29421C2F200010860A7
:100D200069460020086041F28C12C2F2000241F2D2
:100D30002C23C2F200030A20102101F06DFE0146AF
:100D400048F6A460C2F200000160006860B1FFE7ED
:100D500048F6A460C2F20000006846F2AD11C0F689
:100D6000010101F0A5F900E0FFE700E0FFE701F075
:100D7000ADF804B080BD000080B582B0FFE748F256
:100D8000DC60C2F20000006808B3FFE701F072F80F
:100D900048F68C60C2F20000C068C06801900198FB
:100DA000043000F099FF48F2D861C2F200010868EF
:100DB0000138086048F2DC61C2F2000108680138BD
:100DC000086001F083F8019800F08CF8D7E702B0D2
:100DD00080BD000080B582B0019000910198006C48
:100DE000B8B1FFE70199C8680A6C1044C86001985F
:100DF0008168C068884204D3FFE701990868C86029
:100E000000E0FFE70098019AD168126CEFF7FEFA54
:100E1000FFE702B080BD000080B586B00590049168
:100E20000392002002900598806B01900598006C59
:100E300078B9FFE70598006848B9FFE7059880682A
:100E400002F0CCFF029005990020886000E0FFE7E7
:100E500041E00398B8B9FFE7059A04995068126C0D
:100E6000EFF7D4FA059948680A6C10444860059970
:100E700048688968884204D3FFE705990868486094
:100E800000E0FFE726E0059A0499D068126CEFF7BE
:100E9000BDFA0599C8680A6C801AC860059801688F
:100EA000C068884206D2FFE7059988680A6C801AF4
:100EB000C86000E0FFE70398022809D1FFE7019826
:100EC00020B1FFE701980138019000E0FFE700E062
:100ED000FFE7FFE7FFE70198013005998863029873
:100EE00006B080BD80B582B00090009890F859009F
:100EF00040B9FFE70098006B01F00EF8009801F090
:100F00000BF81CE0009890F85900012804D1FFE785
:100F1000009801F001F811E0009890F859000228BB
:100F20000BD0FFE74FF0500080F31188BFF36F8FB5
:100F3000BFF34F8F0190FFE7FEE7FFE7FFE702B047
:100F400080BD000082B001900198406A38B1FFE78F
:100F50000198006B0068C0F13800009002E00020AA
:100F60000090FFE7009802B07047000082B0019047
:100F700041F28420C2F2000000680068B0FA80F0FC
:100F80004009019908600198006848B9FFE741F2FB
:100F90008420C2F200000068C0680068009002E08F
:100FA00000200090FFE7009802B0704784B04FF433
:100FB000C040009042F2CC60C2F2000001909DF867
:100FC0000400400788B1FFE70198073001900198BD
:100FD00020F007000190019A42F2CC61C2F20001B8
:100FE0000098891A08440090FFE70198029002993E
:100FF00048F67060C2F20000016000214160029872
:10100000009A10440190019808380190019820F04E
:1010100007000190019A41F28C20C2F200000260A8
:101020000268516002681160029903910199039A64
:10103000891A51600068039908600398406848F66F
:101040000061C2F2000108600398406848F6F85158
:10105000C2F20001086048F6CC51C2F200014FF024
:101060000040086004B0704780B582B00190FFE78F
:10107000FFF782FE41F29820C2F2000000680228C9
:101080000CD3FFE74EF60451CEF200014FF0805032
:101090000860BFF34F8FBFF36F8F00E0FFE7E7E714
:1010A00080B582B00190019868B1FFE701980023F4
:1010B0008360019803600198C360019819461A463D
:1010C00001F090FD00E0FFE702B080BD80B584B084
:1010D000DDF818C00390029101928DF80330029858
:1010E00018B9FFE70698006003E0019806990860C8
:1010F000FFE703980699C863029806990864069862
:10110000012101F011FD9DF80300069981F84C00C2
:1011100004B080BD80B588B0DDF834C0DDF830C0E3
:10112000DDF82CC0DDF828C00690059104920393E9
:101130000C98006B04998900A522EFF7DEF90C9852
:10114000006B049900EB810004380290029820F0B3
:10115000070002909DF80800400758B1FFE74FF0E4
:10116000500080F31188BFF36F8FBFF34F8F07904C
:10117000FFE7FEE70598F8B1FFE700200190FFE7E1
:1011800001980F2813D8FFE70598019A805C0C9905
:10119000114481F8340005980199405C08B9FFE7D3
:1011A00005E0FFE7FFE7019801300190E8E70C99BF
:1011B000002081F8430004E00C99002081F83400FD
:1011C000FFE70A98382803D3FFE737200A9000E0AA
:1011D000FFE70A980C99C8620A980C99C8640C99A0
:1011E0000020009008650C98043000F0DDFD0C989C
:1011F000183000F0D9FD00980C9909610A99C1F1E5
:1012000038010C9A91610C9949620C9948650C99C6
:1012100081F8580002980699039A00F0E7FC0C99AF
:1012200008600B9820B1FFE70C980B99086000E06C
:10123000FFE708B080BD000080B584B000200390B7
:10124000FFE70398372810D8FFE7039800EB8001E9
:1012500041F29820C2F2000000EB810000F08CFD0A
:10126000FFE7039801300390EBE748F6D050C2F255
:101270000000019000F080FD48F6E450C2F200004A
:10128000029000F079FD48F61860C2F2000000F00C
:1012900073FD48F68C60C2F2000000F06DFD48F668
:1012A0007860C2F2000000F067FD0199029841F2F7
:1012B0008822C2F20002116041F29021C2F20001C4
:1012C000086004B080BD000083B0029048F67060F2
:1012D000C2F200000190FFE701980068029988427D
:1012E00005D2FFE7FFE7019800680190F4E7019855
:1012F000009000980199496808440299884209D1F0
:10130000FFE70298426801994868104448600198D4
:10131000029000E0FFE70298009000980299496867
:10132000084401990968884220D1FFE701980068C4
:1013300041F28C21C2F20001096888420DD0FFE71A
:101340000198006842680299486810444860019812
:10135000006800680299086007E041F28C20C2F240
:101360000000006802990860FFE704E00198006847
:1013700002990860FFE701980299884204D0FFE7CC
:1013800002980199086000E0FFE703B07047000091
:1013900080B586B0059004910392029300200190DD
:1013A000049805994860059800610498039988425B
:1013B00016D8FFE703980299401A0599896988426F
:1013C00003D3FFE70120019009E041F29420C2F22B
:1013D000000000680599043100F0EEFCFFE717E01B
:1013E00003980299884208D2FFE70498029988423C
:1013F00003D3FFE70120019009E041F28420C2F20B
:10140000000000680599043100F0D6FCFFE7FFE713
:10141000019806B080BD000080B582B0019000F058
:1014200029FD0198806B18B9FFE70120009002E0C8
:1014300000200090FFE700F049FD009802B080BD59
:1014400080B582B0019000F015FD0198806B019984
:10145000C96B884203D1FFE70120009002E0002021
:101460000090FFE700F032FD009802B080BD000060
:1014700008480068006880F308884FF0000080F397
:10148000148862B661B6BFF34F8FBFF36F8F00DF72
:1014900000BF00BF08ED00E080B586B00490039166
:1014A00041F28420C2F200000068C068C068019068
:1014B0000198043000F010FC019890F828004007D3
:1014C000002823D5FFE70198049B81691944039AFA
:1014D000FFF75EFFC0B1FFE70198049A6946002359
:1014E0000B60194602F0EEFE0290029858B9FFE731
:1014F0004FF0500080F31188BFF36F8FBFF34F8F11
:101500000590FFE7FEE700E0FFE707E0019991F8AB
:10151000280000F0FE0081F82800FFE70198016A2A
:10152000884706B080BD000080B58EB0FFE748F662
:10153000A460C2F20000006807A9002201F044FD87
:10154000002800F0B880FFE70798B0F1FF3F17DCF4
:10155000FFE707A804300290029858B9FFE74FF060
:10156000500080F31188BFF36F8FBFF34F8F0B9044
:10157000FFE7FEE702990A6848688968904700E03B
:10158000FFE70798002800F19580FFE7099806908B
:101590000698406928B1FFE70698043000F09CFBEC
:1015A00000E0FFE705A800F0FBF803900798019022
:1015B000092800F27D800199DFE801F00505053D6D
:1015C000456605053D45069991F8280040F0010063
:1015D00081F828000698089B81691944039AFFF74F
:1015E000D7FE30B3FFE70698016A8847069890F85F
:1015F0002800400700281AD5FFE706980899826955
:101600000A44694600230B60194602F05BFE049011
:10161000049858B9FFE74FF0500080F31188BFF3EA
:101620006F8FBFF34F8F0C90FFE7FEE700E0FFE7FF
:1016300000E0FFE73DE0069991F8280000F0FE0089
:1016400081F8280035E0069991F8280040F0010063
:1016500081F828000898069988610698806958B929
:10166000FFE74FF0500080F31188BFF36F8FBFF397
:101670004F8F0D90FFE7FEE70698039B81691944A1
:101680001A46FFF785FE14E0069890F828008007B8
:10169000002804D4FFE7069800F03EFC07E0069916
:1016A00091F8280000F0FE0081F82800FFE700E034
:1016B000FFE7FFE73BE70EB080BD000080B584B0D8
:1016C0000390029101F00AF8684600F069F8019071
:1016D0000098D8BBFFE7029860B9FFE7039801992B
:1016E000884207D8FFE702F0DFFC03980199FFF773
:1016F000D3FE2AE0029858B1FFE741F29420C2F2EB
:10170000000000680068B0FA80F040090290FFE72E
:1017100048F6A460C2F2000000680399019A891A91
:10172000029A00F0EFFC02F0BFFC60B9FFE74EF652
:101730000451CEF200014FF080500860BFF34F8F8C
:10174000BFF36F8F00E0FFE7FFE702E002F0ACFCC1
:10175000FFE704B080BD000081B041F28820C2F2F2
:1017600000000068006840B9FFE748F60461C2F273
:1017700000014FF0FF3008600FE041F28820C2F214
:1017800000000068C068C06800900098406848F693
:101790000461C2F200010860FFE701B07047000079
:1017A00080B582B0019002F0B1F90090009841F24A
:1017B0007C21C2F200010968884206D2FFE700F0EE
:1017C00011F801990120086003E0019900200860E8
:1017D000FFE7009841F27C21C2F200010860009806
:1017E00002B080BD80B588B0FFE741F28420C2F22C
:1017F00000000068006800284ED0FFE741F2842016
:10180000C2F200000168C968096806910068C068F2
:10181000C06803900398043000F05EFA0398016AF0
:101820008847039890F828004007002832D5FFE742
:101830000698039989690844059005980699884295
:101840000FD9FFE70598039948600398006141F2BA
:101850008420C2F2000000680399043100F0ACFA61
:1018600017E00398069A694600230B60194602F0B8
:1018700029FD0290029858B9FFE74FF0500080F31D
:101880001188BFF36F8FBFF34F8F0790FFE7FEE71D
:10189000FFE700E0FFE7A8E741F28422C2F200027E
:1018A0001068049041F29421C2F2000108681060AF
:1018B0000498086008B080BD83B00020009040F21A
:1018C0006C30C2F200000068013058B1FFE74FF001
:1018D000500080F31188BFF36F8FBFF34F8F0190DB
:1018E000FFE7FEE74FF0500080F31188BFF36F8FE2
:1018F000BFF34F8F0290FFE7009808B9FFE7FBE7BF
:1019000003B0704780B584B00390FFE701A8FFF7EC
:101910002DFB029002980199FFF7D0FEFFF704FE1D
:10192000F4E7000080B582B0019000F0A3FA0198BE
:1019300090F845008DF80300FFE79DF903000128AA
:1019400016DBFFE70198406A58B1FFE701982430A1
:1019500002F042FB18B1FFE700F062FD00E0FFE794
:1019600000E005E09DF8030001388DF80300E4E78E
:101970000199FF2081F8450000F0A8FA00F07AFAFA
:10198000019890F844008DF80200FFE79DF90200ED
:10199000012816DBFFE70198006980B1FFE7019895
:1019A000103002F019FB18B1FFE700F039FD00E03C
:1019B000FFE79DF8020001388DF8020000E000E02A
:1019C000E4E70199FF2081F8440000F07FFA02B0BB
:1019D00080BD000080B58AB006900020029000F023
:1019E0007DFE41F28C20C2F20000006818B9FFE7CA
:1019F000FFF7DCFA00E0FFE7069848F6CC51C2F2A8
:101A000000010968084240F0C580FFE7069800B36E
:101A1000FFE70698083006909DF818004007B0B11F
:101A2000FFE7069820F00700083006909DF81800A0
:101A3000400758B1FFE74FF0500080F31188BFF323
:101A40006F8FBFF34F8F0790FFE7FEE700E0FFE7E0
:101A500000E0FFE70698002800F09A80FFE706986C
:101A600048F6F851C2F200010968884200F29080FD
:101A7000FFE748F67060C2F200000490006805902D
:101A8000FFE705984168069A00209142019007D22D
:101A9000FFE705980068002818BF01200190FFE7C4
:101AA0000198C00730B1FFE70598049005980068D9
:101AB0000590E6E7059841F28C21C2F20001096821
:101AC000884263D0FFE704980068083002900598C8
:101AD000006804990860059840680699401A112822
:101AE00021D3FFE705980699084403909DF80C0060
:101AF000400758B1FFE74FF0500080F31188BFF363
:101B00006F8FBFF34F8F0890FFE7FEE7059840689F
:101B10000699401A03994860069805994860039809
:101B2000FFF7D2FB00E0FFE70598426848F6F8505F
:101B3000C2F200000168891A0160006848F600617D
:101B4000C2F20001096888420BD2FFE748F6F8505C
:101B5000C2F20000006848F60061C2F200010860AD
:101B600000E0FFE748F6CC50C2F200000268059999
:101B700048681043486005990020086048F60C61E9
:101B8000C2F2000108680130086000E0FFE700E0F1
:101B9000FFE700E0FFE702F087FA9DF80800400742
:101BA00058B1FFE74FF0500080F31188BFF36F8FFB
:101BB000BFF34F8F0990FFE7FEE702980AB080BDA0
:101BC00041F28020C2F20000006848B1FFE741F214
:101BD0008020C2F200000168086D01300865FFE74F
:101BE00041F28020C2F200000068704783B002908A
:101BF0000191009202980438029002994FF080708F
